:020000040800F2
:1000000000000420A16F0108A16F0108A16F010881
:10001000A16F0108A16F0108A16F01080000000095
:10002000000000000000000000000000A16F0108B7
:10003000A16F010800000000A16F0108A16F010875
:10004000A16F0108A16F0108A16F0108A16F01084C
:10005000A16F0108A16F0108A16F0108A16F01083C
:10006000A16F0108A16F0108A16F0108A16F01082C
:10007000A16F0108A16F0108A16F0108A16F01081C
:10008000A16F0108A16F0108A16F0108A16F01080C
:10009000A16F0108A16F0108A16F0108A16F0108FC
:1000A000A16F0108A16F0108A16F0108A16F0108EC
:1000B000397A0008A16F0108A16F0108A16F01083A
:1000C000A16F0108A16F0108A16F0108A16F0108CC
:1000D000A16F0108A16F0108A16F010835C30008D5
:1000E000A16F0108A16F0108A16F0108A16F0108AC
:1000F000A16F0108A16F0108A16F0108A16F01089C
:10010000A16F0108A16F0108A16F0108A16F01088B
:10011000A16F0108E5C30008A16F0108A16F0108E4
:10012000A16F0108A16F0108A16F0108A16F01086B
:10013000A16F0108A16F0108A16F0108A16F01085B
:10014000A16F0108A16F0108A16F0108A16F01084B
:10015000A16F0108A16F0108A16F0108A16F01083B
:10016000A16F0108A16F0108A16F0108A16F01082B
:10017000A16F0108A16F0108A16F01080000000034
:10018000A16F0108A16F0108A16F0108A16F01080B
:10019000A16F0108A16F0108A16F0108A16F0108FB
:1001A000A16F0108A16F0108A16F0108A16F0108EB
:1001B000A16F0108A16F0108A16F0108A16F0108DB
:1001C000A16F0108A16F010800000000A16F0108E4
:1001D000A16F0108A16F0108A16F0108A16F0108BB
:1001E000A16F0108A16F0108A16F0108A16F0108AB
:1001F000A16F0108A16F01080348044B834202D09C
:10020000034B03B1184770477C0900207C0900208C
:100210000000000005480649091A891001EBD17158
:10022000491002D0034B03B1184770477C090020E6
:100230007C0900200000000010B5064C237843B96B
:10024000FFF7DAFF044B13B10448AFF3008001233A
:10025000237010BD80090020000000000C28050854
:1002600008B5044B1BB104490448AFF30080BDE856
:100270000840CFE700000000840900200C28050892
:10028000A3F5803A704700BF154B002B08BF114BF8
:100290009D46FFF7F5FF00218B460F461148124A95
:1002A000121A17F0FDFE0C4B002B00D098470B4B99
:1002B000002B00D098470020002104000D000B48BF
:1002C00017F0ECFD17F01EFE2000290008F058FB87
:1002D00017F0EAFD00000800000000000000000028
:1002E00000000000800900204C140120D17E01088C
:1002F000F8B504460D4600F036FA04F5CC772946E9
:1003000004F5987000F006FC002304F509713A46E4
:10031000A4F88C31C4E9643322F8023B8A42FBD151
:100320004FF0000204F50E76C4F824320025A4F83C
:10033000283284F82A2204F52272A4F82C32C4E967
:100340008C33334643F8045B9A42FBD14FF48073FD
:10035000C4F88C52C4F890520B20A4F888320023C1
:10036000C4F8985284F89432A4F8AC3284F8AE32CF
:10037000C4F8B03284F8B432C4F89C52C4F8A05225
:10038000C4F8A452C4F8A85217F052FD3023C4F8A0
:1003900024022046A4F88C310B4BC4F89071C4F8A9
:1003A00094310723C4F83062A4F82C32074BC4F808
:1003B0009852C4F83432C4F89C52C4F8A052C4F81D
:1003C000A452C4F8A852F8BD040000206400002024
:1003D00030B5B0F828220346D0F82442551CA05C62
:1003E000A3F82852A154B3F828220A2A84BF002275
:1003F000A3F8282230BD90F82A3280F82A125B1A1E
:1004000058425841704738B5B0F8AC2204460D4602
:10041000052A03D149B3012380F8AE32002DB4F888
:10042000B03216BF80210021551C41EA5301B4F8B7
:10043000B23218BFADB20133A4F8B012A4F8AC5276
:100440009BB294F8AE52A4F8B2324DB37E2912D0CA
:10045000FE294FF000050CD1A4F82C5184F8B452B9
:1004600084F8AE52A4F8B25203E084F8AE12A4F8B5
:10047000AC12284638BDB4F82C31102B04D92046D4
:1004800000F08CF9054610B90025A4F82C51012381
:1004900084F8B432002384F8AE32A4F8B232E8E72C
:1004A00094F8B422012A04D0022AE2D1082BE0D128
:1004B00004E0082BDDD1022384F8B432204600F09A
:1004C0005FF9CFE700F5987000F016BBD0EDA47A85
:1004D0009FED0A7AF4EEC77AF1EE10FA05D80123FF
:1004E00080F8943290F894027047B0EE087AF4EEF7
:1004F000C77AF1EE10FAF5DB0023F1E79999193F7D
:10050000D0F8A43200F52B721649C0F8A832D0F802
:10051000A032C0F8A432D0F89C32C0F8A032D0F893
:10052000983280EDA60AC0F89C3200F52773B3EC30
:10053000017AF1EC016AD0EDA67A9342E6EEC77A31
:10054000C0EDA67AF3D1084B00F526709FED070A9F
:10055000F0EC017AB3EC017A9042A7EE270AF7D1CA
:10056000704700BFC4860108D4860108000000005F
:1005700010B52DED028B90F8882282B0044690F8D9
:1005800089328A42D0EDA37AB2EE047A01D1102BDF
:1005900045D9F4EEC77A9FED2F8AB1EE040A84F8AC
:1005A000881201AA6946F1EE10FA04F50B70C2BF79
:1005B000B3EE047A77EEC77AC4EDA37A07EE903AE9
:1005C000D4EDA36A102BF8EE677A4FF0010388BFD1
:1005D000B0EE408A86EEA77A8DED007A17F096F895
:1005E0009DED000A2046B5EEC00AF1EE10FA4CBFB0
:1005F00038EE400A30EE080AFFF782FFB6EE007AC6
:10060000D4EDA37A0123DDED016A84EDA40AE6EEC0
:10061000C77A84F88932C4EDA37A00200EE0F4EEA4
:10062000C77AF1EE10FAF8DDB3EE047A013380F800
:10063000893277EEC77AC0EDA37A0120B7EE007A4F
:10064000D4EDA37A77EE877AC4EDA37A02B0BDEC3D
:10065000028B10BD000000002DE9F04F85B04FF077
:10066000000A054617460DF104090DF108081E465B
:1006700000F5987002234A4600F03CFA574511D025
:1006800039F81A402846E443C4F3C0342146FFF742
:100690009FFE6040C0B24000013828F81A000AF1FD
:1006A000010AEBE741464FF000080DF10C0A022366
:1006B000C146C346524605F5C67016F0C3FEB8459E
:1006C0002FD03AF818402846E443C4F3C0342146FA
:1006D000FFF74EFF60B195F82A12284685F82A42A6
:1006E0000B1B59425941B9F1000F04D0FFF78BFEA3
:1006F00008F10108E3E7FFF786FE81460028F7D0FE
:100700004FF496722946304617F030FCB5F82C317C
:10071000A6F82C31B5F82E31A6F82E31A5F82CB15B
:10072000E6E7484605B0BDE8F08F30B50023044643
:1007300000F5967504F8013BAC42FBD1A0F82C31D2
:10074000A0F82E3100239CB2A2420BD9B3F5957FBD
:1007500008D0B0F82C41651CA0F82C51CD5C0133B9
:100760000555F0E730BD024600F59671002302F80A
:10077000013B9142FBD1A0F82C31A0F82E317047FB
:10078000B0F82C31B3F5967F1FBF5A1CA0F82C216E
:10079000C154012008BF00207047000070B5B0F8B8
:1007A0002C114FF0FF330022104E8C1E551C92B2BC
:1007B000944209D9825C5A40C3F30723D2B236F877
:1007C000122053402A46F1E7DB43045D9BB2DAB2C4
:1007D000944209D1014411F8012CB2EB132F03D13B
:1007E000A0F82E31012070BD0020FCE7E88601084A
:1007F000B0F82C214FF0FF3370B5044616180D4D9C
:10080000B44209D014F8011B5940C3F30723C9B2FD
:1008100035F811104B40F3E7DB43911C9BB2A0F875
:100820002E3183540132C3F30723A0F82C1192B266
:10083000835470BDE886010870B5002500F10C06F0
:10084000044600F5A6730580C0E90155304620F83E
:10085000025B9842FBD10321FFF74AFD062104F217
:100860000440FFF745FD092104F2BC60FFF740FD9D
:100870008223A4F87459204623800A4B6660A36043
:100880001E23C4F87859C4F87C39074BC4F8805942
:10089000C4F884394BF24033A4F888390F2384F824
:1008A0008A3970BD800000208000000190F8860920
:1008B00070472DE9F041CEB20F4605461446F11EB1
:1008C00000F5A6709846C4EB041449B2FFF7FAFD90
:1008D000394605F204402401FFF7F4FDF11C05F24E
:1008E000BC6049B2FFF7EEFDC5F87C4985F8848904
:1008F000BDE8F08190F88A1990F8883990F8872936
:100900004B40534090F889291A4480F88839D2B274
:1009100080F8892901EB5202534080F88A397047E8
:1009200090F8873990F88A1990F8882901334A405D
:10093000DBB280F88739534090F8892980F88839EC
:100940001A44D2B280F8892901EB52025340DBB23B
:1009500080F88A39184670472DE9F041CEB0044638
:100960009046022301AA04F5A67716F06BFDD4F891
:10097000783902A80133C4F87839FFF7F4FE02ABE6
:10098000424601A93846FFF767FED0B1BDF83631BF
:10099000B4F874299A4203D1D4F87829022A0CD9E0
:1009A000BDF8342102A9A4F874390023023A4C4856
:1009B000C4F8783992B20AF0E5FA4A4948480AF090
:1009C00095FB04F2044602AB424601A93046FFF70C
:1009D00043FED0B1BDF83631B4F874299A4203D140
:1009E000D4F87829022A0CD9BDF8342102A9A4F838
:1009F00074390023023A3A48C4F8783992B20AF0BE
:100A0000C1FA394936480AF071FB04F2BC6502AB01
:100A1000424601A92846FFF71FFED0B1BDF8363186
:100A2000B4F874299A4203D1D4F87829022A0CD94F
:100A3000BDF8342102A9A4F874390023023A2848E9
:100A4000C4F8783992B20AF09DFA284924480AF08D
:100A50004DFBD4F88039D4F87C2902339342C4F892
:100A6000803922D300233846C4F88039FFF72EFDA1
:100A700007463046FFF72AFD06462846FFF726FDC3
:100A800094F8853905460FB906B988B153B90121E3
:100A9000174806F06DFA0121154806F075FA012392
:100AA00084F88539002384F886394EB0BDE8F0819A
:100AB0004BB101460E4806F05BFA29460C4806F099
:100AC00063FA84F8855994F884592046FFF728FF83
:100AD000854234BF0020012084F88609E5E700BF85
:100AE000C0D90020E8880108FB8801080E890108A8
:100AF000708A002016F0A6BC03460922063123F8AE
:100B00000C2BC9B24360024B53F82130836070470D
:100B100084010020002300F10C0210B5044603807C
:100B2000C0E901335C3022F8023B9042FBD1204601
:100B3000FFF7E2FF10BD024600F51671002302F830
:100B4000013B9142FBD14FF4B472A0F85832A0F8A7
:100B50005A32A0F85C22A0F85E3280F8603270470A
:100B6000F0B58DB0B0F85E321424104F02AE3246AC
:100B700037F91350B9B1AD1006339BB2013C6D107B
:100B8000772B26F8025B84BF783B9BB214F0FF04FE
:100B9000EED1A0F85E320B2114230548009406F034
:100BA000BFFD0DB0F0BD0B33E7E700BF3289010890
:100BB000708A002070B5B0F858320446002B31D04E
:100BC000194B1B782BB3194806F0B4F9184E05469B
:100BD000142D27D9B4F85A322046143DD91003F009
:100BE00007020133ADB2615CB25CA4F85A32114223
:100BF00014BF01210021FFF7B3FFB4F85A22B4F863
:100C000058329A42E4D30023A4F85A32A4F8583256
:100C100008E0B0F85A32002BD5D10648FFF746FE5F
:100C20000028D0D170BD00BF31070020708A00209D
:100C300021890108680A002001EB41018900A0F820
:100C40005C127047B0F8580200280CBFFF2000204B
:100C5000704729B990F8603283F0010380F8603260
:100C600090F86002704700002DE9F043CDB00446D3
:100C7000664D6846FFF759FD6846FFF7B9FD00234A
:100C8000B4F85CC2A4F85832A4F85A3284F860323E
:100C9000A4F85E329AB2944517D994F86002B4F879
:100CA000582280F0010002F00701D61084F860029B
:100CB0006F5CA15D30B139430132A1550133A4F815
:100CC0005822E7E721EA0701F6E7504F08223E469F
:100CD00016F8013B204613F07E0F14BF01210021BE
:100CE000FFF7B7FFB4F85832002853D0D91003F0FB
:100CF0000700615C285C0143013AD810013392B2CD
:100D00002154A4F85832002AE2D19146DFF800813C
:100D100093B2BDF82C01B3EBC00F19464DD2C2F30C
:100D2000CC0103F0070320461DF8016018F80330DA
:100D30001E4014BF01210021FFF78BFFB4F8583289
:100D400080B3D91003F00700615C285C0143D81020
:100D50002154591C89B2A4F85812C6B109F10106F0
:100D6000F6B2052E13D194F86002CE1001F00701FF
:100D700080F0010015F801C084F86002A15DC8B1DF
:100D80004CEA0101A15502330026A4F85832013281
:100D9000B146BDE703F00701685CD910615C21EA48
:100DA0000001A9E703F00701685CD910615C21EA42
:100DB0000001CCE721EA0C01E4E7082217F8013B27
:100DC000204613F07E0F14BF01210021FFF741FFE1
:100DD000B4F8583290B1D91003F00700615C285C78
:100DE0000143013AD810013392B22154A4F8583289
:100DF000002AE3D110464DB0BDE8F08303F00701AF
:100E0000685CD910615C21EA0001EAE721890108E8
:100E100029890108002310B5044603804360083087
:100E200004F12A01024602F8013B9142FBD184F809
:100E30002A302222024917F099F8204610BD00BF3F
:100E4000E58A010830B5C1EBC1010E4D847D6B18F8
:100E5000695C24F00F045A7801F00F01C2750C434D
:100E60009A7884750276DA7842761A7982765A7997
:100E70009B79C276027F23F00F0302F00F021A4320
:100E8000027730BD2B8A010830B5C1EBC1010E4D90
:100E9000847D6B18695C24F00F045A7801F00F010F
:100EA000C2750C439A7884750276DA7842761A799C
:100EB00082765A799B79C276027F23F00F0302F083
:100EC0000F021A43027730BD558A010810B5044657
:100ED0002E4802F06BFB2D4802F0D7F9002835D0E0
:100EE0006378013B032B4FD8DFE803F00217313C56
:100EF0000121264802F09CF909222549234802F0E5
:100F0000BDF822222349214802F00AFA01211F4894
:100F100002F0FEF80223637018E094F82A102046CD
:100F2000FFF790FF222204F10801184802F0F8F9B7
:100F300094F82A30052B06D1002384F82A30237830
:100F400023B90323E7E7013384F82A3010BD2222B6
:100F500011490E4802F0E4F90C4802F08BF9042321
:100F60006060D8E7094802F085F963681E3398424B
:100F7000ECD90021054802F0CBF8044802F074F9DE
:100F8000002384F82A30C6E70023C4E784580020F1
:100F9000228A01087F8A0108A18A010810B5044647
:100FA0001D4801F0F7F81C4801F0A4F968B1637816
:100FB000022B0BD0032B24D0012B29D1222217493D
:100FC000154801F09FF90223637010BD94F82A10B0
:100FD0002046FFF759FF222204F108010E4801F0D4
:100FE00091F994F82A30052B07D1002384F82A3090
:100FF0002378002BE9D10323E6E7013384F82A3074
:10100000E3E722220649044801F07CF90023DBE7EC
:1010100000236370F2E700BF98310020C38A010803
:10102000078B010808B5124B1B785C3B062B1DD8BB
:10103000DFE803F0181C14041C1C0400017841B103
:101040000C48012102F06EF80A48BDE8084002F0A1
:10105000ADBA0848BDE8084002F064B8BDE80840F1
:10106000FFF734BFBDE80840FFF798BF08BD00BFD9
:10107000A99A002084580020012A11D10978012959
:101080000CBF0123002303700CD1437853B9064AE7
:10109000127802F0FD025C2A00D1417018467047B8
:1010A0000423FBE70023F9E7A99A0020002300F1BD
:1010B0000C0200F13C0103600371836022F8023BE3
:1010C0009142FBD14FF0000380F83C3070470000A4
:1010D000836837B55B00002990F83C200446B8BF10
:1010E00043F001038360531C00EB4202DBB2172B79
:1010F00080F83C30918184BF002380F83C308068C8
:1011000020F07F432D4858400BF01CFB022825D8C7
:1011100004F10C0104F13C054FF47A53284A31F9EB
:10112000020B8242B8BF02468342A8BF03468D42EB
:10113000F5D1D11A052911DD00218DF802202148B1
:101140008DF8001011121A128DF804308DF801106C
:1011500069468DF80320052209F078FFA06820F089
:101160007F43194858400BF0EDFA022824D804F1C7
:101170000C014FF47A533C34114A31F9020B82428C
:10118000B8BF02468342A8BF03468C42F5D1D11AAC
:10119000052911DD80218DF802200A488DF8001004
:1011A00011121A128DF804308DF8011069468DF86D
:1011B0000320052209F04AFF03B030BD68B4AA003D
:1011C00080C1FFFFC0D90020974B55002DE9F041A9
:1011D00004460E460025174643F23338ABB29F4211
:1011E00021D936F915102379CA0F934209D0236803
:1011F000B3F5004F2ABF6FF4CC7003F299131B189C
:1012000023602368227103EB0802B2F5803F02D20B
:1012100022600135E2E7A3F54C432046CD3B236035
:10122000FFF756FFF5E7BDE8F0810022027042802B
:101230007047000030B5044685B07E4803F094F94D
:10124000237873B37B4803F065FA042829D901AAEF
:1012500079480C231146013B10F8015B13F0FF03A2
:1012600002F8015BF7D162881520B2FBF0F300FBB6
:1012700013239BB243B1012A15D130238DF80D30D1
:101280004DF60263ADF80E300C226A4803F090FA76
:10129000638840F276210133B3FBF1F201FB123394
:1012A000638005B030BD022A05D134238DF80D309E
:1012B0004DF61963E6E7032A05D131238DF80D3089
:1012C0004DF66F63DEE7042A05D11F238DF80D303C
:1012D0004FF22B63D6E7052A05D132238DF80D3066
:1012E0004BF22233CEE7062A05D124238DF80D30A8
:1012F0004EF22A03C6E7072A05D133238DF80D30B5
:101300004BF23B33BEE7082A01D1502354E0012BB6
:1013100005D125238DF80D3049F24F33B2E7022B6A
:1013200005D170238DF80D304DF60B23AAE7032B62
:1013300005D125238DF80D304DF21D63A2E7042B56
:1013400005D133238DF80D304BF21B339AE7052B73
:1013500005D125238DF80D304DF26F7392E7062BE2
:1013600001D13923E6E7072B05D125238DF80D3070
:101370004CF20C7386E7082B05D150238DF80D3005
:101380004DF26F037EE7092A4DD0092B05D12523A5
:101390008DF80D304DF21E0374E70A2A43D00A2B54
:1013A00005D121238DF80D304CF20C236AE70B2A6E
:1013B00039D00B2B05D125238DF80D304BF26F332F
:1013C00060E70C2A2FD00C2B05D13D238DF80D3072
:1013D0004DF2027356E70D2A25D00D2B01D125239E
:1013E00064E70E2A1FD00E2B8FD00F2A1BD00F2B95
:1013F00005D125238DF80D304DF21B6342E7102AED
:1014000011D0102B05D123238DF80D3043F61B236B
:1014100038E7112A07D0112B05D121238DF80D3083
:101420004FF225532EE716238DF80D304FF2295336
:1014300028E700BF407A0020298B0108012A38B52F
:10144000044616D10B78012B03780CBF012500252B
:1014500009D12BB9438029220749084803F082F9B2
:101460000020257038BD002BFAD0044803F0C6F9DF
:10147000F6E70420F6E700BF358B0108407A00202C
:1014800000224FF4C061C0E90022816002737047FE
:101490002DE9F341444E0446027B33789A4268D0EA
:1014A000663B40F6BF12052B55D8DFE803F0030773
:1014B0000A0D10134FF46F7323800CE040F20F43BA
:1014C000FAE740F2DF43F7E740F26163F4E740F602
:1014D0001F03F1E70280238893423ED040F61F02AB
:1014E00093423CD040F2616293423AD040F2DF42F4
:1014F000934238D040F20F42934236D0B3F56F7F1B
:101500004ED10523294F17EBC30749D07B8860686C
:10151000638008B116F0B6FC00256088A84640003C
:1015200016F086FC60606288ABB29A421FD94046D2
:1015300016F064FCB4F90830626883FB0001C30F45
:1015400043EA4103A9B2013503F30F0322F8113036
:101550007B689844E7E70023AEE70023D2E7012346
:10156000D0E70223CEE70323CCE70423CAE733788E
:101570002373A37AA3B10E484FF0000805F0DAFCFC
:101580000B4F05466388AB420AD2CDF8008038463F
:101590006268317806F0C4F86388ED1AADB2F1E7FD
:1015A00002B0BDE8F08100BFA99A0020608B01085D
:1015B000708A0020012A06D10B785A1E53425341EB
:1015C0008372002070470420704700220270704729
:1015D00010B50446084807F003F823785BB10648C5
:1015E00007F0B1F8012806D9312204490248BDE8C4
:1015F000104007F0B0B810BDAC950020908B0108EA
:10160000012A06D10B785A1E534253410370002021
:101610007047042070470022027042708270704749
:1016200010B50446104807F037FE0F4807F0FBFEE0
:10163000A8B16378012B13D1A17831220B4BC1EBF8
:10164000C1010948C1EBC101194407F0F4FEA378B8
:10165000013303F00303A370237803B9637010BD53
:1016600000236370A370FAE728AA0020C18B010849
:10167000012A0BD10A78012A0CBF01230023037031
:1016800006D1437823B94270184670470423FBE71C
:101690000023F9E7002202704270704710B504463B
:1016A0000F4808F0B7FC0E4808F04EFD68B16378AB
:1016B000012B03D0022B09D0002305E0D9220949D0
:1016C000074808F049FD0223637010BDD92206497E
:1016D000034808F041FD2378002BF5D00123F3E700
:1016E00000D2002026030020FF030020012A0BD196
:1016F0000A78012A0CBF01230023037006D1437826
:1017000023B94270184670470423FBE70023F9E72A
:10171000002202707047000008B5037853B10648F4
:1017200005F008FCA52805D9AA210448BDE8084011
:1017300008F096BD08BD00BF708A002080D7002049
:10174000012A06D10B785A1E5342534103700020E0
:101750007047042070470022C0E900224FF6FF7254
:10176000826070472DE9F74304460E460025174670
:1017700045F6BF58DFF85C90ABB29F4226D936F8E9
:1017800015206189636891422189134438BF6281C1
:101790009142636088BF2281226801324245226003
:1017A00012D9A1684846B3FBF2F309BA5BBA062224
:1017B00000916946ADF8043009F070FC0023C4E9DB
:1017C00000334FF6FF73A3600135D5E703B0BDE8E2
:1017D000F08300BFC0D90020024600F57A710023D3
:1017E00002F8013B9142FBD1A0F8E833A0F8EA33BC
:1017F00080F8EC33704700002DE9F341B0F8E8338E
:101800000446002B3BD01F4805F094FB1E4F0546B5
:10181000DFF87C801B4E182D31D9B4F8EA333046FE
:10182000183DD91003F00702ADB2BA5C635C6121C8
:10183000134015BF00230093144A182316BF0093CA
:101840004246182305F06CFF94F8EC330133DBB209
:10185000312B84F8EC3307D9B4F8EA330133A4F818
:10186000EA33002384F8EC33B4F8EA23B4F8E8331D
:101870009A42D0D30023A4F8EA33A4F8E83302B0A4
:10188000BDE8F081708A0020988E0108D8040020FD
:10189000380A00202DE9F74F0E46904600214FF4FC
:1018A0007A72044616F0FCFB0823DFF8C4E0A4F8C3
:1018B000E8330023A4F8EA3384F8EC33DDB245457D
:1018C00041DA00210C20CAB242430EEB02001EF89E
:1018D0000220B2B3775D01319742F3D190F808B09E
:1018E0004FF0000C4FF0004501905FFA8CF1B4F816
:1018F000E8238B4525D902F007071A484FEAE20989
:101900000CF1010C10F807A0019814F809104768B1
:1019100035EA07000CBF41EA0A0121EA0A0104F88E
:10192000091040F2E2318A4206D900230420A4F8CB
:10193000E83303B0BDE8F08F01326D08A4F8E82366
:10194000D3E70133BAE7B4F8E823082AEDD005322B
:101950000548064992B2A4F8E82312B209F0A8FE9D
:101960000020E6E7988E0108C0D90020A08E01086B
:10197000888C01080023A0F8E833A0F8EA3380F847
:10198000EC337047002300F1140200F65431036178
:10199000C0E90033C0E9023322F8023B8A42FBD19E
:1019A00042F20F72C0F8543BC0F8583B0021A0F837
:1019B0005C2B00F5B552C0F8603BC0F8643B1C32AC
:1019C000C0F8683BC0F86C3BC0F8703BC0F8743B93
:1019D000A0F8783B4FF0000380F87A3B00F67C33A8
:1019E00023F8021B9A42FBD170470023C0F8603BEA
:1019F00080F8753B80F8763B80F8783BC0F8583B20
:101A000042F20F73A0F85C3B704700002DE9F74FDE
:101A1000BDF83040BDF9388004EB4202BDF934A076
:101A2000DFF88C90C8F1000B92B20192019AA242A9
:101A30003BD000EB4102671C4FEAE40E04F00706BE
:101A4000958ABFB2023413F80EC0A5EB0A05FA104E
:101A500007F0070719F806602DB219F80770A4B24D
:101A60005D4506DA2CEA060603F80E609D5C2F43FE
:101A700008E0002D11DA2CEA060603F80E609D5CE2
:101A800025EA07079F544A1D92B2B2F5B46F24BFEE
:101A9000A1F29B518AB21146C8E74CEA06064545B9
:101AA00003F80E609D5CE2DAEAE703B0BDE8F08F70
:101AB000BC8E0108B0F8543B50F823302DE9F04FAC
:101AC00023F07F430446904889B0884658400AF086
:101AD00039FEC31E8146DBB2122B40F2B780B4F848
:101AE000563B0022894D4FF6FD7A03F22D511646E2
:101AF000DFF82CE24FF0030B89B2B1F5B46F28BFC9
:101B0000A3F173014FF47A5328BF89B204930846B6
:101B100004EB4007049BB7F91470BD42B8BF3D46C3
:101B2000BB42A8BF3B46B9F1020F04938ABF784B72
:101B300012F90EC012F903C0BCF1010F00F0898048
:101B4000BCF1030F05D0BCF1FF3F40F084803E4460
:101B500001E017FB0A66471D0132BFB2B7F5B46F4B
:101B60002ABFA0F29B50384680B2182AD0D1D4F8B0
:101B7000600BB0426ADA049B0DF1180A20462B4430
:101B80005B101FB2ED1A44F631435D43042345F365
:101B9000CF3500935346CDE90175FFF737FFB9F113
:101BA000020F5C4969D84FF0000B5B4AD94611F827
:101BB000013B1AF80BC00BF1010B12F8010B03EA01
:101BC0000C030591049258400AF0ACFDBBF1070FDD
:101BD0008144DDE904215FFA89F9E8D1B9F1030F05
:101BE00034D8B8F1000F39D00023A4F8725BA4F800
:101BF000705BA4F86E5BA4F86C5BA4F86A7BA4F835
:101C0000687BA4F8667BA4F8647B84F8743B40236B
:101C1000C4F8606B84F8753BB4F8563B03F21A4283
:101C2000A4F8583B92B2B2F5B46F28BFA3F5C372C3
:101C3000A4F85A2B03F20D1292B2B2F5B46F2ABF78
:101C4000A3F29343A4F85C2BA4F85C3B09B0BDE875
:101C5000F08FF61B7FE717FB0B667CE794F8743B6D
:101C600004EB43020133DBB2A2F86C5BA2F8647BA5
:101C7000032BCAD984F8748BC9E74FF0000B274AAD
:101C8000D94611F8013B1AF80BC00BF1010B12F801
:101C9000010B03EA0C030591049258400AF042FD3F
:101CA000BBF1070F8144DDE904215FFA89F9E8D12E
:101CB000B9F1030FCAD8B8F1000F16D00023A4F869
:101CC000725BA4F8705BA4F86E5BA4F86C5BA4F87C
:101CD0006A7BA4F8687BA4F8667BA4F8647B84F82C
:101CE000743BC4F8606B202394E794F8743B04EBD6
:101CF00043020133DBB2A2F86C5BA2F8647B032BD6
:101D0000EDD984F8748BECE76E28760080C1FFFF74
:101D1000F18E0108C48E0108CB8E0108D28E010815
:101D2000D98E010880F8771B70470000B0F85A3B45
:101D30000A463C3370B49BB24FF4077500245E1C16
:101D400000EB4301013DB6B2B1F87C1BADB2B6F574
:101D5000B46F0C442ABFA3F29F5333469BB2002DAD
:101D6000EDD14FF4077301210648B4FBF3F4C4F33B
:101D7000072382F8234082F82230242370BC08F025
:101D800081BE00BFC0D9002070B50446B0F8560B24
:101D900000298EB004EB40039982A3F87C2BB4F8A1
:101DA000542B54F822304FEA4303B8BF43F00103E9
:101DB00044F8223094F8783B002B6AD10121204668
:101DC000FFF778FEB4F85C2BB4F8563B934240F032
:101DD0009680B4F9662B03F21231B4F9645B2046A5
:101DE000B4F96C6B89B21544B4F9682BB1F5B46FD2
:101DF0001544B4F96A2B28BFA3F28E214FF00803D3
:101E00001544B4F96E2B28BF89B200931644B4F977
:101E1000702B45F38F0505AB1644B4F9722B1644AD
:101E200094F8752B46F38F068DF814208422CDE9A3
:101E30000156FFF7EBFD94F8753B402B40F0C08056
:101E400004A801F01DF80DF113030DF112020DF1BC
:101E5000150104A801F042F894F8772B9DF8123090
:101E60009A4247D100239DF8142084F8763B84F8E9
:101E7000793B9DF813301A438DF814200A2B00F299
:101E80009980DFE803F079698397979725565697ED
:101E90005600B4F8581B01F29F534A1C9BB292B2F1
:101EA000B3F5B46F24BF01F1FF339BB2B2F5B46F49
:101EB00024BFA1F29F5292B2934206D2984281D39C
:101EC00090423FF67FAF002179E79842F8D3FAE7D6
:101ED0002B46B4F9582B6449644800960AF051F92E
:101EE00005A92046FFF722FF022384F8783B002350
:101EF00084F87A3B0023C4F8603B84F8753BB4F85F
:101F0000563B94F8780B01339BB2B3F5B46F28BFFE
:101F10000023A4F8563BB4F8543B01339BB2042B86
:101F200088BF0023003018BF0120A4F8543B0EB036
:101F300070BD94F8783B022BDCD12B46B4F9582BBA
:101F40004B494A4800960AF01CF905A92046FFF7BC
:101F5000EDFE9DF81330CBE72B46B4F9582B4549DD
:101F6000009642480AF00DF905A92046FFF7DEFE6B
:101F7000012384F8783BBDE794F8783B012BF7D137
:101F800000962B46B4F9582B3B49EAE794F8783B86
:101F9000012BAFD12B46B4F9582B38490096334862
:101FA0000AF0EFF8204605A9FFF7C0FE2046FFF72C
:101FB0001CFD9FE700962B46B4F9582B3049EEE7FD
:101FC000202B12D12B46B4F9582B2E4927480096C6
:101FD0000AF0D7F805A92046FFF7A8FE002384F8E9
:101FE000763B0123A4F8783B84E794F8783B73B1FF
:101FF00094F8763B0133DBB20C2B84F8763B06D9A0
:102000001A48012108F070FD2046FFF7EEFC94F815
:10201000783B012B17D194F8793B05AA012113488D
:10202000042B8BBF202301338DF81430DBB28BBF20
:10203000002384F8793B84F8793B8DF8143022230F
:1020400008F020FD56E7022B7FF454AF94F87A3B5A
:10205000002B3FF44FAF43F0400305A920468DF815
:102060001430FFF763FE45E7098F0108C0D900204F
:102070003A8F01086C8F01089E8F0108D38F0108E9
:1020800009900108339001082DE9F04100240E4623
:102090000546174698462146444509D036F914109E
:1020A000284637F814200134FFF76EFE0146F3E7A7
:1020B0000248BDE8F04104F05BBF00BF708A002019
:1020C00070B5044600254FF4B97004F11C06258153
:1020D000208065816573257315F0AAFE04F13C0329
:1020E00032466060A561C4E9045522F8025B934260
:1020F000FBD104F2EC41002203F8012B9942FBD101
:10210000F023C4F8EC2400212022C4F8F034304637
:1021100015F0C6FF05232046237409236382024B72
:10212000C4E9053670BD00BF08050020F0B58FB0CA
:102130000A4600234FF4E37502A940F252564FF6C7
:10214000AE274FF63A6C02F0C004802C1DD0C02C94
:1021500018D0002C0CBF64463C4621F813400133D4
:102160009200042BD2B2EED104AA103014F088FFF2
:10217000002304AA022100931423054805F0D0FA95
:102180000FB0F0BD21F81360E9E721F81350E6E73E
:10219000708A002038B5B0F8EC340446E3B13C480E
:1021A00004F0C8FE0546142D45D9B4F8EE34204697
:1021B000143D5A1C2344ADB2A4F8EE2493F83C100D
:1021C000FFF7B4FFB4F8EE24B4F8EC349A42EAD343
:1021D0000023C4F8EC342EE0428903899BB2934279
:1021E00012D1037B3BB303882BB32A4B1B781BBB59
:1021F000D4F8F0245F20591C9BB29A4212D9234490
:1022000083F83C000B46F6E7438902899A4204D9D9
:10221000038942899B1A9BB2E6E7428901880389B8
:102220000B44F7E7A4F8EC240023A4F8EE34B4F848
:10223000EC34002BB3D138BD04F13C0304F15D0054
:1022400000212589628992B2AA4201D1227B72B112
:102250006568628992B2AA5C1A7021736289013240
:1022600092B2628162892588954200D861810133EA
:102270008342E6D1084A04F1840112F8010B03F805
:10228000010B8B42F9D14823A4F8EC34CCE700BF12
:10229000708A0020AA9A0020639001080C234FF452
:1022A000167203FB0121B1F5966F8ABF4FF4966356
:1022B000C0F8F014C0F8F0347047418903890288EF
:1022C0009BB28B4205D1037B002B0CBF1046002034
:1022D000704743890189994208D90389408910448C
:1022E000C01A80B2904288BF00207047438900899D
:1022F000181AF6E708B5FFF7E0FF2323B0FBF3F069
:10230000C0B208BD222AF8B504460D4624D1FFF715
:10231000D4FF202822D901231946227B02F0FF0096
:102320002AB161730133222BF7D10020F8BD666812
:102330002289EF5C92B2B7542289013292B2228193
:1023400022892688964200D820812089628992B20B
:102350008242E7D12173E5E70420E7E70520E5E7BE
:10236000002300F1140200F23C510361C0E9003384
:10237000C0E9023322F8023B9142FBD1C0F83C3560
:1023800042F20F72C0F84435C0F848354FF00003F0
:10239000A0F8402580F84C3570470023C0F844353C
:1023A000C0F84835C0F83C3542F20F73A0F840350C
:1023B000704700002DE9F74FBDF83040BDF9388077
:1023C00004EB4202BDF934A0DFF88C90C8F1000B99
:1023D00092B20192019AA2423BD000EB4102671CEB
:1023E0004FEAE40E04F00706958ABFB2023413F8F0
:1023F0000EC0A5EB0A05FA1007F0070719F80660EA
:102400002DB219F80770A4B25D4506DA2CEA06066B
:1024100003F80E609D5C2F4308E0002D11DA2CEAD2
:10242000060603F80E609D5C25EA07079F544A1DC7
:1024300092B2B2F5257F24BFA1F28F218AB2114654
:10244000C8E74CEA0606454503F80E609D5CE2DAF3
:10245000EAE703B0BDE8F08F8A900108B0F83C25A8
:10246000002950F822304FEA4303B8BF43F001037C
:102470002DE9F04F40F822300446B0F83E3591B0D7
:1024800000EB4303998250F822307A4823F07F43CF
:1024900058400AF057F9022800F28E80B4F83E3511
:1024A0001825DFF8E4E1002603F22121724F4FF6F0
:1024B000FD784FF0030989B2B1F5257F28BFA3F15C
:1024C00073014FF47A5328BF89B20A4604EB4200E5
:1024D0001EF901CBB0F914008742B8BF074683420A
:1024E000A8BF0346BCF1010F00F0BE80BCF1030F92
:1024F00005D0BCF1FF3F40F0B980064401E010FB7D
:102500000866501D013D80B2B0F5257F2ABFA2F2BA
:102510008F22024692B215F0FF05D7D1D4F8442598
:10252000B24249DA3B440DF11C0A182220465B10E6
:10253000DFF858B1A9460FFA83F8FB1A44F6314781
:102540005F43042347F3CF3700935346CDE9018718
:10255000FFF730FF494A12F8013B1AF8091009F158
:1025600001091BF8010B0B405840CDE904220AF089
:10257000D9F8B9F1070F0544049AEDB2EBD1032D58
:102580001AD83B4642463E493E4809F0C3FDB4F8DE
:102590003E35C4F8446503F20D12A4F84885A4F84A
:1025A0004A7592B2B2F5257F29BF6FF4C372A4F8C1
:1025B00040259B18A4F84035B4F84025B4F83E35C2
:1025C00093423BD1991D8422204689B2B1F5257FE3
:1025D00028BFA3F28E21B4F94A35029328BF89B2ED
:1025E000B4F9483501930823009307ABFFF7E2FEE7
:1025F00006A800F045FC0DF11B030DF11A020DF1C8
:102600001D0106A800F06AFC94F84C259DF81A30CC
:102610009A420CD19DF81B30032B08D1C32307AA83
:10262000002118488DF81C30222308F02BFA42F2C2
:102630000F73A4F840350023C4F84435B4F83E3590
:1026400001339BB2B3F5257F28BF0023A4F83E35A4
:10265000B4F83C3501339BB2042B88BF0023A4F8A7
:102660003C3511B0BDE8F08F361A4AE710FB096619
:1026700047E700BF6E28760080C1FFFF92900108F7
:10268000B8900108C0D90020A090010899900108D5
:1026900070B505460C4601EB4206B44205D034F94C
:1026A000021B2846FFF7DAFEF7E770BD80F84C15ED
:1026B000704710B50446002100F062F8012104F6CD
:1026C000546000F05DF8204610BD00002DE9F84F81
:1026D00006460024884691469A46204625469DF89F
:1026E00028B006F65467A3B29B451BD91AF80430EC
:1026F000042B15D0082B02D1304600F074F839F8BD
:102700001420304638F9141000F01EFA39F814205D
:1027100038F9141005463846013400F015FAE2E79E
:102720003846EAE7002D14BF294601460248BDE8B5
:10273000F84F04F01DBC00BF708A002038B5044675
:102740000D4600F0D5F9294604F65460BDE838403E
:1027500000F0CEB938B504460D4600F0CCF9294654
:1027600004F65460BDE8384000F0C5B910B5044621
:1027700000F043F804F65460BDE8104000F03DB8A6
:102780000023017000F1180200F5E4614361C0E923
:102790000133C0E9033322F8023B8A42FBD142F203
:1027A0000F72C0F82037C0F824370021C0F82C374A
:1027B000C0F83037C0F83437C0F83837C0F83C3785
:1027C000C0F84037C0F844374FF00003C0F828275E
:1027D00000F6526280F8483700F24A7323F8021B71
:1027E0009A42FBD170470023A0F82A37C0F820375F
:1027F000C0F82C3780F841377047002342F20F723F
:1028000080F8413780F8423780F84637C0F82037E3
:10281000C0F82437C0F82827C0F82C3770470000CC
:102820002DE9F74FBDF83040BDF9388004EB420286
:10283000BDF934A0DFF88090C8F1000B92B201928C
:10284000019AA24235D001F10C02671C4FEAE40E56
:1028500004F0070630F81250BFB2023413F80EC06D
:10286000A5EB0A05FA1007F0070719F806602DB264
:1028700019F80770A4B25D4506DA2CEA060603F8DB
:102880000E609D5C2F4308E0002D0ADA2CEA060654
:1028900003F80E609D5C25EA070705319F5489B255
:1028A000CEE74CEA0606454503F80E609D5CE9DA82
:1028B000F1E703B0BDE8F08FE4900108B0F82037ED
:1028C00000EB83035B682DE9F04F23F07F43044660
:1028D000804889B08846584009F034FFC31E8146BD
:1028E000DBB2122B40F29880B4F8221700224FF48A
:1028F0007A53794D73391646DFF8F0E14FF6FD7AD9
:1029000089B24FF0030B04930F4607F10C00049BB0
:1029100034F910008542B8BF05468342A8BF03467C
:10292000B9F1020F04938ABF6C4B12F90EC012F971
:1029300003C0BCF1010F72D0BCF1030F04D0BCF195
:10294000FF3F6ED1064401E010FB0A6601320537F5
:10295000182ABFB2D9D1D4F82C07B0425CDA049B54
:102960000DF1180A20462B445B101FB2ED1A44F6F5
:1029700031435D43042345F3CF3500935346CDE9FE
:102980000175FFF74DFFB9F1020F55495BD84FF0C4
:10299000000B544AD94611F8013B1AF80BC00BF151
:1029A000010B12F8010B03EA0C0305910492584045
:1029B00009F0B8FEBBF1070F8144DDE904215FFA9D
:1029C00089F9E8D1B9F1030F26D8B8F1000F2BD05F
:1029D0000023A4F83E57A4F83C57A4F83A57A4F8AB
:1029E0003857A4F83677A4F83477A4F83277A4F8E7
:1029F000307784F840374023C4F82C6784F8413797
:102A0000B4F82237A3F5C372A4F8243703F20D13E8
:102A1000A4F82627A4F8283709B0BDE8F08F361AA5
:102A200094E710FB0B6691E794F8403704EB430200
:102A30000133DBB2A2F83857A2F83077032BD8D98C
:102A400084F84087D7E74FF0000B274AD94611F8A2
:102A5000013B1AF80BC00BF1010B12F8010B03EA52
:102A60000C0305910492584009F05CFEBBF1070F7E
:102A70008144DDE904215FFA89F9E8D1B9F1030F56
:102A8000CAD8B8F1000F16D00023A4F83E57A4F816
:102A90003C57A4F83A57A4F83857A4F83677A4F866
:102AA0003477A4F83277A4F8307784F84037C4F844
:102AB0002C672023A2E794F8403704EB430201334C
:102AC000DBB2A2F83857A2F83077032BEDD984F89F
:102AD0004087ECE76E28760080C1FFFF199101085E
:102AE000EC900108F3900108FA90010801910108A7
:102AF00080F843177047A0F84417704730B4B0F817
:102B000026470A4604F13C0304F516749BB2A5B2AD
:102B10000024591C00EB4303B3F84A371C448BB222
:102B2000AB42F6D14FF40773B4FBF3F4C4F30723BD
:102B300082F8234082F8223024230178014830BCF7
:102B400007F0A0BFC0D90020B0F82A3770B5013314
:102B500004468EB09BB2B4F844579D42A0F82A3781
:102B600090F8460704D9003018BF01200EB070BDA0
:102B7000B4F82237B4F828579D42F4D3B3F5617FF7
:102B8000F1D204EB43050029A5F84A272983B4F8BC
:102B9000205704EB85056A684FEA4202B8BF42F04D
:102BA00001026A60002865D1A3F5C8735A2B03D8C7
:102BB00001212046FFF782FEB4F82837B4F8221727
:102BC00099427AD1B4F93237A1F28E21B4F9305753
:102BD0008422B4F9386789B21D44B4F934372046E9
:102BE0001D44B4F936371D44B4F93A371E44B4F9DC
:102BF0003C3745F38F051E44B4F93E371E4494F824
:102C0000413746F38F068DF814300823CDE901567D
:102C1000009305ABFFF704FE94F84137402B40F0DA
:102C2000C18004A800F02CF90DF113030DF112027C
:102C30000DF1150104A800F051F994F843279DF80F
:102C400012309A4239D100239DF8142084F842377B
:102C500084F847379DF813301A438DF814200A2B57
:102C600000F29580DFE803F0675276939393123A6F
:102C70003A933A00B4F82427511E89B28B429BD371
:102C8000013292B2934297D8002192E72378744997
:102C9000002B7448B4F9243714BF02220122CDE975
:102CA000005609F0B5FA05A92046FFF727FF0223D1
:102CB00084F84637002384F84837B4F8223794F86C
:102CC00046070133A4F82237B4F8203701339BB20A
:102CD000042B88BF0023A4F8203744E794F8463734
:102CE000022BEAD123786049002B5E48B4F92437DF
:102CF00014BF02220122CDE9005609F089FA05A984
:102D00002046FFF7FBFE9DF81330D4E723785749A0
:102D1000002BB4F9243714BF02220122CDE900565A
:102D2000504809F075FA05A92046FFF7E7FE012390
:102D300084F84637C1E794F84637012BF7D123785A
:102D40004B49002BB4F92437CDE9005614BF0222B9
:102D50000122E5E794F84637012BAED123784549A7
:102D6000002BB4F9243714BF02220122CDE900560A
:102D70003C4809F04DFA05A92046FFF7BFFE0023A5
:102D800084F8463742F20F73A4F8283795E7237882
:102D90003949002BB4F92437CDE9005614BF02227B
:102DA0000122E5E7202B17D123783449002B2D4849
:102DB000B4F9243714BF02220122CDE9005609F0EC
:102DC00027FA05A92046FFF799FE002384F8423729
:102DD0000123A4F8463770E794F8463793B194F886
:102DE00042370133DBB20C2B84F842370AD9217801
:102DF0001C4807F079FE002384F8463742F20F732F
:102E0000A4F8283794F84637012B17D194F84737A0
:102E100005AA2178042B13488BBF202301338DF89A
:102E20001430DBB28BBF002384F8473784F8473770
:102E30008DF81430222307F025FE3EE7022B7FF4A5
:102E40003CAF94F84837002B3FF437AF43F04003D2
:102E500005A920468DF81430FFF750FE2DE700BF7E
:102E600031910108C0D9002068910108A0910108A2
:102E7000D8910108139201084F9201087F9201082E
:102E800070470000B1F5006F10B50DD34FF48023EB
:102E900040F6754405480B4201D15B08FBE7DA0AAE
:102EA000624351400142F6D1084610BD00F8FFFFD1
:102EB00010B54C780B78E40004EBC3248B7804EB5A
:102EC00053142146FFF7DEFF034B53F82000604008
:102ED000C0F3C72010BD00BFB892010873B51E46ED
:102EE0004B7B0C7B15469A099B0042EA84020C7DC1
:102EF000C97C23F03F038DF80420890001F03C01D8
:102F0000194341EA9411A4008DF8051001A924F099
:102F10000F048DF80640FFF7CBFF030900F00F0008
:102F20002B70307002B070BD02F00F0242EA011146
:102F3000134AC8B2197B21F03F0130B541EA900134
:102F400032F810401973E5B2597BA40AAA0801F0BF
:102F50000F0104F03C0441EA801102F0300002F05D
:102F60000F0201435973D97C21F00F0111431A7DDF
:102F700002F00302D97442EA851222431A7530BD69
:102F8000B8B201082DE9F04100254FF4B9760446A6
:102F900005810680458145730573304614F048FF6E
:102FA00026826060304604F12C06258365776583B0
:102FB000257714F03DFF04F14C0233466061A562B1
:102FC000C4E9085523F8025B9A42FBD14FF0000395
:102FD00004F16E01002284F84C3004F14D0303F833
:102FE000012B9942FBD104F16F0884F86E2004F1A3
:102FF0007B070022434603F8012B9F42FBD104F1DB
:1030000087023B46002103F8011B9A42FBD104F1E1
:10301000AF03002102F8011B9342FBD104F1D70258
:10302000002503F8015B9A42FBD1C4E93655C4E997
:103030003855A4F8E85020220021304615F030F829
:1030400005230C220B4984F8203009233846638479
:10305000094BC4E9093614F089FF0C2205494046A2
:1030600014F084FFA4F8E8502046C4E93855BDE8C0
:10307000F08100BFC0B4010862050020092A2DE9D3
:10308000F04104460D4627D10C2200217B30134E1F
:1030900015F006F8124F002316F8011B03F007087D
:1030A00004EBD10001F0070117F801C0D91090F826
:1030B0007B20013315F801E017F808101EEA010F14
:1030C00014BF42EA0C0222EA0C02442B80F87B2057
:1030D000E2D10020BDE8F0810420FBE7CCB4010878
:1030E000B8B40108012A04D10978012903D00229C2
:1030F00008D004207047002380F8E810C0F8E030C2
:1031000018467047002380F8E920C0F8E430F7E75C
:10311000002380F84C10C0E93733C0F8E430A0F841
:10312000E8307047002914BF0523002380F84C3095
:10313000704700002DE9F04194B006461746002480
:1031400003AD4FF4E37240F252504FF6AE2C4FF6FF
:103150003A6E01F0C003802B2AD0C02B25D0002B63
:103160000CBF7346634625F8143001348900042CE3
:10317000C9B2EED10DF1140814220021404614F01A
:103180008FFF23460AAA294606F120008DF81E70FB
:1031900013F076FF14230AAA02210748CDF8008015
:1031A00004F0BEFA14B0BDE8F08125F81400DCE7A5
:1031B00025F81420D9E700BF708A00201B4B1B782C
:1031C000622B10B512D100F1870300F1A8025F2431
:1031D000002183F8284003F8011B9342F9D12123F1
:1031E000A0F8D8300023A0F8DA3010BD5F2BF9D159
:1031F00000F1870300F18E025524002183F8284056
:1032000003F8011B9342F9D15F2300F19602FF24DA
:10321000002180F8B63000F18F0383F8284003F8CE
:10322000011B9342F9D10F23DAE700BFA99A0020CE
:1032300037B500F14D040D4621220749204614F010
:1032400095FE01A8FFF71CFE23460922294601A886
:10325000FFF76AFE03B030BD10B5010800230381FB
:10326000437343810373704700230383437743838E
:1032700003777047D0F8DC00704708B5FFF71DF8FA
:103280002323B0FBF3F0C0B208BD08B51030FFF740
:1032900014F82323B0FBF3F0C0B208BD222AF8B51E
:1032A00004460D4633D1FFF708F8202831D994F8A9
:1032B000E83033B1002323816373638184F8E830FD
:1032C000237301231946227B02F0FF0052B1617380
:1032D0000133222BF7D1114B1878E0B9012384F880
:1032E0004C30F8BD66682289EF5C92B2B7542289EF
:1032F000013292B2228122892688964200D820810A
:103300002089628992B28242E2D12173E0E70420EF
:10331000E7E70520E5E70020E3E700BFAA9A0020E1
:10332000222AF8B504460D4634D11030FEF7C5FF09
:10333000202831D994F8E93033B10023238363770F
:10334000638384F8E930237701231946227F02F052
:10335000FF0052B161770133222BF7D1104B18785F
:10336000E0B9012384F84C30F8BD6669228BEF5C2C
:1033700092B2B754228B013292B22283228B268AD8
:10338000964200D82083208B628B92B28242E2D197
:103390002177E0E70420E7E70520E5E70020E3E701
:1033A000AA9A0020428903899BB2934205D1027BED
:1033B00002F0FF0382B100887047438902899A4274
:1033C00004D903894089181A80B270474289038959
:1033D00000881844801AF7E718467047F8B5D0F807
:1033E000DC3004460F461646013300F16F05C0F885
:1033F000DC30D0F8E0300133C0F8E030D0F8E43011
:103400000133C0F8E43090F86E300B2B13D9002351
:1034100080F86E302046FFF7C5FF00286BD104F11D
:103420001000FFF7BFFF002865D10C22364928465F
:1034300014F09CFD01E0002BECD094F86E100322F8
:1034400004F1AF00294414F091FD012E4FF000006B
:103450000CBF0823042384F8870084F88930D4F84B
:10346000DC3084F88800132B06D904EB0610FFF734
:1034700099FF003018BF01207B1E94F86E2059423E
:103480005941002A3BD0B2F1090C4FF0010518BF99
:103490004FF0010C94F8AF30012F80EA010681EA69
:1034A000050143EAC0100CBF08230023614514BF87
:1034B00020210021184394F8B03043EAC513AE42EE
:1034C00014BF02250025664514BF0226002684F895
:1034D000AF0043EACC032B4384F8B03094F8B1300A
:1034E0001943032331431A44C4F8D83084F8B11087
:1034F00084F86E20F8BD0C2204F17B0197E7154695
:103500004FF0010CC6E700BFC0B40108F8B500EBEE
:10351000011605460C463046FFF744FF202809D91E
:10352000D5F8DC30132B05D904F1380355F82330D6
:10353000052B10D82C44002205F14D0305F16E0136
:1035400084F8E82013F8010B8B4283F8610083F8BC
:103550003920F7D126E005EB041405F1870105F1C8
:10356000A80700202346B4F808C0628992B26245D9
:1035700001D1227B92B1D6F804C05A8992B21CF8CC
:10358000022081F8282018735A89013292B25A8198
:103590005A89B6F800C0944500D8588101F8010B4B
:1035A0008F42E0D12123C5F8D830F8BD38B590F866
:1035B0004C300446002B41D0B0F8D820F2B123485B
:1035C00003F0B8FC0546142D38D9B4F8DA3020469B
:1035D000143DE2180133ADB292F8AF1092F8872093
:1035E000A4F8DA30FFF7A6FDB4F8DA20B4F8D83042
:1035F0009A42E8D30023C4F8D8301FE0013B042BE3
:103600001DD8DFE803F0031C100A15000021FFF7A6
:103610007DFF042384F84C300CE000220121FFF7E9
:10362000DDFE0323F6E70121FFF770FF0223F1E738
:10363000FFF7C4FDB4F8D830002BC0D138BD01224B
:103640000021FFF7CBFE0123E4E700BF708A0020D2
:103650000022034630B503F8082B002400F13002A5
:103660000025E3E802459A42FBD100F5D053002142
:103670000C3322F8021B9342FBD100F5EE511A469F
:1036800000230C3122F8023B9142FBD141F6CC528F
:103690002F49835041F6D052815041F6D4522D49E2
:1036A000815041F6D85242F20F71815241F6DC52FC
:1036B0004FF00001835000F5EF52136041F6E452E1
:1036C000835241F6E652815441F6E852002183507C
:1036D00041F6EC52835041F6F052835041F6F452D9
:1036E000835041F6F852835000F5EF5200F5F55340
:1036F0001C32043342F8041B9342FBD11A4600F5F6
:10370000FA5300210C3342F8041B9342FBD11A46B2
:1037100000F5FF530021143342F8041B9342FBD100
:103720001A4600F5025300211C3342F8041B934251
:10373000FBD100F503510022063103F8012B994219
:10374000FBD142F2C803C25042F2CC03C25230BD98
:1037500000000F270F270F27002341F6DC521149E5
:103760000370835000F5EF52136041F6CC52835042
:1037700041F6D052815041F6D4520B49815041F666
:10378000D85242F20F71815241F6E452835241F60F
:10379000E652835442F2C802835042F2CC02835272
:1037A000704700BF00000F270F270F2742F2CC03FE
:1037B00010B50446C05AB0B142F2C8032B22E358F8
:1037C000B3FBF0F3C3F3072081F82A3081F8290016
:1037D000064807F0C3F8002342F2C802A35042F2A1
:1037E000CC02A35210BD2922F2E700BFC0D90020AD
:1037F00042F2CC0310B50446C05AA0B142F2C8034D
:103800000E22E358B3FBF0F3C3F307204B730873A6
:10381000064807F0CFF8002342F2C802A35042F254
:10382000CC02A35210BD0C22F2E700BFC0D9002089
:1038300041F6CC53002170B5C35A0446013350F809
:1038400033301F4823F07F43584008F08FFF022891
:1038500033D841F6D0531B4D18200021E25A02F212
:103860006D139BB2B3F5F07F24BFA2F173039BB23B
:1038700003F6045215F8016B04EB4202B2F904207E
:10388000CEB1891A5A1D013892B2B2F5F07F29BF24
:103890006FF4ED7213469B189BB210F0FF00E7D156
:1038A00041F6DC53E2588A4204DAE15041F6CE5345
:1038B000E052012070BD1144E4E70020FAE700BFA8
:1038C00050765500EDBC0108F8B541F6CC530578AB
:1038D00004460021C35A022D03F1010318BF00253D
:1038E00050F83330314823F07F43584008F03EFF12
:1038F000A84258D841F6D0532D4E18200025E25A40
:1039000002F26D139BB2B3F5F07F24BFA2F17303F3
:103910009BB203F6045116F8017B04EB4101B1F9A7
:103920000410002F3DD06D1A591D013889B2B1F530
:10393000F07F29BF6FF4ED770B46DB199BB210F0D7
:10394000FF00E6D104F5EF531968A94228DA1D609B
:1039500041F6E45341F6D251E05241F6D453E252DB
:10396000531D9BB2B3F5F07F24BF6FF4ED701318B5
:1039700001206352531C41F6D8519BB2B3F5F07F3E
:1039800024BF6FF4EF73D318635202F2DF1341F6D2
:10399000D6519BB2B3F5F07F28BF02F1FF336352DB
:1039A000F8BD0D44C0E70020FAE700BF68B4AA00E4
:1039B000D5BC010838B504460D46FFF739FFB0B154
:1039C00041F6E6530522E25441F6CE52A35A03F1E2
:1039D0001800013324F81050A352002342F2C80209
:1039E000A35042F2CC02A3520123237038BD2046DB
:1039F000FFF76AFF0028F9D00649074807F076FB71
:103A00000121064803F0B4FA0121044803F0BCFA8E
:103A10000223EAE76FBD0108C0D90020708A0020A8
:103A20002DE9F043079E0025BDF820C0DFF844E0F3
:103A3000DFF84480ACB29C421AD231F9129004F003
:103A40000704EF100532B9F1000F05F10105F05D33
:103A500092B2B5BF18F804401EF80440204320403D
:103A6000624528BFA2EB0C02F05528BF92B2E1E7F5
:103A7000BDE8F08342B701084AB7010841F6CC53CC
:103A80002DE9F041C35A0446002586B0013329468A
:103A900050F833304F48584008F068FE012818D8D5
:103AA0004D494E4807F022FB29464D4803F060FA85
:103AB00029464B4803F068FA484806F0C5FF41F62E
:103AC000DC53E55004F5EF531D60257006B0BDE8EA
:103AD000F08141F6D653E15A41F6D853E25A41F605
:103AE000D0539142E35A24D2994204D89A4202D345
:103AF0002046FFF7E9FE41F6E45834F80830952BEC
:103B00001AD93849354807F0F1FA0021344803F052
:103B10002FFA0021324803F037FA304806F076FFDA
:103B2000002341F6DC52A35004F5EF5213602370DA
:103B3000CCE79942DAD8DBE741F6D05341F6D857C3
:103B4000E25AE35B9A42C1D14FF4F07341F6D25688
:103B500002AD04F5D0510193204600956023A25B8D
:103B60000C31FFF75DFF34F808201521B2FBF1F3AB
:103B700001FB13239BB233BBA2B955231A49174843
:103B80008DF8113041F22D63ADF8123041F6D65365
:103B9000E35E0193E35F009341F6D453A25FE35EDB
:103BA00008F036FB29462046FFF722FE41F6E45294
:103BB000A35A0133A352002341F6DC52A35004F56B
:103BC000EF54236082E70C222946044806F0F2FEF7
:103BD000ECE700BF5E13AAAA05BD0108C0D900200A
:103BE000708A002025BD01084DBD010841F6E8534B
:103BF0002DE9F04FC45841F6EC5341F6FC5941F61B
:103C00004C7B50F803E004F007020B680EEB03084E
:103C100041F6F453C65847460B6906EB030CE3081C
:103C2000E04500EB8303A8BF6746E04553F8095021
:103C300041F6A468B5BFDFF8E8C0DFF8E8C01CF8BB
:103C400002C01CF802C0B4BF0CEA05054CEA050529
:103C500043F809504D68AE444D692E44F44653F87C
:103C60000850B645A8BFB446B645B5BF2C4E2D4E3C
:103C7000B65CB65CB4BF3540354343F8085041F6F6
:103C8000F0558E6950F805E08D680EEB050A41F697
:103C9000F8554559D04605EB060953F80B60CA455F
:103CA000A8BFC846CA45B5BFDFF87490DFF8749066
:103CB00019F8029019F80290B4BF09EA060649EA19
:103CC000060641F6F47943F80B60CE68C96976447C
:103CD0000D4453F80910B646AE42A8BFAE46AE42F8
:103CE00019DA0F4DAA5C0A4043F8092041F6EC535B
:103CF0000134C75041F6F05340F803C041F6F45385
:103D000040F8038041F6F85340F803E041F6E853E9
:103D1000C450BDE8F08F034DAA5C0A43E4E700BF3E
:103D200032B701083AB70108D1E9003270B583F023
:103D3000010588B0D11882F001062A44334400916D
:103D40007419029301940793CDE905126946CDE9F0
:103D50000324FFF74BFF08B070BD0000002240F2C3
:103D60004911F0B513462E4D42F29C042D4F032B02
:103D70001DD8DFE803F002203846CE1001F007031B
:103D800006F27E7615F803C000EB860673681CEA1F
:103D9000030318BF022300EBD20C02F007061CF845
:103DA00004E0BE5D06EA0E0601320CF8046011F173
:103DB000FF31DCD2F0BDCE1001F0070306F5F56649
:103DC00015F803C000EB860673681CEA030318BFEE
:103DD000022300EBD20C02F007061CF804E0AE5DF3
:103DE00046EA0E06E0E7CB1001F0070603F2D273B5
:103DF000AE5D00EB83035B681E420CBF012303230F
:103E0000C9E7CE1001F0070C06F2FC7615F80CC0DD
:103E100000EB860676681CEA060F08BF0123D8E788
:103E20003AB7010832B7010830B54FF0FF32481EEB
:103E300001F126040F4D10F8013F5340C2F3072251
:103E40008442DBB235F8133083EA02031A46F2D11A
:103E5000DB4391F827009BB2DAB2904207D191F888
:103E60002820B2EB132F0CBF0120002030BD002012
:103E7000FCE700BF32B501082DE9F0434B1E0546B3
:103E800099B016468D4801F1520413F8017F10F8DD
:103E9000012B9C4282EA07021A70F6D1002303AA82
:103EA0001846013302F8010B542BFAD1DFF814E263
:103EB0000022802774460EEB4200B2F5257F63DBBB
:103EC000002441F6EC524FF080084027AC5041F6F8
:103ED000F052AC5041F6F452AC5041F6F852AC50AE
:103EE00041F6E852AC5018AB284603EBE40313F854
:103EF000542C04F00703023428FA03F127FA03F3E1
:103F0000114214BF012100211342029101A914BFE3
:103F1000012300230193FFF707FFB4F5257FE2D1CA
:103F2000FFF71CFF731E06F12802002103F8011F92
:103F30009A42FBD140F2491242F29C04604F4FF08A
:103F4000010C104605EBE20102F00708831A11F894
:103F500004E017F808101EEA010F09D0D90803F091
:103F6000070316F801E00CFA03F343EA0E03735457
:103F700012F1FF32E6D231462846FFF755FF19B05D
:103F8000BDE8F0831A4698E7D31011F803C01CF07F
:103F9000010F0CD018AB90F800809844437818F8C3
:103FA000549C27FA03F343EA090308F8543C1CF035
:103FB000020F0CD018AB90F802809844C37818F820
:103FC000549C27FA03F343EA090308F8543C1CF015
:103FD000040F0CD018AB90F804809844437918F87B
:103FE000549C27FA03F343EA090308F8543C1CF0F5
:103FF000080F0CD018AB90F806809844C37918F8D5
:10400000549C27FA03F343EA090308F8543C131DB0
:104010000830B3F5257FB5DA1CF0100F0FD014F877
:1040200013000DF1600804EB430340445B7810F883
:10403000548C27FA03F343EA080300F8543C1CF0BD
:10404000200F10D0531D0DF1600814F8130004EB7D
:10405000430340445B7810F8548C27FA03F343EA97
:10406000080300F8543C1CF0400F10D0931D0DF1D4
:10407000600814F8130004EB430340445B7810F825
:10408000548C27FA03F343EA080300F8543C1CF06D
:10409000800F10D0D31D0DF1600C14F8130004EB49
:1040A000430360445B7810F854CC27FA03F343EAE7
:1040B0000C0300F8543C0832FDE600BF52B701087B
:1040C0003AB70108ADB7010870B541F6E655A2B0A0
:1040D00004460E46435D23B1FFF7AAFB635D013B37
:1040E000635541F6CE52A35A03F1180001339BB237
:1040F00024F81060A35240F6E942934219D140F6E9
:10410000E4430DAD052204F13001019320460095F2
:104110004FF42573FFF784FC02AA29462046FFF7D7
:10412000ABFE78BB41F6DC532070E05004F5EF5352
:10413000186041F6CE53E25A40F6EE439A421FD140
:1041400041F6E45300221649E25241F6D0534FF0B3
:10415000EE721448E25041F6D453134AE2504FF441
:10416000EC7341F6D852A3524FF4EB72CDE9003212
:1041700040F2D7134FF4EE7208F04AF8022323708E
:1041800022B070BD0121094802F0F2FE012107486A
:1041900002F0FAFE02A92046FFF708FBC9E700BFBC
:1041A00090BD0108C0D90020D701D601708A002037
:1041B0002DE9F04700F5EE5804460D4616461F4619
:1041C0004FF0000908F10C081FFA89F39F424AD901
:1041D00042F2C80236F8191041F6D05AA3580B44DF
:1041E000A35042F2CC02A35A0133A352B8F80020E4
:1041F00035F9191004EBC202D2E90230DB18404154
:104200000029B8BF43F00103C2E9023034F80A3094
:1042100003F6045304EB430399802378012B05D064
:10422000022B1CD02046FFF7C5FB02E02046FFF71B
:104230004BFF34F80A3009F1010901339BB2B3F5A1
:10424000F07F28BF002324F80A30B8F8003001338B
:104250009BB2042B88BF0023A8F80030B4E72046A7
:10426000FFF70CFCE5E7BDE8F087000070B50446F9
:1042700000254FF4B97004F11C062581208065816A
:104280006573257313F0D4FD04F144033246606076
:10429000A561C4E9045522F8025B9342FBD104F501
:1042A0002771002203F8012B9942FBD13C23C4F86B
:1042B0009C2200212822A4F8A032304613F0F0FE00
:1042C00005232046237403236382024BC4E9053689
:1042D00070BD00BFBC0500202DE9F04F501E99B005
:1042E00002F15209002403AD034603F8014F99453A
:1042F00005F8014BF9D14B1EDFF8BCA10093002358
:104300001D461C460099AC460027254611F8016F52
:10431000CDE900161E46012101FA07F40199214258
:1043200014BF0124002404EB0C0EAC44A4440EF092
:10433000010E1CF0010F0CD006F0070C18A91AF89A
:104340000C8001EBD60C1CF854BC48EA0B080CF8A6
:10435000548CBEF1000F0ED006F1010C18A901EB30
:10436000DC0E0CF0070C1EF8548C1AF80CC04CEA4A
:10437000080C0EF854CC01370236AC46082F40F03A
:1043800087801033B3F5287FBCD1DFF830C100231C
:10439000012564460CEB4301B3F5257F7CD218AEB2
:1043A00006EBD30616F8546C37060AD591F800E0F0
:1043B0004F7812F80E8005FA07F747EA080702F867
:1043C0000E7077060AD591F802E0CF7812F80E80C9
:1043D00005FA07F747EA080702F80E70B7060AD58C
:1043E00091F804E04F7912F80E8005FA07F747EAD2
:1043F000080702F80E70F7060AD591F806E0CF79A3
:1044000012F80E8005FA07F747EA080702F80E705F
:104410001F1D0831B7F5257F3CD231070BD514F8A5
:1044200017E004EB4707797812F80E7005FA01F1EE
:10443000394302F80E1071070CD5591D14F811708C
:1044400004EB4101497812F807E005FA01F141EA6D
:104450000E01D155B7070CD5991D14F8117004EB56
:104460004101497812F807E005FA01F141EA0E012D
:10447000D155F1070AD5D91D14F8116004EB41019B
:104480004978975D05FA01F139439155083381E781
:10449000254640E73B467FE7064A10F8011F12F821
:1044A000013B484583EA01030370F6D119B0BDE82A
:1044B000F08F00BFB9BD0108B1BD010814BE0108ED
:1044C00070B59AB00C460023012202A940F249358A
:1044D0004FF6B74632EA040C4FEA420208BF21F811
:1044E0001360D2B218BF21F813500133082BF1D159
:1044F00006AA103012F0C4FD002306AA0121009381
:104500002823024803F00CF91AB070BD708A00200D
:1045100001EB4101490001F59671B1F5167F8ABFA3
:104520004FF41673A0F8A012A0F8A032704703460B
:1045300000895A8992B2824203D11A7B02F0FF00AD
:1045400082B158685A8992B2825C0A70002119734C
:104550005A89013292B25A815A891888904200D8F9
:104560005981012070470000428903899BB2934220
:1045700070B50446A2B0B0F89C5220D1037B0BB1B9
:1045800003880BB9002D5BD0638962689BB2D35C52
:10459000002B4ED1002D56D15C4B1B78EBB9B4F8F3
:1045A000A002AA22A9B2B4F89C3288423DD9591C73
:1045B00023440135A4F89C1283F84420F2E7438990
:1045C00002899A4204D9038942899B1A9BB2D8E78F
:1045D0004289018803890B44F7E70DF10301204666
:1045E000FFF7A5FF01AB204659190135FFF79FFFE3
:1045F000292DF7D10DF13202204601A9FFF76CFEFB
:104600004AF2EA630CA80022ADF83030B4F89C32CC
:104610009918013210F8015B14FA81F1552A81F8DA
:104620004450F5D15533A4F89C320023A4F89E32AF
:1046300003E0012B06D0022B38D0B4F89C3213B91A
:1046400022B070BDE5B1324802F074FC0546282D59
:10465000F6D9B4F89E322046283D5A1C2344ADB208
:10466000A4F89E2293F84410FFF72AFFB4F89E2284
:10467000B4F89C329A42EAD30023C4F89C32DFE7B4
:104680000C250CA92046FFF752FFB4F89C12013DFF
:1046900020464B1C4431A4F89C322144FFF747FFCD
:1046A00015F0FF05F1D1A4F89E52C6E7002DCAD13E
:1046B0000CA92046FFF73BFFB4F89C325522C826D0
:1046C00003F112017A2589B2E01880F84420581CC1
:1046D00014FA80F080F84420981C14FA80F080F8D6
:1046E0004420D81C14FA80F080F84420181D14FAD5
:1046F00080F080F84460581D063314FA80F09BB2B5
:1047000080F844508B42DFD18DE700BFAA9A002089
:10471000708A002008B5FDF7D0FD0D23B0FBF3F043
:10472000C0B208BD037B10B503F0FF021BB101232B
:104730004373002010BD446803899BB2E154038990
:1047400001339BB2038103890188994200D8028119
:10475000028943899BB293424FF0010300D1037356
:104760001846E7E7292A70B506460C4619D1FDF729
:10477000A4FD292806D802B20B490C4806F098FF80
:10478000052070BD651E283400213046FFF7CAFFA2
:1047900015F8011F3046FFF7C5FFA542F8D10020EC
:1047A000EFE70420EDE700BF3CC30108C0D90020BB
:1047B0000C2A70B506460C4619D1FDF77EFD0C2873
:1047C00006D802B20B490C4806F072FF052070BDF6
:1047D000651E0B3401213046FFF7A4FF15F8011FB9
:1047E0003046FFF79FFFA542F8D10020EFE70420F5
:1047F000EDE700BF79C30108C0D9002010B5044619
:10480000FDF75BFD024628B90548064906F050FF52
:10481000052010BD02212046FFF784FF0020F8E7A5
:10482000C0D900205CC3010800224FF4804102601F
:1048300081808271826002737047C901D201018058
:104840004942828041807047B0F9003030B593B161
:10485000827932B98B420ADC0123837100238360A1
:1048600003738368B3F5166F07D9002119E0B0F917
:1048700002308B42F0DA084630BD047B0D49621CE1
:10488000B0F9045051F82410D2B269430B2A0273D4
:104890004FEAE13188BF002201F30F0109B288BF5E
:1048A0000273013342F6DF6293428360E3D900234F
:1048B0008371E0E798C3010838B500F678450446EF
:1048C000284602F0AAF8A0B1284602F0ABF880B161
:1048D0000849094806F00AFC0023284684F84C3CA5
:1048E00002F091F804F6584002F08DF8012384F8A4
:1048F000983C38BDD7C40108C0D90020034670B524
:10490000D0E90254D0E904021E686A4300FB012288
:10491000986906FB0022D8695E6800FB1422186AB9
:1049200006FB1020C01300F30E0000B2C3E90054D0
:10493000C3E9021070BD38B50025044600F5456096
:1049400000F8045C02F05FF804F6584002F05BF8EF
:1049500004F6684002F057F804F5476002F053F897
:1049600004F6784002F04FF804F5486002F04BF886
:1049700004F6884002F047F804F5496002F043F875
:1049800004F5406001F024FD04F5806001F030FF83
:1049900004F5006001F02CFF204601F029FF04F52A
:1049A000446002F017F8A4F8585D04F55660A4F8C6
:1049B0005A5D84F85D5D84F85C5D02F055F804F59D
:1049C000526001F0F1FD04F6284001F0C3FF84F8C5
:1049D000985CA4F8805D38BD2DE9F74F9DF8344010
:1049E00099469DF838300F46C4EB04149DF84010EA
:1049F00001939046A4009DF844209DF8483000F5AE
:104A0000466AA4B29DF8305080F84D1C064680F8E6
:104A10004E2C214680F84F3C002250469DF83CB079
:104A200001F0DFFF0022C5EB051106F545608900A6
:104A300089B201F0D6FF14B1504601F0DFFF019BAF
:104A40004246394630460C934B46CDF834B003B05D
:104A5000BDE8F04F01F0C0BD2DE9F047BDF824706E
:104A600004469DF820608846914600213A4600F6AB
:104A700078409A469DF8285001F0B3FF2EB13A468F
:104A8000314604F5476001F0ACFF53464A464146C3
:104A900004F58060CDE90855BDE8F04701F09CBD04
:104AA0002DE9F04F85B01D46044616469DF8383076
:104AB0009DF84CE000939DF83C309DF850C0019368
:104AC0009DF840309DF8540002939DF85C309DF8AD
:104AD000582003939DF864309DF844B0A4F81C3D21
:104AE00084F818ED84F819CD9DF848A084F81A0DC3
:104AF00004F6584084F81B2D00229DF860709DF844
:104B000068909DF86C8001F06CFF0022594604F615
:104B1000684001F066FF0022514604F5486001F04C
:104B200060FF314604F5446001F022FF32464946F9
:104B300004F60850FFF781FE3A46039904F6284030
:104B4000A4F83E8D01F083FE294604F54060DDE9BE
:104B5000002301F0B3FB40B9029A294604F54260F4
:104B600005B0BDE8F04F01F03DBC05B0BDE8F08FE9
:104B700070B41D469DF810400126A0F81E2DBDF80A
:104B80000C302A4680F83C6D00F50060CDE9034406
:104B900070BC01F021BD000070B504460D4600F563
:104BA000456001F033FF294604F6584004F6884674
:104BB00001F02CFF294604F5466001F027FF294645
:104BC00004F6684001F022FF294604F5476001F031
:104BD0001DFF294604F6784001F018FF294604F528
:104BE000486001F013FF2946304601F00FFF04F53D
:104BF0004960294601F00AFF304601F00EFF68B116
:104C0000304601F00FFF48B194F84C1C044806F000
:104C10007BF93046BDE8704001F0F0BE70BD00BFCA
:104C2000C0D9002038B504460D46D9B100F6584524
:104C3000284601F0F2FE40B3284601F0F3FE20B30F
:104C40001248134906F052FA0423284684F84C3CD3
:104C500001F0D9FE94F83C3DBBB10C48BDE83840AA
:104C600006F072B90B4802F083F92946094802F0B0
:104C70008BF90949054806F039FA032304F6784010
:104C800084F84C3C01F0BAFEE4E738BDC0D90020FE
:104C900023C40108708A002037C4010870B5044697
:104CA00000F678450E4699B10121144802F060F9EA
:104CB0000121124802F068F91148124906F016FA6B
:104CC0000223284684F84C3CBDE8704001F09BBEAE
:104CD000284601F0A2FE78B1284601F0A3FE58B1A3
:104CE0000949074806F002FA284684F84C6C01F09E
:104CF0008AFE04F65840E7E770BD00BF708A0020C6
:104D0000C0D90020C2C40108D7C4010838B5044680
:104D1000A9B100F65845284601F07FFEE0B12846CB
:104D200001F080FEC0B10D480D4906F0DFF90923FE
:104D3000284684F84C3CBDE8384001F064BE074882
:104D4000084906F0D3F9082304F6784084F84C3C6F
:104D5000BDE8384001F052BE38BD00BFC0D90020C8
:104D60006BC4010880C4010810B5044661B108484D
:104D7000084906F0BBF9072304F6784084F84C3C58
:104D8000BDE8104001F03FBEBDE81040FFF794BD04
:104D9000C0D90020EAC4010838B504460D4699B9C7
:104DA0000A4802F0E5F82946084802F0EDF80848FC
:104DB000084906F09BF9052304F6784084F84C3C3A
:104DC000BDE8384001F01ABE38BD00BF708A00202F
:104DD000C0D900200AC4010870B5044600F6784521
:104DE0000E4699B10121144802F0C2F8012112487F
:104DF00002F0CAF81148124906F078F9042328464F
:104E000084F84C3CBDE8704001F0FDBD284601F03F
:104E100004FE78B1284601F005FE58B1094907485B
:104E200006F064F9284684F84C6C01F0ECFD04F6B9
:104E30005840E7E770BD00BF708A0020C0D900204D
:104E400023C40108D7C4010810B5044661B9074856
:104E5000074906F04BF90A2304F6784084F84C3CE5
:104E6000BDE8104001F0CABD10BD00BFC0D9002090
:104E700051C4010810B5044661B10848084906F05C
:104E800035F9092304F6784084F84C3CBDE810401D
:104E900001F0B9BDBDE81040FFF70EBDC0D900203C
:104EA0006BC4010838B500F546650446284601F094
:104EB000B4FD78B1284601F0B5FDA0B10A490B4810
:104EC00006F014F9204601F0ACFC2846BDE8384055
:104ED00001F094BD0548044906F008F92046BDE8F4
:104EE000384001F09EBC38BDC8C30108C0D90020BD
:104EF00070B5044600F668450E46E9B1284601F053
:104F000091FD002843D02249224806F0EFF8022301
:104F1000284684F84C3C01F076FD94F84D3CB3B340
:104F200094F84F3C9BB32046FFF7BCFF04F5456067
:104F3000BDE8704001F062BD174802F019F8314633
:104F4000154802F021F81549124806F0CFF8284616
:104F500084F84C6C01F057FD04F6584001F053FD05
:104F600004F5476001F04FFD04F5456001F04BFD8D
:104F700004F6884001F047FD012384F8983C94F83A
:104F80003C3D23B10348BDE8704005F0DDBF70BD76
:104F9000C2C40108C0D90020708A0020D7C401080B
:104FA00038B504460D4699B300F65845284601F039
:104FB00034FDD8B1284601F035FDB8B11E491F486F
:104FC00006F094F8042304F5476084F84C3C01F0A3
:104FD0001AFD284601F017FD04F5446001F0F4FCC9
:104FE00094F83C3D13B1154805F0AEFF04F5456556
:104FF000284601F012FDF0B1284601F013FDD0B1B2
:105000002046FFF74FFF2846BDE8384001F0F6BCC8
:105010000B4801F0ADFF2946094801F0B5FF0949E9
:10502000064806F063F8032304F6784084F84C3C05
:1050300001F0E4FCD4E738BD23C40108C0D9002046
:10504000708A002037C4010870B5044600F6784520
:1050500029B301212B4801F08BFF0121294801F0E0
:1050600093FF2948294906F041F80223284684F88D
:105070004C3C01F0C8FC04F54565284601F0CDFC28
:1050800000283ED0284601F0CDFC002839D020462B
:10509000FFF708FF2846BDE8704001F0AFBC284686
:1050A00001F0BBFC0028E6D0284601F0BBFC00283C
:1050B000E1D0154804F54766154906F017F80B23AB
:1050C000304684F84C3C01F0A8FC18B1304601F0A1
:1050D000A9FC50B10F490C4806F008F804F58060AF
:1050E00001F09FFB304601F08EFC284601F08BFC5E
:1050F00004F6584001F087FC04F5486001F07EFC9E
:10510000B9E770BD708A0020C0D90020C2C4010870
:105110009BC40108A9C4010870B5044600F668459F
:105120000E46E1B1284601F07DFCA0B31A491B48A8
:1051300005F0DCFF0723284684F84C3C01F063FCB3
:1051400094F84D3C3BB394F84F3C23B32046FFF713
:10515000A9FE04F54560BDE8704001F04FBC104960
:105160000E4805F0C3FF284684F84C6C01F04BFC58
:1051700004F6584001F047FC04F5476001F043FC99
:1051800004F5456001F03FFC04F6884001F03BFC6B
:10519000012384F8983C70BDEAC40108C0D90020FE
:1051A000D7C4010838B5044669B300F65845284607
:1051B00001F033FCA8B1284601F034FC88B118494D
:1051C000184805F093FF092304F5476084F84C3C28
:1051D00001F019FC284601F016FC04F5446001F0CA
:1051E000F3FB04F54565284601F017FCB8B12846E5
:1051F00001F018FC98B12046FFF754FE2846BDE8A0
:10520000384001F0FBBB0849064805F06FFF082352
:1052100004F6784084F84C3C01F0F0FBE1E738BD3F
:105220006BC40108C0D9002080C4010870B50446D1
:1052300000F67845E9B12848284905F057FF0723CB
:10524000284684F84C3C01F0DEFB04F54565284611
:1052500001F0E3FB00283ED0284601F0E3FB0028E4
:1052600039D02046FFF71EFE2846BDE8704001F009
:10527000C5BB284601F0D1FB0028E6D0284601F046
:10528000D1FB0028E1D0144804F54766144905F025
:105290002DFF0B23304684F84C3C01F0BEFB18B1C7
:1052A000304601F0BFFB50B10E490B4805F01EFF20
:1052B00004F5006001F0B5FA304601F0A4FB284681
:1052C00001F0A1FB04F6584001F09DFB04F5486095
:1052D00001F094FBB9E770BDC0D90020EAC4010811
:1052E0009BC40108B5C4010838B504460D46B9B9D8
:1052F000154801F03DFE2946134801F045FE1349CB
:10530000134805F0F3FE052384F84C3C94F84E3C1A
:1053100013B12046FFF7C6FD04F6784001F06EFB9E
:1053200004F54565284601F078FB58B1284601F0A0
:1053300079FB38B12046FFF7B5FD2846BDE8384077
:1053400001F05CBB38BD00BF708A00200AC40108B0
:10535000C0D9002038B5044600F6784521B30121B4
:10536000284801F005FE0121264801F00DFE2648DF
:10537000264905F0BBFE0423284684F84C3C01F086
:1053800042FB04F54565284601F047FB002838D06C
:10539000284601F047FBA0B32046FFF783FD2846CF
:1053A000BDE8384001F02ABB284601F036FB002852
:1053B000E7D0284601F036FB0028E2D01449124815
:1053C00005F094FE0B2304F5446084F84C3C01F096
:1053D00001FB10490C4805F089FE04F5806001F0DE
:1053E00020FA284601F00FFB04F5476001F00BFBA3
:1053F00004F6584001F007FB04F5486001F0FEFA9E
:10540000BFE738BD708A0020C0D9002023C401083E
:105410009BC40108A9C4010838B5044651B90F4816
:105420000F4905F063FE0A2304F6784084F84C3CEB
:1054300001F0E4FA04F54565284601F0EEFA58B1AA
:10544000284601F0EFFA38B12046FFF72BFD284639
:10545000BDE8384001F0D2BA38BD00BFC0D9002045
:1054600051C4010838B5044600F67845E1B1254835
:10547000254905F03BFE0923284684F84C3C01F001
:10548000C2FA04F54565284601F0C7FA002838D06D
:10549000284601F0C7FAA0B32046FFF703FD2846CF
:1054A000BDE8384001F0AABA284601F0B6FA002853
:1054B000E7D0284601F0B6FA0028E2D01349114897
:1054C00005F014FE0B2304F5446084F84C3C01F015
:1054D00081FA0F490B4805F009FE04F5006001F060
:1054E000A0F9284601F08FFA04F5476001F08BFA25
:1054F00004F6584001F087FA04F5486001F07EFA9E
:10550000BFE738BDC0D900206BC401089BC40108A7
:10551000B5C4010810B5044600F6584001F06EFA13
:1055200004F54760BDE8104001F068BAF8B50446DC
:10553000174600F5456571B301212E4801F018FDAD
:1055400001212C4801F020FD2B492C4805F0CEFD0F
:10555000022384F84C3C2A49284805F0C7FD04F58D
:10556000806001F045F904F5006001F041F9204642
:10557000FFF7D0FF284601F050FA002838D028461F
:1055800001F050FAA0B32046FFF78CFC2846BDE896
:10559000F84001F033BA2AB11A49184805F0A6FDBF
:1055A0000723D6E700F54866304601F036FA0028B2
:1055B000E0D0304601F036FA0028DBD012490F481F
:1055C00005F094FD304684F84C7C01F01CFA04F69A
:1055D000884001F018FA94F84E3C13B12046FFF7CA
:1055E00061FC284601F00FFA012384F8983CC1E7DA
:1055F000F8BD00BF708A0020C2C40108C0D90020D5
:10560000D6C30108EAC40108D7C4010808B500F5EB
:10561000566001F0C9FAF023B0FBF3F0C0B208BD48
:1056200008B500F5566001F028FA002008BD037B9C
:1056300010B503F0FF021BB101234373002010BD1E
:10564000446803899BB224F81310038901339BB289
:10565000038103890188994200D802810289438924
:105660009BB293424FF0010300D103731846E6E763
:1056700070B51825002400F554664D43AC4205D0A2
:1056800000213046FFF7D3FF0134F7E770BD00007B
:105690002DE9F041044600F08AFF0025012604F5BB
:1056A000806004F6884800F082FF04F5006000F096
:1056B0007EFF04F5406000F0F3FD04F5426000F069
:1056C0008DFE04F6284001F0BAF804F5446001F0BC
:1056D00047F9C4F84C5C04F5456004F5496701F0EE
:1056E0007CF904F6584001F078F904F5466001F0C1
:1056F00074F904F6684001F070F904F5476001F0B0
:105700006CF904F6784001F068F904F5486001F09E
:1057100064F9404601F061F9384601F05EF94FF452
:1057200035734FF4B56284F8985CC4F8AC3C04F669
:105730000850C4F8B43C464BC4F8B02CC4F8B83C8C
:1057400045F26833434AC4F8BC3C4FF40043C4F804
:10575000D82C414AC4F8D03CC4F8DC2C44F66C2266
:10576000C4F8F43CC4F8FC3C3C4BC4F8E02CC4F84E
:10577000003D47F6E4233A4AC4F8043DC4F8F82C47
:10578000C4F8A45CC4F89C5CC4F8A85CC4F8A05C31
:10579000C4F8D45CC4F8C85CC4F8C05CC4F8CC5C81
:1057A000C4F8C45CC4F8EC5CC4F8E45CC4F8F05C15
:1057B000C4F8E85CFFF738F84FF001134FF4C871F4
:1057C000C4F8186DC4F81C3D04F5526000F060FE8A
:1057D00040F66113A4F8485D41F2C220A4F8403DB0
:1057E000A4F84A5D84F83C5DA4F83E6D84F84C5DF5
:1057F00084F84D5D12F01CFB4FF41663A4F8585D5D
:10580000A4F8503DC4F8440D4FF49650A4F85A5DE6
:1058100084F85D5D84F85C5D12F00AFBC4F8540DF9
:1058200004F5566001F009F92A4631464046A4F8CD
:10583000805D01F0D6F896222946384601F0D1F86D
:1058400020466421FFF714FF2046BDE8F08100BF29
:10585000F96BFFFF0080FFFF5D3BFFFFB505FFFF1A
:105860000000FFFF70B51825002400F555664D4374
:10587000AC4205D000213046FFF7D9FE0134F7E7EE
:1058800070BD000038B5044600294BD000F66845CD
:10589000284601F0AEF8C0B14049414805F026FC69
:1058A0000123284684F84C3C01F0A8F894F84D3CBC
:1058B0002BB194F84F3C13B92046FFF7F3FA94F854
:1058C0004C3C013B012B0BD938BD3649344805F01F
:1058D0000DFC022384F84C3C94F84D3C002BEBD19A
:1058E00032212046FFF7BEFF2046FFF713FE04F5E6
:1058F000456001F083F804F5496001F084F8012166
:10590000294801F035FB0121274801F03DFB04F651
:10591000884001F073F894F84C1C2148BDE83840E9
:1059200005F0F2BA002ACFD000F66845284601F00B
:1059300060F8C0B11D491A4805F0D8FB0623284677
:1059400084F84C3C01F05AF894F84D3C2BB194F893
:105950004F3C13B92046FFF7A5FA94F84C3C063BA0
:10596000012BB1D80AE012490D4805F0BFFB07230F
:1059700084F84C3C94F84D3C002BEBD1322120466E
:10598000FFF770FF2046FFF7C5FD04F5456001F005
:1059900035F804F5496001F036F8B8E7DFC30108CF
:1059A000C0D90020C2C40108708A0020F4C30108D5
:1059B000EAC4010838B590F84C3C04460B2B0AD8D1
:1059C000DFE803F00635393D4145494E53585D62E5
:1059D0002046FFF757FF94F84C3C3BBB04F5806032
:1059E00000F00FFF10BB04F5006000F00AFFE8B9FB
:1059F000204600F006FFC8B904F54965284601F0C5
:105A00000CF828B994F8983C13B1284600F0F6FF3A
:105A1000284601F002F848B1284601F003F828B101
:105A2000284600F0F0FF002384F8983C38BD20465B
:105A3000FFF75EFACFE72046FFF7B2FACBE7204642
:105A4000FFF702FBC7E72046FFF74EFCC3E72046FF
:105A5000FFF780FCBFE711462046FFF75DFBBAE782
:105A600011462046FFF79EFBB5E711462046FFF79B
:105A7000DDFBB0E711462046FFF7CEFCABE7114651
:105A80002046FFF7EFFCA6E72046FFF74FFDA2E711
:105A900010B5044609B31849184805F027FB02233E
:105AA0000121174884F84C3C01F062FA01211448A6
:105AB00001F06AFA04F6584000F0A0FF04F54960CE
:105AC00000F0A1FF04F6884000F098FF94F84C1C09
:105AD0000A48BDE8104005F017BA5AB1094907480D
:105AE00005F004FB07233221204684F84C3CFFF7E5
:105AF000B9FEDFE710BD00BFC2C40108C0D9002055
:105B0000708A0020EAC4010838B590F84C3C04467D
:105B10000A2B0AD8DFE803F00609272B2F2F0933B9
:105B2000383D42002046FFF7B3FF94F84C3CCBB918
:105B300004F54965284600F070FF28B994F8983CB0
:105B400013B1284600F05AFF284600F066FF48B11E
:105B5000284600F067FF28B1284600F054FF0023D4
:105B600084F8983C38BD2046FFF75CF8DDE7204616
:105B7000FFF794F8D9E72046FFF70EF9D5E711466D
:105B80002046FFF7C3F8D0E711462046FFF7ECF8B0
:105B9000CBE711462046FFF757F9C6E711462046E6
:105BA000FFF768F9C1E7000070B5044615460E46D8
:105BB00011B390F8803DEBB901213B4801F0D8F9D1
:105BC0000121394801F0E0F994F8813D7BB937496A
:105BD000374805F08BFA022304F6884084F84C3CE1
:105BE00000F00CFF94F84C1C314805F08DF90123AE
:105BF00084F8803D0DB940E0EAB194F8813DCBB91D
:105C000094F8803D7BB92B49294805F06FFA0723AA
:105C100004F6884084F84C3C00F0F0FE94F84C1CEC
:105C2000234805F071F932212046FFF71BFE0123BE
:105C300084F8813DBEBB94F8803DEBB100211A4849
:105C400001F096F90021184801F09EF994F8816D51
:105C50004EB91748184905F049FA84F84C6C04F617
:105C6000884000F0D0FE002384F8803D94F83C3D4D
:105C700013B10F4805F068F9ADB994F8813D93B1BF
:105C800094F8805D4DB90A480B4905F02FFA84F865
:105C90004C5C04F6884000F0B6FE012384F8983C82
:105CA000002384F8813D70BD708A0020C2C40108C1
:105CB000C0D90020EAC40108D7C4010890F8193DF2
:105CC0000BB1FFF771BF034B1B780BB1FFF772BE2F
:105CD000FFF71ABF31070020034600895A8992B2A4
:105CE000824203D11A7B02F0FF008AB158685A89B8
:105CF00092B230F912200A80002119735A890132B8
:105D000092B25A815A891888904200D8598101204C
:105D1000704700002DE9F04F9B4690F81A3D85B082
:105D200004460E4690460BB181F00106594604F632
:105D3000284A08EB4B0BAD4F2046FEF72DFFC3451D
:105D400000F0518138F9021BB4F93E3D090291FB84
:105D5000F3F194F81B3D09B2ADF80C101BB150469D
:105D600000F078FD06460DF10E0104F5566000F0D6
:105D7000D9FE054608B194F83C5D94F8183D012B16
:105D80001CD09BB1022BBDF90C1004F5406000F053
:105D9000DC8000F0B1FA0DB950B166B13B780A2B46
:105DA00009D000282A4608BF0146DFE01DB916B910
:105DB0003B780A2BC3D12A4631461CE0BDF90C10B2
:105DC00004F5406000F098FA04F55463BDF90C1036
:105DD000814618460193FFF72AFC019B03A9184648
:105DE000FFF77AFF3B7855B9B9F1000F07D10A2BBD
:105DF000A5D12A4649462046FFF760FF0AE00A2B54
:105E0000F7D02A4649462046FFF758FF94F84C3C05
:105E1000002B94D03B780A2B91D194F84C3C002B6A
:105E200000F0AD8094F84C3CBDF90C109A1FB4F909
:105E30001C5DD2B2012A03D8BDF90E10B4F91E5D63
:105E40006B480078002800F0B680013B012B02D996
:105E5000012A00F2C38004F60850FEF7F5FC94F81E
:105E60003C3D81464BB194F84C3C013B012B04D89E
:105E7000014604F5526000F01FFB19FB05F52DB239
:105E8000204604F5806900F0BEFC48B904F50060C6
:105E900000F0B9FC20B9484600F026FC05442DB2BC
:105EA000204600F0B0FC48B9484600F0ACFC28B9E8
:105EB00004F5006000F018FC05442DB2484600F0DF
:105EC000A2FC78B904F5006000F09DFC50B994F88C
:105ED0004C3CADB22046002B40F0828000F004FC28
:105EE00005442DB2294604F69C40FEF707FD014605
:105EF00004F54C60FEF702FD014604F6E440FEF7AF
:105F0000FDFC0546204600F07EFC70B9484600F0D6
:105F10007AFC50B904F5006000F075FC28B904F56E
:105F2000446000F029FD05442DB204F5496000F0FD
:105F300074FD014604F5426000F098FA284401B26D
:105F400004F55560FFF773FBF9E600F0D5F901465B
:105F50003DB928B93B780A2B7FF4F1AE2A464AE7CF
:105F60005EB13B780A2B04D000292A4618BF31467F
:105F700049E7002918BF3146F0E73146EEE704F55E
:105F8000806000F03EFC00287FF44CAF04F5006018
:105F900000F037FC00287FF445AF204600F031FCCC
:105FA00000287FF43FAF04F5496000F036FD00287B
:105FB0007FF438AFC3E6012A02D811FB05F55EE78E
:105FC00094F83C2D002A3FF4BAAE013B012B3FF67A
:105FD000B6AE04F5526000F06FFAB0E600254FE768
:105FE00000F0C4FB7CE705B0BDE8F08FA99A002063
:105FF000310700202DE9F04F994690F81A3D85B001
:1060000004460E4690460BB181F00106494604F65F
:10601000284A08EB4909634F2046FEF7BDFDC845F5
:1060200000F0BC8038F9021BB4F93E3D090291FB37
:10603000F3F194F81B3D09B2ADF80C101BB15046BA
:1060400000F008FC06460DF10E0104F5566000F064
:1060500069FD054608B194F83C5D94F8183D012BA4
:106060001BD093B1022BBDF90C1004F540607BD01E
:1060700000F042F90DB950B166B13B780A2B09D056
:1060800000282A4608BF01467FE01DB916B93B78B3
:106090000A2BC4D12A46314619E004F5546BBDF9E8
:1060A0000C1004F5406000F027F9BDF90C100190C8
:1060B0005846FFF7BCFA03A95846FFF70DFE019BAF
:1060C0003A7845B93BB90A2AA9D12A461946204649
:1060D000FFF7F4FD0AE00A2AF7D02A4619462046BF
:1060E000FFF7ECFD94F84C3C002B98D03B780A2B42
:1060F00095D194F8803D6BB194F83C3D53B1BDF916
:106100000C1004F60850FEF79FFB014604F55260A0
:1061100000F0D2F994F8813D002B80D0BDF80E300C
:1061200004F69C40B4F81E1D11FB03F109B2FEF702
:10613000E5FB014604F54C60FEF7E0FB014604F682
:10614000E440FEF7DBFB054604F5496000F065FC22
:10615000014604F5426000F089F9291804F55560FC
:1061600009B2FFF764FA5AE700F0C6F801463DB9F4
:1061700028B93B780A2B7FF452AF2A46A7E75EB1D5
:106180003B780A2B04D000292A4618BF3146A6E7DF
:10619000002918BF3146F0E73146EEE705B0BDE80B
:1061A000F08F00BFA99A002010B490F8194D1CB1CF
:1061B0005DF8044BFFF71EBF5DF8044BFFF7AABD67
:1061C0002DE9F0470446C0B0334800F0B3FEB4F800
:1061D0005A2DB4F8583D9BB2934247D194F85C3D98
:1061E0003BB3B4F8502D0A2823D9632A21D90238A9
:1061F00004AF002604F5556A85B2B946B046642D51
:1062000028BF642501360DF10E015046ADF80E8011
:10621000B6B2FFF761FDBDF80E30B54227F8023B7C
:10622000F0D1CDF800802B464A460A211A4801F0E9
:1062300077FA94F83C3DB3B104F55264204600F07F
:1062400097F94F280FD904AD00262F46013629466D
:106250002046033500F06CF9502EF7D1F022394674
:106260000E4804F009FE40B0BDE8F087B4F85A3D8E
:10627000B4F8582D9A4206D9B4F8582DB4F85A3DBE
:10628000D21A92B2AFE7B4F85A3DB4F8501DB4F840
:10629000582D0A44F4E700BF708A0020C0D90020BE
:1062A000002230B50024002502820277C0E90045B3
:1062B000C0E90222C0E9052230BD0000F0B500258A
:1062C0000024C0E900450B4D2601775D8F4209D1BE
:1062D0003544D5E9024554EA0501C0E9004505D138
:1062E0000420F0BD0134322CEED1F9E7C0E90223DD
:1062F0000020F6E700C501082DE9F743D0E905764F
:10630000D0E900254FEAE779044607FB05F301EBE6
:106310006101876102FB0933A7FB028999444FEAB7
:10632000D87343EA490303F31E03C6EB43035E1825
:10633000038A41F27071013346619BB28B42038242
:106340003DD190F81CE086FB0601C30F43EA4103F0
:1063500087FB070187FB06674FEAD07CF00F4CEA0A
:10636000410C40EA470000F31E00C7174543A0FB5D
:10637000020102FB075503F31E030CF31E0C294414
:106380006344C20F42EA410202F31E02A3EB42023F
:10639000A368BEF1000F00D0E3689A42B4BF0021A9
:1063A00001217145217706D000911BB212B2064936
:1063B000064805F0E6FE00232382C4E90533207F6A
:1063C00003B0BDE8F08300BF20C80108C0D9002099
:1063D0000023C0E905330377038270470022C0E938
:1063E000002270472DE9F0470023064614461E4D53
:1063F00015F833208A4205D115EBC30506D10420D8
:10640000BDE8F0870133322BF2D1F8E76B883068B2
:10641000B38008B111F036FD04EB440AB08804EBF8
:106420008A0A00244000274611F002FD3060B2883D
:10643000BBB29A4215D9204611F0E0FC32684FEA0F
:10644000E079A0FB0A010AFB0911C30F43EA4103EB
:10645000B9B2013703F30F0322F811306B681C4403
:10646000E5E70020CCE700BF40C80108C3885A1CFC
:1064700010B592B20468C28034F913308488944213
:106480009CBF0022C28009B15B421BB2184610BDFE
:1064900038B50025044601800581457345810573A3
:1064A00001EB410011F0C4FC04F1100360602046D0
:1064B00025612576636138BD037E01F50061F0B585
:1064C00043B1032B09D00133DBB2052B88BF002376
:1064D0000376F0BD09030161F5E702691143027B10
:1064E000016102F0FF0522B1012242730022026124
:1064F000E9E74269446892F800C0577896780289C3
:1065000002EB4202A11804F802C002894F70013266
:106510008E7092B2028102890188914200D8058171
:106520000189428992B28A42E0D101220273DDE7F9
:10653000034600895A8992B2824203D11A7B02F043
:10654000FF00A2B15A68588900EB4000024410884D
:10655000088092788A70002119735A89013292B2A8
:106560005A815A891888904200D859810120704771
:10657000428903899BB2934205D1027B02F0FF035B
:1065800082B100887047438902899A4204D90389FD
:106590004089181A80B270474289038900881844DC
:1065A000801AF7E7184670470023037670470023E8
:1065B000024600F2E93102F8013B02F8013B914248
:1065C000FBD1A0F8EA33C0F8EC33A0F8F033C0F800
:1065D000FC33C0E9FD3370472DE9F74F0446DFF87F
:1065E000048100200193A4F8EA03C5B24D5D002D9B
:1065F00043D04FF0000C0C275FFA8CF67E4308EB7B
:10660000060718F80660B6B3B5420CF1010CF2D1DA
:1066100097F808B04FF0000E4FF0004C5FFA8EF57F
:10662000AB4528D9B4F8EA530EF1010E2C4B05F016
:10663000070A04EBD50913F80AA07B6899F80160F2
:106640003CEA030340F2E2330CBF46EA0A0626EABC
:106650000A069D4289F8016007D900230425A4F8A1
:10666000EA33284603B0BDE8F08F01354FEA5C0CF1
:10667000A4F8EA53D2E70130B7E79DF83010019B48
:10668000A4F8FC139DF83410D4F8F403A4F8FE1316
:1066900045F6C051B1FBF2F2B1FBF3F3A4F8EE23DF
:1066A000A4F8F83308B111F0EDFBB4F8F80311F0D9
:1066B000BFFB00234FF0010CC4F8F4031F4698B24F
:1066C000B4F8F8638642CCD9D4F8F413B0EB560F83
:1066D00003F1010334BF01F800C00F54EFE700BF1E
:1066E000E0CB0108D0C9010830B503460078002886
:1066F00039D0B3F8EC231C4D03EBD20002F00704B1
:10670000B3F8FA1340782C5D204007D0D3F8F44357
:10671000B3F9FC03645C0CB9404200B20131B3F838
:10672000F84389B28C42A3F8FA13B3F8EE439CBF46
:106730000021A3F8FA13B3F8F013013189B28C42A7
:10674000A3F8F0130FD80132B3F8EA43002192B254
:10675000A3F8F0139442A3F8EC239EBF1970A3F89A
:10676000EC13A3F8FA1330BDE0CB010830B50346B3
:106770000078002839D0B3F8EC231C4D03EBD2008D
:1067800002F00704B3F8FA1340782C5D204007D0DC
:10679000D3F8F443B3F9FE03645C0CB9404200B291
:1067A0000131B3F8F84389B28C42A3F8FA13B3F875
:1067B000EE439CBF0021A3F8FA13B3F8F0130131A4
:1067C00089B28C42A3F8F0130FD80132B3F8EA4330
:1067D000002192B2A3F8F0139442A3F8EC239EBFD9
:1067E0001970A3F8EC13A3F8FA1330BDE0CB01083D
:1067F00000230370A0F8EC33A0F8F033A0F8FA33CC
:10680000704700787047B0F8EC3343B9B0F8F03314
:106810002BB9B0F8FA03003018BF012070470120EF
:10682000704708B50246FFF7EEFF38B90123A2F81A
:10683000EC03A2F8F0031370A2F8FA0308BD0022DB
:10684000C0E9002202818282C0E903227047C0E9C8
:10685000001270472DE9F743D0E90376394D04461D
:10686000028905FB07F3013207614FEAE379DB0F89
:1068700092B243EA490303F31E03C6EB43033C2AE7
:10688000028103EB8111C16052D181FB0189037D3B
:106890004FEAD87040EA490087FB078981FB076708
:1068A0004FEAD87200F31E0042EA490202F31E0CBE
:1068B000F20F604442EA470202F31E026A43D7170E
:1068C000D20F42EA470202F31E02A0EB4202002B63
:1068D00032D06068824206DA002106E0617D013133
:1068E000C9B2617502E0A17D0131A175617D0929FF
:1068F00016D9A17D09298CBF0021012121758BB1F9
:1069000091B9A175009103B212B20F490F4805F079
:1069100038FCA37D627D0E490C4805F0FBFB03E0CB
:106920000021EBE70029EDD100232381C4E90333E3
:10693000207D03B0BDE8F08320688242CEDB19469B
:10694000CFE700BF4DC5FB30E8CB0108C0D9002020
:1069500010CC01080023C0E903330375038170479D
:106960004FF48042028000228270426002727047BF
:1069700001EB8101018070470246807810B5E8B1D3
:10698000546842F6DF639C4219D9117A0D4B108886
:1069900033F8113013FB00F3DB1303F30F0318B2CA
:1069A0004B1CDBB23B2B88BF00231372013445F62E
:1069B000BF518C428ABF00235460536010BD002039
:1069C000F4E700BF2CCC010801238370002343604F
:1069D000037270470023837070470022C0E90022D1
:1069E000704718235A4345F6C05303FB0121016049
:1069F000704700681823B0FBF3F0704703680BB1D1
:106A000001234360704700234360704743681BB114
:106A100002680AB11944416070474068003018BFED
:106A200001207047036833B1406828B183422CBF0E
:106A30000020012070471846704738B500254FF4F4
:106A40006163044685820570C5828381057645763B
:106A5000C0E9015542F6302011F0EAF9231D20610A
:106A600020462577A36038BD002383820370C3824C
:106A7000436003764376037770470323B2FBF3F258
:106A800002EB42022DE9F0410A440124914227D051
:106A9000037E03F0FF0713B144760331F6E706697E
:106AA000838A91F8008003EB430391F801E091F8A9
:106AB00002C0F51806F80380838A85F801E00133E7
:106AC00085F802C09BB28382838A85899D4200D863
:106AD0008782858AC38A9BB2AB42DED10476DCE72B
:106AE000037F7BB9C28A838A9BB293420CD1027E18
:106AF00002F0FF0302B18389B3F5967F94BF0023B0
:106B000001230377BDE8F081C38A828A9A4204D9BF
:106B1000838AC28A9B1A9BB2EEE7C28A8189838AE2
:106B20000B44F7E70346007FF0B580B11A781AB13D
:106B3000032A35D000222AE09C8ADA8A92B2A24245
:106B400006D11C7E04F0FF0214B910461A77F0BD7E
:106B50001D69DA8A02EB4202AC18AF5C002266784B
:106B6000A5781A76DC8A0134A4B2DC82DC8AB3F818
:106B70000CC0A44500D8DA821C4644F8042F1F71CB
:106B80005E719D715A689C60120BA2F500620A80CA
:106B90001A780132D2B2052A88BF00221A70D6E7CD
:106BA0005A68C2F30B02F0E7C18A838A82899BB2DA
:106BB0008B4208D1037E002B0CBF1046002000EB57
:106BC000400080B27047C38A818A994208D9838A7B
:106BD000C08A1044C01A80B2824238BF0020EEE75B
:106BE000C38A808A181AF6E770B50446062500267F
:106BF00086F001062046013D314601F01FF831467E
:106C0000204601F02BF83146204601F02FF831469E
:106C1000204601F033F83146204601F037F831467E
:106C2000204601F03BF83146204601F03FF8FA21BA
:106C3000204601F079F815F0FF05D9D12946204604
:106C400001F014F82946204601F018F8294620469C
:106C500001F01CF82946204601F020F8294620467C
:106C600001F024F82046012101F000F82046FA2125
:106C700001F05AF82046012101F000F82046FA21DF
:106C800001F052F82046012101F000F82046FA21D7
:106C900001F04AF82046012101F000F82046FA21CF
:106CA00001F042F82046012101F000F82046FA21C7
:106CB00001F03AF82946204600F0F8FF2046FA2174
:106CC00001F032F82946204600F0E8FF2046FA217C
:106CD00001F02AF82946204600F0D8FF2046FA2184
:106CE00001F022F82946204600F0C8FF2046FA218C
:106CF00001F01AF829462046BDE8704000F0B6BF02
:106D00002DE9F74F00254FF416760446858105706E
:106D100004F1600AC5818680057445744FF41660DD
:106D200011F086F84FF4FA73A583A382A0604FF4A4
:106D3000FA60E58384F8215084F8205011F078F847
:106D4000A585A0614FF49660E585A68484F830504F
:106D500084F8315011F06CF81022A062294604F139
:106D6000340011F09DF904F1440304F1B002A4F8D9
:106D7000545001935346C4E91155C4E91355C4E96D
:106D8000165523F8025B9A42FBD104F1BC0904F5C5
:106D9000A4710023A4F8B0504A46C4E92D5522F846
:106DA000023B9142FBD104F5AA78A4F8483104F5DE
:106DB000F0714246C4E95333002322F8023B91426A
:106DC000FBD104F5F677A4F8E03104F50A713A46F0
:106DD000C4E97933002322F8023B9142FBD104F548
:106DE0000D76A4F8283204F521713246C4E98B33BC
:106DF000002322F8023B9142FBD104F52475A4F84C
:106E0000843204F547710022C4E9A2332B4623F8EB
:106E1000022B99424FF0000BF9D14FF4804384F8D4
:106E20003823C4F83C230021A4F81E334FF040233C
:106E3000A4F84423C4F83033C4F84823102284F85B
:106E40001CB384F84CB30198C4E9C833C4E9CA330D
:106E50004FF00823C4F834330123C4F8403311F051
:106E60001FF9012384F840B0502263630021019B85
:106E70005046A363294BE36311F012F90C23C4F8C5
:106E800058A08C22A4F854300021254B48464FF0DE
:106E90002A0AE36511F004F9C4F8B490DFF8909081
:106EA0008C22A4F8B0A00021C4F8B890404611F09C
:106EB000F7F8A4F848A13C2200213846C4E95389D8
:106EC00011F0EEF80623C4F8E4715022A4F8E03182
:106ED0000021144B3046C4F8E83111F0E1F80A23E0
:106EE0008C220021A4F8283228460F4BC4F82C62CB
:106EF000C4F8303211F0D4F80C4B2046A4F884A228
:106F0000C4F88C32C4F8885200F084FC2046FFF7A5
:106F10006BFE204603B0BDE8F08F00BFBC0600202A
:106F2000A2060020DA0500208E0600203A06002086
:106F3000E6050020C18B838B828A9BB28B4206D1EF
:106F400090F82030002B0CBF104600207047C38BF8
:106F5000818B994208D9838BC08B1044C01A80B2B0
:106F6000824238BF00207047C38B808B181AF6E727
:106F700038B5044C0D4622788A4201D000F06EFEEE
:106F8000257038BDA89A002080F841137047000092
:106F900070B5314D04460E462B788B4237D0013BFD
:106FA000092B09D8DFE803F00512161A1E2622085D
:106FB000082A002100F05AFE731E092B26D8DFE8AC
:106FC00003F021272C3136403B252545002100F0D8
:106FD00055FEF1E7002100F059FEEDE7002100F039
:106FE0005DFEE9E7002100F061FEE5E7002100F029
:106FF00065FEE1E7002100F073FEDDE7002100F00F
:1070000081FED9E70121204600F030FE2E7070BDD0
:107010000121204600F032FEF8E70121204600F071
:1070200035FEF3E70121204600F038FEEEE70121AE
:10703000204600F03BFEE9E70121204600F03EFE3D
:10704000E4E70121204600F04BFEDFE70121204666
:1070500000F058FEDAE700BFA99A002038B505789D
:1070600004464DB900F0FCFC01232946204623705C
:10707000BDE83840FFF78CBF38BD2DE9F0439DF8DF
:10708000409080F81C334FEAC9199DF820309DF8D4
:107090001C80A0F83093DB019DF844904FEAC8189B
:1070A000A0F820334FEAC9199DF824E09DF828C0C4
:1070B000A0F832934FEACE1EBDF94C904FEACC1C9B
:1070C0009DF82C7009F500699DF830609DF83450EA
:1070D000FF01A0F83493F601BDF94890ED019DF849
:1070E000384009F500699DF83C30E401A0F81E83A2
:1070F000DB01A0F836939DF85090A0F822E3A0F8A9
:1071000024C3A0F82673A0F82863A0F82A53A0F897
:107110002C43A0F82E3380F8389319B1C8F1000839
:10712000A0F81E83B2B1CEF1000ECCF1000C7F426C
:1071300076426D4264425B42A0F822E3A0F824C389
:10714000A0F82673A0F82863A0F82A53A0F82C43CF
:10715000A0F82E33BDE8F083B0F84233003318BFF7
:1071600001230B70B0F84433003318BF01231370B0
:107170000023A0F84233A0F84433704703460022AE
:1071800090F8210083F82120704703460022407CBC
:107190005A7470470023C0F848337047D0F848034A
:1071A000704790F84C037047428903899BB2934221
:1071B00005D1027B02F0FF0382B10088704743894A
:1071C00002899A4204D903894089181A80B270470B
:1071D0004289038900881844801AF7E718467047E7
:1071E000D0F83C33027801332DE9F04104468CB0ED
:1071F000C0F83C33002A00F05881D0F848234BF601
:107200007F339A420FD9B14B1B785A1E042A40F2A1
:107210003F81063B012B03D800212046FFF7B8FE33
:107220000023C4F84833D4F83C2345F6BF539A42B0
:107230000BD994F840130023204681F00101C4F8D3
:107240003C3384F8401300F0F9FC94F8383323B150
:10725000204600F0E7FC84F84C0304F11400FFF72B
:10726000A3FF60B99A4B1A784AB11870204694F877
:107270001C1300F0EBFC9749974803F037FF201DE3
:10728000FFF792FF012840F21D8104AD0DF10C0CB7
:1072900000220DF1140E2E466746114640F6FF7887
:1072A000A089E3899BB2834201D1237C7BB1A3688F
:1072B000E08903EB800318682174E3890A900133A5
:1072C0009BB2E381E389A088984200D8E1819DF8D0
:1072D0002A30A08D0CF8013BE38D9BB2834202D192
:1072E00094F830308BB1A06AE38D9BB230F8133044
:1072F00084F830102EF81230E38D01339BB2E38511
:10730000E38DA08C984200D8E18594F8413363B1B5
:10731000BDF828309BB21BB1BDF82830984504D188
:10732000B4F842330133A4F84233BDF82830B4F83E
:107330003403181AB4F81E3313FB00F3DB1303F302
:107340000F0325F8023B002A00F0EE8094F84C333E
:10735000002B40F0B780022208A930460FF054FEFF
:1073600002230AAA08A904F1340010F03DFCDDE96B
:107370000A321344BDF8102003EBD3735B1403F3FC
:107380000F039BB2D21AADF81820BDF81220D31A01
:10739000ADF81A304D4B1D78002D40F0CE804F4B8C
:1073A0001B7863B1022307AA06A904F1540010F068
:1073B00049F8022305AA07A94948FCF7F9FE494BF9
:1073C0001B7863B1022307AA06A904F5F07010F038
:1073D00039F8022305AA07A9434802F0FFFC434BF2
:1073E0001B7863B1022307AA06A904F50A7010F0FE
:1073F00029F8022305AA07A93D4801F053FE3D4B99
:107400001B7883B1022307AA314604F1B00010F0C3
:1074100019F8394B1B78002B00F08880022207A94D
:107420003648FBF735F9364B1B7863B1022307AAC0
:1074300006A904F5A47010F005F8022305AA07A90F
:10744000304805F0F5FC304B1B7863B1022307AAE6
:1074500006A904F521700FF0F5FF022305AA07A97C
:107460002A4800F0E9FF2A4B1B7843B1204600F080
:10747000D9FB0223014606AA2648FEF795FE264BB5
:107480001B78FBB1022206A92448F9F765FA19E036
:10749000022B7FF4C1AE0E4B1B78002B3FF4BCAE29
:1074A00000211F48FBF734FEB6E61E498B4209D97E
:1074B00090F84013C0F83C2381F0010180F840139C
:1074C00000F0BCFB0CB0BDE8F08100BFA99A002021
:1074D000AA9A0020AACC0108C0D9002030070020B9
:1074E0007059002035070020BCAF00203407002071
:1074F000AC9A00202F070020310700208C36002096
:1075000037070020F0DB002033070020C08D00206B
:1075100032070020E87C00202E070020680A0020A7
:10752000845800207FA903000122B9E6022305AA9E
:1075300007A95748FAF7A8FD75E7012D11D1554B5A
:107540001B78002BBED007AA06A904F15400022321
:107550000FF078FF022305AA07A94F48FCF728FE81
:10756000B0E7022D25D14D4B1B78002BAAD02B461E
:1075700007AA314604F1B0000FF064FF484B1B78B6
:1075800083B1484B1B783BB100953B4605AA07A940
:107590004548FBF79BF895E72A4607A94348FBF7C0
:1075A00077F88FE72B4605AA07A93948FAF76CFD4B
:1075B00088E7032D11D13E4B1B78002B82D007AA00
:1075C00006A904F5A47002230FF03CFF022305AACC
:1075D00007A9384805F02CFC74E7042D12D1364B6E
:1075E0001B78002B3FF46EAF07AA06A904F5F070D4
:1075F00002230FF027FF022305AA07A92F4802F054
:10760000EDFB5FE7052D12D12D4B1B78002B3FF4CE
:1076100059AF07AA06A904F50A7002230FF012FF5A
:10762000022305AA07A9274801F03CFD4AE7072DD8
:1076300012D1254B1B78002B3FF444AF07AA06A9B3
:1076400004F5217002230FF0FDFE022305AA07A90D
:107650001E4800F0F1FE35E70A2D3FF407AF632D19
:107660000CD107AA314604F1540002230FF0EAFEC0
:10767000022207A91648F9F7A9FD23E7602D7FF438
:1076800021AF022205A91348FAF76CF81AE700BFE8
:10769000DC1A002030070020705900202F0700203E
:1076A00031070020AA9A0020DC3B00208C36002005
:1076B00037070020F0DB002035070020BCAF00209A
:1076C00034070020AC9A002033070020C08D002032
:1076D00084160020E0160020037B13B503F0FF02A0
:1076E000019123B101234373002002B010BD44680F
:1076F00003899BB244F82310038901339BB20381B1
:1077000003890188994200D80281028943899BB28A
:1077100093424FF0010300D103731846E5E70000E0
:107720002DE9F3479846037804460E4617460A9D0E
:10773000002B66D090F84C33002B62D1324B1A7874
:1077400052B9012290F81C1351401A7000F07EFAD1
:107750002E492F4803F0CAFC711E0A2946D8DFE8DB
:1077600001F0062D3033363C3945453F4200B4F92F
:1077700022934FF0000A04F11406D04541D037F8A7
:107780001A30B4F8362313FB09F3DB1303F30F03AA
:1077900013449BB2B3F5805F22BFB4F84423013297
:1077A000A4F844232DBBADF800308DF802500099A9
:1077B00030460AF1010AFFF78FFFDEE7B4F92493A0
:1077C000D7E7B4F92693D4E7B4F92893D1E7B4F90D
:1077D0002A93CEE7B4F92C93CBE7B4F92E93C8E7FC
:1077E000B4F93093C5E7B4F93293C2E7B4F9209302
:1077F000BFE7ADF8043015F80A308DF8063001996E
:10780000D6E702B0BDE8F087AA9A0020A4CC010810
:10781000C0D900202DE9F7430225684607F07EFB1A
:107820004FF400733E4E284601210124ADF8063086
:107830004FF020098DF8055009F0ECFC4FF400538F
:10784000694630468DF80440009307F0C7FA214698
:10785000284609F0DFFC4FF4804369463046314F3B
:107860004FF4806800938DF8044007F0B7FA214682
:10787000204609F0CFFC69463846CDF800908DF8D7
:10788000044007F0ABFA2146284609F0C3FC4FF448
:10789000004369463046009300238DF8043007F01A
:1078A0009DFA2146284609F0B5FC69463046CDF8D8
:1078B00000808DF8044007F091FA2146284609F02F
:1078C000A9FC10236946304600938DF8044007F068
:1078D00085FA2146284609F09DFC69463046CDF8D8
:1078E00000908DF8044007F079FA2146284609F007
:1078F00091FC08236946304600938DF8044007F058
:107900006DFA2146204609F085FC69463846CDF8D7
:1079100000808DF8044007F061FA03B0BDE8F08301
:1079200000040240000002404FF4006337B5ADF898
:107930000030002304468DF80230828BC38B9BB24B
:10794000934202D190F820308BB1A369E28B03EB14
:1079500082030022186884F82020E38B0090013312
:107960009BB2E383E38BA18A994200D8E283BDF8FE
:107970000010002006F0E0FC02212D4806F034FB48
:1079800000BBADF8000002210546294806F05AFB6D
:10799000274805F0ADFF009A237C019203F0FF0118
:1079A000CBB10123637494F8303003F0FF0243B38A
:1079B000012384F83130D4F848330133C4F8483314
:1079C00003B030BD1A4806F06FF8ADF80000194852
:1079D00006F06AF8D7E7A068A3899BB240F8232095
:1079E000A38901339BB2A381A389A2889A4200D8BC
:1079F000A181A289E3899BB29342D4D1012323744C
:107A0000D1E7A16AA38D9BB221F81350A38D013356
:107A10009BB2A385A38DA18C994200D8A285A28D8B
:107A2000E38D9BB29342C6D1012384F83030C2E784
:107A3000002001400021014008B501214FF08040A5
:107A40000CF0CAFE48B14FF0804001210CF022FF3B
:107A50000248BDE80840FFF767BF08BD708A0020F4
:107A6000F0B5022197B0694806F0BEFA10B1684837
:107A7000FFF75AFF01A8012507F050FA03A805F007
:107A8000D9FD10A805F088FD012100240326084631
:107A9000022709F0BFFB01214FF4807009F044FC7C
:107AA00001A95C4801958DF808608DF80B4007F03E
:107AB00095F92946284609F0ADFB29464FF4007098
:107AC00009F032FC01A9534801978DF808608DF840
:107AD0000B4007F083F9062303A8CDE90334CDE971
:107AE000054405F063FD10A948481094ADF84440E2
:107AF00014948DF85450CDE9124405F0CDFC29467C
:107B0000424805F02BFF23462A4621463F4805F010
:107B100077FE29463D4805F093FD10A93E4805F043
:107B2000BBFC29463C4805F019FF2A462346294656
:107B3000394805F065FE2946374805F081FD01A862
:107B400007F0ECF907A806F069FB2946284609F07A
:107B500061FB29464FF0005009F0C4FB102301A936
:107B60002C4801938DF808608DF80B4007F036F92A
:107B700007A920460A94CDE9074406F0FFFA2946F2
:107B8000204606F051FB2946284609F0ABFB2A4661
:107B90000F21204807F0C8FC4FF4004301A91D48FD
:107BA00001938DF8087007F019F90BA80AF0DCF8BA
:107BB000F9230BA94FF080400B93CDE90C45CDE99B
:107BC0000E440AF03DF82346224621464FF08040FD
:107BD0000DF014FA29464FF080400AF051FC2A4675
:107BE00029464FF080400CF097FC0C4B6846009300
:107BF00005F0A0FB4FF48041094807F06BFB202102
:107C0000044807F027FB17B0F0BD00BF002001407B
:107C1000708A002000000240002101401C00010188
:107C20000004024008B54FF40041034807F0C8F9CA
:107C3000431E5842584108BD000402400A4602480B
:107C4000202107F087BB00BF000002400A4602481F
:107C50004FF4005107F07EBB000402400A46024880
:107C60004FF4804107F076BB000402400A46024808
:107C70004FF4806107F06EBB000402400A460248E0
:107C8000102107F067BB00BF000402400A4602480B
:107C9000202107F05FBB00BF000402400A460248F3
:107CA000082107F057BB00BF000402400A46024803
:107CB0004FF4806107F04EBB0000024038B5074C1E
:107CC0000D460A464FF48061204607F043FB2A46E2
:107CD00020460821BDE8384007F03CBB00040240C4
:107CE00038B5074C0D460A464FF48061204607F030
:107CF00031FB2A4620461021BDE8384007F02ABB58
:107D00000004024038B5074C0D460A464FF4806126
:107D1000204607F01FFB2A4620462021BDE83840B8
:107D200007F018BB00040240064B1A684FF47A7340
:107D3000B2FBF3F221B11346013BFDD10139F9E762
:107D4000704700BF100900200220704708460C222F
:107D5000014910F00BB900BF20F4F01F0023821D71
:107D600000F286710360838022F8023B8A42FBD1D5
:107D7000154A00F2BC71A0F88637C0F88827134A6C
:107D8000C0F89437C0F88C27C0F890270022C0F8BC
:107D9000983700F29C7323F8022B8B42FBD1A0F89A
:107DA000BC2700F2DE7100F2BE72002322F8023B13
:107DB0009142FBD16322A0F8DE37C0F8E43780F8A7
:107DC000E027A0F8E837704700000F270F270F279C
:107DD0006322002380F8E0270B4A0370C0F888274D
:107DE0000A4AA0F8BC37A0F8DE37A0F88637C0F8FA
:107DF0008C27C0F89027C0F89437C0F89837C0F89F
:107E0000E437A0F8E837704700000F270F270F2747
:107E1000F7B54FF47A53374E04464FF0000C1F4627
:107E200030461FFA8CF5AA421ED904EB4105B5F97C
:107E30000650002D11DDA842B8BF2846AF42A8BFAA
:107E40002F464D1D0CF1010CADB2B5F5707F24BF6E
:107E5000A1F2BB318DB22946E3E7AB42A8BF2B4666
:107E6000AE42B8BF2E46ECE7C21933442249521045
:107E700022485B10D5181BB26D102EB2551B12B2E2
:107E80002DB2CDE9006504F0C3F994F8E03704F2AF
:107E90009C7104F2BC70632B1FD10B4623F8026B5C
:107EA00098421D84FAD1002384F8E03700231A4653
:107EB000A4F8BC37A4F8DE3731F9025B2A440D8CF4
:107EC00088422B4412B21BB2F6D112111B11A4F836
:107ED000BC27A4F8DE3703B0F0BD04EB4302013346
:107EE000DBB2A2F89C67A2F8BE570F2B84F8E037EC
:107EF000D9D8DBE780C1FFFF83CD0108C0D90020BE
:107F00002DE9F04F85B04FF00009DFF8B0B0BDF9B2
:107F10003C40BDF940A00294BDF83850CAF10004BD
:107F2000019203941FFA89F4019A944243D200EB20
:107F3000410405F1010C039A4FEAE508E6881FFAAF
:107F40008CFC029C05F00707023513F808E0361B8D
:107F50004FEAEC040CF0070C1BF8077036B21BF864
:107F60000CC0ADB2964207DA2EEA070703F8087094
:107F70001E5D4CEA060C08E0002E14DA2EEA070714
:107F800003F808701E5D26EA0C0C03F804C04C1DB3
:107F900009F10109A4B2B4F5707F24BFA1F2BB318D
:107FA0008CB22146BEE74EEA0707564503F8087033
:107FB0001E5DDEDAE7E705B0BDE8F08FB1CC010861
:107FC0002DE9F0479846B0F88637044686B003445A
:107FD00015465878484004F0A5FB9DF83830984283
:107FE00000F29180B4F8883705F1FF3CEA1D47485C
:107FF00003F29D3700254FF6FD7E4FF00309BFB217
:10800000B7F5707F28BFA3F123074FF47A5328BF39
:10801000BFB2394604EB41061CF901AFB6F9066060
:10802000B042B8BF3046B342A8BF3346BAF1010FE1
:1080300064D0BAF1030F04D0BAF1FF3F60D13544E8
:1080400001E016FB0E554E1DB6B2B6F5707F2ABF85
:10805000A1F2BB31314689B29445DBD1D4F89427E3
:10806000AA4250DA94F8E027632A0AD103445B104D
:10807000A4F8BC37C31A44F63E104343DB13A4F8FC
:10808000DE37B4F9DE37002608223946029320464F
:10809000B4F9BC370096019305ABFFF731FF98F8B0
:1080A00000309DF81400584004F03CFB98F8013073
:1080B00081469DF81500584004F034FB48449DF873
:1080C0003C30C0B283421ED304230120C4F894572D
:1080D000A4F89837B4F88837A4F88A7703F297326F
:1080E000A4F88E3792B2B2F5707F2ABF293BA4F86C
:1080F0008C27A4F88C3706B0BDE8F087AD1BA2E74B
:1081000016FB09559FE70020F5E700BF80C1FFFF80
:1081100073B5002504462C4BF2212C4ACDE90055BD
:10812000FFF74EFF06462A4B0D212A4A2046CDE98D
:108130000055FFF745FF054606B9E0B194F89A37B8
:10814000CBB9C4F8E4370121A4F8E8372248FEF798
:108150000FFF01212048FEF717FF632384F8E03763
:10816000052384F89A3716B1012384F89B3715B19B
:10817000022384F89B3794F89A3713B3013BDBB2A0
:10818000012B84F89A371CD1B4F88E3703F2BF3232
:1081900092B2B2F5707F28BF03F1FF32A4F89027A6
:1081A0005A1C92B2B2F5707F2ABFA3F2BF33A4F873
:1081B0009227A4F8923794F89B3723700023A4F8F1
:1081C0009A3702B070BD00BFBDCC0108CFCC01080A
:1081D000BBCC0108C7CC0108708A002010B504464A
:1081E000B0F8E80798B1D4F8E4373322B3FBF0F3E2
:1081F000C3F3072081F8323081F83100054802F0DE
:10820000A3FD0023C4F8E437A4F8E83710BD3122F9
:10821000F4E700BFC0D9002010B50446B0F8E80765
:1082200098B1D4F8E4373322B3FBF0F3C3F307205B
:1082300081F8323081F83100054802F0B3FD0023A7
:10824000C4F8E437A4F8E83710BD3122F4E700BFE2
:10825000C0D90020F0B5B0F8901793B0B0F89227CD
:108260000446B0F88837914280F0A080994239D80E
:108270009A4237D301260225654B0D21654ACDE987
:108280000065FFF79DFE0746634BFD21634A2046CC
:10829000CDE90065FFF794FE07B1257010B3B4F97E
:1082A000DE37B4F98E2700935D49B4F9BC375D48D9
:1082B00003F067FF00215C48FEF75AFE00215A4890
:1082C000FEF762FE574802F09BFD42F20F72002358
:1082D000A4F88C276322237084F8E027A4F89A3747
:1082E000C4F89437B4F88827B4F88C379A425BD135
:1082F000B4F89837042B16D1B4F88E3703F2BF3296
:1083000092B2B2F5707F28BF03F1FF32A4F8902734
:108310005A1C92B2B2F5707F2ABFA3F2BF33A4F801
:108320009227A4F89237C022B4F88A172046FFF7A4
:108330006FFD2178B4F9BC370129B4F9DE2742D0AA
:10834000022948D0B4F9DE37C022B4F88A17204693
:108350000293B4F9BC3701930823009305ABFFF7F0
:10836000CFFDB4F89857013DADB2A4F89857002D51
:1083700036D12E492B4802F0B9FE29462A48FEF78D
:10838000F7FD29462848FEF7FFFD264802F056FD76
:1083900042F20F732570A4F88C376323A4F89A5720
:1083A00084F8E037C4F8945713B0F0BD994201D96E
:1083B0009A4297D301260225154B0D21154A2046D6
:1083C000CDE900655DE700921949B4F98E2715489B
:1083D00003F0D7FEB6E700921649B4F98E27F6E708
:1083E000EB1E5D425D412378012B8DF8145007D0C0
:1083F000022B09D00023C4F8943784F89B37D3E7C5
:1084000005A9FFF7EBFEF5E705A9FFF705FFF1E783
:10841000BBCC0108C7CC0108B9CC0108BFCC01080E
:10842000D7CC0108C0D90020708A002062CD010895
:1084300002CD010834CD01082DE9F04104460D4676
:10844000971E01EB43080026454540D037F8022F20
:108450002046D4F8E43735F9021B1344B4F88627D4
:108460000029C4F8E4372244B4F8E83703F10103E3
:10847000A4F8E83753784FEA4303DBB2B8BF43F0C0
:1084800001035370B4F8883704EB4303D980237891
:10849000013B012B18D8FFF7DDFEB4F88837013314
:1084A0009BB2B3F5707F38BFA4F88837B4F886372D
:1084B00028BFA4F8886701339BB2042B94BFA4F8AB
:1084C0008637A4F88667BFE7FFF722FEE5E7BDE839
:1084D000F081000070B5044600254FF47A6004F185
:1084E0001C06258120806581657325730FF0A0FC33
:1084F00004F13C0332466060A561C4E9045522F8EA
:10850000025B9342FBD104F2EC41002203F8012B01
:108510009942FBD1F023C4F8EC24C4F8F8240021DC
:10852000A4F8F0344FF4965320223046C4F8F434C3
:108530000FF0B6FD05232046237409236382024B06
:10854000C4E9053670BD00BFD4060020F0B58FB079
:108550000A4600234FF4F77502A940F2C9564FF6B8
:1085600037274FF6126C02F0C004802C1DD0C02CAF
:1085700018D0002C0CBF64463C4621F81340013350
:108580009200042BD2B2EED104AA10300EF078FD86
:10859000002304AA0721009314230548FFF7C0F81D
:1085A0000FB0F0BD21F81360E9E721F81350E6E7BA
:1085B000708A002010B58EB000240423103004AA65
:1085C00002A9CDE902440EF05BFD142304AA0721A1
:1085D00002480094FFF7A4F80EB010BD708A002086
:1085E00070B5B0F8EC3404461BB34948FEF7A2FC62
:1085F000484E0546142D1BD9B4F8EE342046143DE0
:108600005A1C2344ADB2A4F8EE2493F83C10FFF7B3
:108610009DFF33781BB1D4F8F434C4F8F834B4F8BF
:10862000EE24B4F8EC349A42E4D30023C4F8EC34DA
:1086300070BD428903899BB293422DD1037BA3B1C4
:10864000038893B1344B1B78002B3BD1B4F8F05422
:10865000772198B2B4F8EC24A8422BD30023A4F8D5
:10866000EE34B4F8EC34002BBFD1D4F8F834002B3E
:10867000DED02748FEF75EFC0546142DD8D92046EB
:10868000143DFFF797FFD4F8F834ADB2013BC4F8BE
:10869000F834002BF1D1CBE7438902899A4204D9FF
:1086A000038942899B1A9BB2CBE7428901880389DF
:1086B0000B44F7E7501C22440133A4F8EC0482F881
:1086C0003C10C6E7302300202189628992B28A4299
:1086D00003D1227B02F0FF016AB16168628992B224
:1086E000895C20736289013292B262816289258835
:1086F000954200D86081B4F8EC24013B551C13F07E
:10870000FF032244A4F8EC5482F83C10DCD1A5E726
:10871000708A002031070020AA9A002001EB410155
:10872000890001F51671B1F5966F8ABF4FF4966313
:10873000A0F8F014A0F8F03470474FF49663594352
:10874000C0F8F414704708B5F9F7B7FD3023B0FB53
:10875000F3F0C0B208BD312AF8B504460D4624D165
:10876000F9F7ABFD2F2822D901231946227B02F00D
:10877000FF002AB161730133312BF7D10020F8BD1E
:1087800066682289EF5C92B2B7542289013292B2B4
:10879000228122892688964200D8208120896289F8
:1087A00092B28242E7D12173E5E70420E7E7052092
:1087B000E5E70000014802F0C1B800BFC0D90020C1
:1087C00010B5504803F0B6FB4F48FEF709FD4F4B7C
:1087D0004F4C1B782BB12378012B02D14D48FBF76E
:1087E000C3FE4D4B1B784BB12378022B06D14B4B6C
:1087F0001B78002B7BD04A48FAF7D8FE494B1B78F0
:108800002BB12378032B02D1474804F0F5FB474BEB
:108810001B782BB12378042B02D1454801F0FAFBD9
:10882000444B1B782BB12378052B02D1424800F032
:1088300033FD424B1B782BB12378072B02D14048E4
:10884000FFF7CEFE3F4B1B782BB12378062B52D17E
:108850003D4801F055FD3D4B1B7833B123780BB1FA
:108860000A2B02D13A48F8F7A5F93A4B1B782BB1FD
:1088700023780A2B02D13848FDF7A2FC2378632B1A
:1088800002D13648F8F7D6FC23785C3BDBB2062BE6
:1088900007D84D2222FA03F3DB0702D53048F8F758
:1088A000C1FB2378663B052B02D82E48F8F7F0FD74
:1088B00023785D2B02D12C48F8F7F0FE23785B2B50
:1088C00002D12A48F8F7ACFE23786C2B02D1284855
:1088D000F8F77EFE2378652B02D12648F8F71CFFB7
:1088E000237873B92448BDE81040F8F785BF2348C2
:1088F000F9F750FC82E7144801F0F6FC0028A7D1F4
:10890000A9E710BDC0D90020708A002030070020E0
:10891000A99A0020407A00202F070020310700206C
:10892000845800203707002030EF00203507002052
:1089300000D200203407002028AA0020330700209E
:10894000AC9500203607002080D700202E0700209D
:10895000F413002032070020E87C0020C416002019
:1089600058160020C8160020DC160020D91600205A
:10897000D8160020DE160020EC16002098310020CA
:1089800008B5FFF717FFFFF71BFFFCE708B52F48F7
:10899000FAF75EFE2E48FBF769FC2E48F8F786FBD7
:1089A0002D48F8F742FC2D48F9F7DAFC2C48F9F786
:1089B00080FE2C48FAF7E6FA2B48F8F7E3FF2B483D
:1089C000F9F77EFB2A48F8F725FA2A4803F0F6FE65
:1089D000294804F077FA294800F05CFD284801F0A6
:1089E00055FA2848F8F756FE274800F06DF8274852
:1089F00000F0A6FB2648F8F70EFE2648FFF7AEF972
:108A00002548FFF767FD2548F8F7DFFD244801F00A
:108A1000F3FB2448F8F77CFE2348FCF739FE234893
:108A2000F8F72EFD2248F7F707FF2248F8F783F8FA
:108A30002148F8F790FE2148F8F7CEFE204801F0D3
:108A400031FD2048BDE80840FEF75AB970590020B2
:108A5000407A002084160020C41600208C360020A6
:108A6000DC3B002084580020DC1A002098310020D4
:108A700058160020F0DB002030EF0020BCAF0020B3
:108A800000D20020DC160020AC9A002028AA00208A
:108A9000D9160020C08D0020AC950020D8160020EB
:108AA00080D70020DE160020E87C0020C8160020B9
:108AB000680A0020F4130020E0160020EC160020C5
:108AC000C0D90020708A00200021024600F1160360
:108AD00002F8021B22F8021B9342FBD100F616712A
:108AE000002223F8022B9942FBD1184B00F64C715F
:108AF000A0F8162FC0F8183F154BC0F8242FC0F867
:108B00001C3FC0F8203F4FF00003A0F8282F0022A0
:108B100080F82A3F00F62C7323F8022B9942FBD1F0
:108B2000A0F84C2F00F66E7100F64E72002322F86A
:108B3000023B9142FBD16322A0F86E3FC0F8743F24
:108B400080F8702FA0F8783F704700BF00000F2713
:108B50000F270F276322002380F8702F0C4A037021
:108B6000C0F8182F0B4AA0F84C3FA0F86E3FA0F8B1
:108B7000163FC0F81C2FC0F8202FC0F8243FA0F8E3
:108B8000283F80F82A3FC0F8743FA0F8783F70472C
:108B900000000F270F270F27F7B54FF47A53384EF1
:108BA00004464FF0000C1F4630461FFA8CF5AA42CF
:108BB0001FD904EB4105B5F91650002D12DDA8426E
:108BC000B8BF2846AF42A8BF2F4601F10A050CF1F5
:108BD000010CADB2B5F5F06F24BFA1F276718DB284
:108BE0002946E2E7AB42A8BF2B46AE42B8BF2E46AD
:108BF000EBE7C21933442349521023485B10D518C0
:108C00001BB26D102EB2551B12B22DB2CDE900650C
:108C100003F0FEFA94F8703F04F62C7104F64C70E1
:108C2000632B1FD10B4623F8026B98421D84FAD1A7
:108C3000002384F8703F00231A46A4F84C3FA4F8A0
:108C40006E3F31F9025B2A440D8C88422B4412B2EC
:108C50001BB2F6D112111B11A4F84C2FA4F86E3FD1
:108C600003B0F0BD04EB43020133DBB2A2F82C6F7A
:108C7000A2F84E5F0F2B84F8703FD9D8DBE700BF16
:108C800080C1FFFFFFCD0108C0D900202DE9F04FC2
:108C900085B04FF00009DFF8B4B0BDF93C40BDF934
:108CA00040A00294BDF83850CAF100040192039428
:108CB0001FFA89F4019A944244D200EB410405F171
:108CC000010C039A4FEAE508E68A1FFA8CFC029C25
:108CD00005F00707023513F808E0361B4FEAEC04ED
:108CE0000CF0070C1BF8077036B21BF80CC0ADB2C5
:108CF000964207DA2EEA070703F808701E5D4CEA71
:108D0000060C08E0002E15DA2EEA070703F80870B3
:108D10001E5D26EA0C0C03F804C001F10A0409F1F7
:108D20000109A4B2B4F5F06F24BFA1F276718CB240
:108D30002146BDE74EEA0707564503F808701E5D59
:108D4000DDDAE6E705B0BDE8F08F00BFA3CD01088E
:108D5000B0F8163F00EB43032DE9F047044658886E
:108D600086B0C0F3090080F4A67080F0010003F023
:108D7000E9FC022800F2A280B4F8183F0A20DFF8CC
:108D800044E1002603F226774D494FF6FD784FF077
:108D90000309BFB2B7F5F06F28BFA3F15A074FF42C
:108DA0007A5328BFBFB23A4604EB42051EF901CB05
:108DB000B5F91650A942B8BF2946AB42A8BF2B4609
:108DC000BCF1010F75D0BCF1030F04D0BCF1FF3F23
:108DD00071D12E4401E015FB086602F10A05013845
:108DE000ADB2B5F5F06F2ABFA2F276722A4692B202
:108DF00010F0FF00D8D1D4F8242FB24256DA94F8FC
:108E0000702F632A0AD10B445B10A4F84C3FCB1A95
:108E100044F63E114B43DB13A4F86E3FB4F96E3FAA
:108E200000250A22394602932046B4F94C3F0095AA
:108E3000019305ABFFF72AFF23789DF81400AB429E
:108E400080F0CD000CBF4FF0010A4FF0030A03F091
:108E500069FC80469DF8150080F0F50003F062FC87
:108E600081469DF8160020F00F0080F0900003F07E
:108E700059FC484480445FFA88F8D0451ED8062340
:108E80000120C4F8246FA4F8283FB4F8183FA4F8D0
:108E90001A7F03F21B72A4F81E3F92B2B2F5F06F74
:108EA0002ABF653BA4F81C2FA4F81C3F06B0BDE800
:108EB000F087761B91E715FB09668EE70020F5E742
:108EC00080C1FFFFABCD010810B50446FFF740FF9E
:108ED000A0B194F82A3F8BB9C4F8743F0121A4F8DB
:108EE000783F1948FEF744F801211748FEF74CF87F
:108EF000632384F8703F052384F82A3F94F82A3FBF
:108F00000BB3013BDBB2012B84F82A3F1BD1B4F831
:108F10001E3F03F27F7292B2B2F5F06F28BF03F1E9
:108F2000FF32A4F8202F5A1C92B2B2F5F06F2ABF7C
:108F3000A3F27F73A4F8222FA4F8223F0123237009
:108F4000002384F82A3F10BD708A002010B5044623
:108F5000B0F8780F98B1D4F8743F3322B3FBF0F334
:108F6000C3F3072081F8323081F83100054801F061
:108F70009FFE0023C4F8743FA4F8783F10BD31224F
:108F8000F4E700BFC0D90020B0F8201FB0F8222FAE
:108F9000B0F8183F914230B5044693B06BD2994275
:108FA00004D89A4202D32046FFF7D2FEB4F8182F15
:108FB000B4F81C3F9A425CD1B4F8283F062B16D176
:108FC000B4F81E3F03F27F7292B2B2F5F06F28BF81
:108FD00003F1FF32A4F8202F5A1C92B2B2F5F06FC1
:108FE0002ABFA3F27F73A4F8222FA4F8223FC02245
:108FF000B4F81A1F2046FFF7CFFDB4F96E3FB4F95D
:109000001E2F00932349B4F94C3F234803F0B9F8CD
:10901000B4F96E3FC022B4F81A1F02932046B4F987
:109020004C3F01930823009305ABFFF72FFEB4F8E4
:10903000285F013DADB2A4F8285FFDB91749164875
:1090400002F054F829461648FDF792FF29461448C5
:10905000FDF79AFF104801F059FE42F20F73257098
:10906000A4F81C3F632384F82A5F84F8703FC4F897
:10907000245F13B030BD994293D894E76B1F05A9C4
:109080005D425D418DF81450FFF760FF0023C4F886
:10909000243FEEE7B5CD0108C0D90020DDCD0108A1
:1090A000708A00202DE9F04104460D46971E01EB21
:1090B00043080026454540D037F8022F2046D4F813
:1090C000743F35F9021B1344B4F8162F0029C4F875
:1090D000743F04EB4202B4F8783F03F10103A4F8B3
:1090E000783F53884FEA43039BB2B8BF43F0010374
:1090F0005380B4F8183F04EB4303D9822378012B43
:1091000018D1FFF741FFB4F8183F01339BB2B3F514
:10911000F06F38BFA4F8183FB4F8163F28BFA4F882
:10912000186F01339BB2092B94BFA4F8163FA4F823
:10913000166FBFE7FFF7C8FEE5E7BDE8F081000066
:10914000F8B5044600254FF47A6004F1280725811C
:10915000208004F148066581657325730EF068FE72
:109160003B466060A561A583C4E90455C4E9085580
:1091700023F8025B9E42FBD104F1D4033246002166
:1091800022F8021B9342FBD104F28451002203F81F
:10919000012B9942FBD1F023C4F88425C4F8902513
:1091A0000021A4F8883540F6B83320223846C4F8A8
:1091B0008C350EF075FF8C22002130460EF070FFCA
:1091C0000A2326622046237409236382034BC4E9E1
:1091D00005371623A383024B6362F8BD38070020CE
:1091E000EC070020F0B5ADB00A460446002302A902
:1091F000F52540F2DF264FF621574FF60B7C02F0A3
:10920000C000802825D0C02820D000280CBF604690
:10921000384621F8130001339200042BD2B2EED16C
:1092200004AA04F110000DF02BFF18AA04A904F100
:109230001C0028230EF006F9002318AA052100932C
:1092400028230548FEF76CFA2DB0F0BD21F8136015
:10925000E1E721F81350DEE7708A002030B5ADB0A9
:1092600005460024042304AA02A91030CDE90244D3
:109270000DF006FF18AA04A905F11C0028230EF022
:10928000E1F8282318AA052102480094FEF748FABD
:109290002DB030BD708A002070B5B0F8843504461A
:1092A0001BB35348FDF746FE524E0546282D1BD9E9
:1092B000B4F886352046283D5A1C2344ADB2A4F8A4
:1092C000862593F8D410FFF78DFF33781BB1D4F8BF
:1092D0008C35C4F89035B4F88625B4F884359A42B4
:1092E000E4D30023C4F8843570BD428903899BB25E
:1092F00093421BD1037B002B3DD00388002B3AD037
:109300003D4B197800294DD1B4F888655F25B4F834
:10931000843588B25A1C864204EB030092B213D9FA
:10932000A4F88425013180F8D450F0E743890289FC
:109330009A4204D9038942899B1A9BB2DEE742898B
:10934000018803890B44F7E75721224480F8D410A1
:10935000752182F8D410DA1C0233A4F88425FD228A
:1093600014FA83F383F8D4200023A4F88635B4F8E4
:109370008435002B95D1D4F89035002BB4D01C48FF
:10938000FDF7D8FD0546282DAED92046283DFFF72C
:1093900065FFD4F89035ADB2013BC4F89035002B91
:1093A000F1D1A1E7302300202189628992B28A425B
:1093B00003D1227B02F0FF016AB16168628992B237
:1093C000895C20736289013292B262816289258848
:1093D000954200D86081B4F88425013B551C13F0F8
:1093E000FF032244A4F8845582F8D410DCD1BBE7F3
:1093F000708A002031070020AA9A002001EB410169
:10940000490001F59671B1F5966F8ABF4FF49663E6
:10941000A0F88815A0F8883570474FF416735943A3
:10942000C0F88C15704708B5F8F747FF3023B0FB3C
:10943000F3F0C0B208BD312AF8B504460D4624D178
:10944000F8F73BFF2F2822D901231946227B02F08F
:10945000FF002AB161730133312BF7D10020F8BD31
:1094600066682289EF5C92B2B7542289013292B2C7
:10947000228122892688964200D82081208962890B
:1094800092B28242E7D12173E5E70420E7E70520A5
:10949000E5E7000000F50752002300F1180118323B
:1094A00003704361C0E90133C0E9033321F8023B93
:1094B0009142FBD142F2D81242F2DC118350224A8F
:1094C000425042F2E011425042F2E411425042F264
:1094D000E81242F20F71815242F2EC1200218350E5
:1094E00042F2F01283524FF0000242F2F213C254E1
:1094F00000F5075300F508523433143223F8021BE9
:109500009342FBD142F214230022C15200F50853CA
:1095100000F508511633363123F8022B9942FBD15E
:1095200042F236236321C25242F23823C15442F23E
:109530003C23C25000F509531A804FF0000242F25A
:109540004223C254704700BF0F270F27002342F267
:10955000EC1263210370835042F23822815442F2AC
:10956000D81242F2DC118350114A425042F2E0110B
:10957000425042F2E411425042F2E81242F20F71BC
:10958000815242F21422835242F23622835242F234
:10959000F012835242F2F212835442F23C22835080
:1095A00000F50952138042F242228354704700BFF3
:1095B0000F270F27F7B54FF47A533D4E04464FF06F
:1095C000000C1F4630461FFA8CF5AA421FD901F144
:1095D0000C0534F91550002D12DDA842B8BF2846FD
:1095E000AF42A8BF2F464D1D0CF1010CADB2B5F531
:1095F000875F22BFA1F586511B398DB22946E2E76C
:10960000AB42A8BF2B46AE42B8BF2E46EBE7C2190D
:1096100033442849521028485B10D5181BB26D10EE
:109620002EB2551B12B22DB2CDE9006502F0F0FD4D
:1096300042F2382104F5075204F50850635C3432D5
:109640001430632B24D1134623F8026B98421D84F7
:10965000FAD142F238230021E154002342F21421CE
:10966000635242F236216352194632F9025B2944B1
:10967000158C90422B4409B21BB2F6D1091142F26B
:1096800014221B11A15242F23622A35203B0F0BDA4
:1096900004EB4307013342F2F41CDBB227F80C6001
:1096A00042F216260F2BBD536354D2D8D5E700BF24
:1096B00080C1FFFF7ECF0108C0D900202DE9F04F07
:1096C00085B04FF00009DFF8B4B0BDF93C40BDF9FA
:1096D00040A00294BDF83850CAF1000401920394EE
:1096E0001FFA89F4019A944245D201F10C0405F164
:1096F000010C039A4FEAE50830F814601FFA8CFC5D
:10970000029C05F00707023513F808E0361B4FEA04
:10971000EC040CF0070C1BF8077036B21BF80CC0F9
:10972000ADB2964207DA2EEA070703F808701E5D0D
:109730004CEA060C08E0002E15DA2EEA070703F8BB
:1097400008701E5D26EA0C0C03F804C04C1D09F1DC
:109750000109A4B2B4F5875F22BFA1F586511B3978
:109760008CB22146BCE74EEA0707564503F808705D
:109770001E5DDDDAE6E705B0BDE8F08F20CE01081A
:1097800042F2D813C35A00EB83035B682DE9F04F14
:1097900023F07F4304466B4887B0584002F0D2FF65
:1097A000022800F2CB8042F2DA13DFF8A0C11825BC
:1097B0000027E35A4FF47A5163484FF6FD7E03F5D4
:1097C00083564FF003080D36B6B2B6F5875F24BF57
:1097D000A3F17306B6B2334603F10C021CF9019BE8
:1097E00034F912209042B8BF10469142A8BF1146EA
:1097F000B9F1010F00F09D80B9F1030F05D0B9F167
:10980000FF3F40F09880174401E012FB0E775A1D8D
:10981000013D92B2B2F5875F29BFA3F58652134688
:109820001B3A93B215F0FF05D6D142F2EC13E35880
:10983000BB4280F2858042F23823E35C632B0CD17B
:109840000B1842F214225B10A35244F63E12C31AC4
:10985000534342F23622DB13A35242F2362318223C
:1098600031462046E35E0DF11009DFF8E4A04FF029
:109870000608029342F21423E35E0193002300934F
:1098800004ABFFF71BFF2378002B0CBF4FF0020B3C
:109890004FF0040B19F8010B1AF8013B584002F085
:1098A00041FF054408F1FF30EDB210F0FF08F1D19F
:1098B0005D4543D842F2EC13052242F2E011E75035
:1098C00042F2F013E25242F2DA1342F2E812E35AA1
:1098D000A35242F2DE12A65203F58352073292B22D
:1098E000B2F5875F28BFA3F1790262522278E2B90C
:1098F00042F2E61242F2E211A35242F2DC12A65206
:1099000003F2BB7292B2B2F5875F28BFA3F62512AD
:10991000625203F2BD7242F2E41192B2B2F5875F75
:109920002ABFA3F6231362526352012007B0BDE899
:10993000F08FBF1A6BE712FB087768E70020F5E7A6
:109940002846F3E7A030FB0080C1FFFF2ECE0108C0
:1099500028CE010838B50446FFF712FFB8B142F22D
:10996000F215635D9BB942F23C2201211E48A350CF
:1099700004F509521380FDF7FBFA01211A48FDF79F
:1099800003FB42F238236322E2540A23635542F276
:10999000F212A35C33B3013BDBB2012BA35421D100
:1099A00042F2E61342F2E211E35A03F2BB7292B2C0
:1099B000B2F5875F28BFA3F62512625203F2BD728B
:1099C00042F2E41192B2B2F5875F2CBFA3F62313E3
:1099D00062524FF0000228BF63520123237042F20B
:1099E000F213E25438BD00BF708A002042F2DC134B
:1099F0000822C35A03F1780189B2B1F5875F28BF05
:109A0000A3F5835142F23623F0B5C35E9FB028BF61
:109A100008390446029342F2142328BF89B2C35E78
:109A200001930023009304ABFFF748FE9DF811302B
:109A300042F2422203F00F0383540F2B33D8DFE8A6
:109A400003F00832328C3232327A323232325732CA
:109A500032B142F2DC1542F236274FF4C67242F2BE
:109A60001426415BFFF7A6FDE35F42F2E612604970
:109A70000093A25EA35F5F4802F083FBE35F4FF4B5
:109A8000C672615B02932046A35F01930823009393
:109A900005ABFFF713FE012364228DF8143005A9EE
:109AA000544801F08FF842F2E81342F2E211E35A0F
:109AB00003F586521F3292B2B2F5875F28BF03F1D9
:109AC000FF3262525A1C42F2E41192B2B2F5875F41
:109AD0002CBFA3F5865362524FF0000224BF1F3BF8
:109AE00063520223237042F2EC13E2501FB0F0BD28
:109AF00042F2E61542F23627B42242F21426415BC6
:109B0000FFF758FDE35F625F00933B49A35F39486D
:109B100002F037FBE35FB422615B02932046A35F50
:109B200001930823009305ABFFF7C8FD01232E2204
:109B30008DF81430B3E742F2DC1542F23627B42236
:109B400042F21426415BFFF735FDE35F42F2E61275
:109B50002A490093A25EA35FD9E742F2DC1542F2E4
:109B60003627482242F21426415BFFF723FDE35FCC
:109B700042F2E61222490093A25EA35F1D4802F062
:109B800000FBE35F4822615B02932046A35F0193E1
:109B90000823009305ABFFF791FD012313228DF8F5
:109BA00014307CE742F2DC1542F23627D82242F22A
:109BB0001426415BFFF7FEFCE35F42F2E612114917
:109BC0000093A25EA35F0B4802F0DBFAE35FD822AA
:109BD000615B02932046A35F01930823009305ABCA
:109BE000FFF76CFD012337228DF8143057E700BFD3
:109BF00046CE0108C0D9002074CE0108A2CE0108CB
:109C0000D1CE0108FFCE010842F2E213C15A42F25E
:109C1000E413C25A42F2DA139142C35A10B5044611
:109C200013D2994204D89A4212D32046FFF7A8FDD6
:109C300042F2DA13E25A42F2E413E35A9A4207D1AB
:109C40002046BDE81040FFF7D1BE9942EBD8ECE7C3
:109C500010BD000038B500F5095504462888A0B1AC
:109C600042F23C23DB22E358B3FBF0F3C3F30720BB
:109C700081F8DA3081F8D900054800F0CFFF0023E1
:109C800042F23C22A3502B8038BDD922F4E700BF1A
:109C9000C0D9002042F2E213C15A42F2E413C25A80
:109CA00042F2DA139142C35AF0B50446BDB07CD2F9
:109CB000994204D89A4202D32046FFF761FD42F24E
:109CC000DA13E25A42F2E013E35A9A426BD142F2BB
:109CD000F013E35A052B1AD142F2E81342F2E211D3
:109CE000E35A03F586521F3292B2B2F5875F28BF5E
:109CF00003F1FF3262525A1C42F2E41192B2B2F501
:109D0000875F29BFA3F5865362521F3B635242F21D
:109D1000DE1542F236274FF458722046615B42F25C
:109D20001426FFF747FCE35F42F2E812274900934D
:109D3000A25EA35F264802F024FAE35F615B4FF462
:109D4000587202932046A35F01930823009305AB4A
:109D5000FFF7B4FC42F2F013E55A013DADB2E55213
:109D600035BB1C491A4801F0C1F929461A48FDF7CC
:109D7000FFF829461848FDF707F9154800F07AFF63
:109D800042F2E01342F20F722570E25242F238239F
:109D90006322E25442F2F213E55442F2EC13E5502E
:109DA00042F24223E5543DB0F0BD994282D883E7A8
:109DB0002B1F05A95D425D418DF81450FFF74AFF46
:109DC00042F2EC130022E250EDE700BF2FCF010872
:109DD000C0D900205DCF0108708A00202DE9F8432A
:109DE00000F5075504460E46971E01EB430818354B
:109DF000464548D042F23C2237F8020F36F9021BA2
:109E000042F2DA19A35800290344A35004F5095279
:109E1000138803F1010313802A8804EB820253683C
:109E20004FEA4303B8BF43F00103536034F80930ED
:109E30000C3324F813102378012B05D0022B1ED0ED
:109E40002046FFF787FD02E02046FFF7DDFE34F8ED
:109E5000093001339BB2B3F5875F25BF002342F27F
:109E6000422224F8093024F8093028BFA3542B8853
:109E700001339BB2042B88BF00232B80B8E7204618
:109E8000FFF708FFE3E7BDE8F8830000F8B50446F4
:109E900000254FF47A6004F128072581208004F121
:109EA00048066581657325730DF0C2FF3B4660600F
:109EB000A561A583C4E90455C4E9085523F8025BEC
:109EC0009E42FBD104F1C0033246002122F8021B5E
:109ED0009342FBD104F5AE61002203F8012B9942B5
:109EE000FBD1F023C4F87025C4F87C250021A4F828
:109EF000743541F2707320223846C4F878350EF07C
:109F0000CFF87822002130460EF0CAF805232662E9
:109F10002046237408236382034BC4E905372023BA
:109F2000A383024B6362F8BD180800206808002074
:109F3000F0B599B005460B46002402A94FF4D27043
:109F400040F2EC464FF614374FF65C6C03F0C0025B
:109F5000802A26D0C02A21D0002A0CBF62463A4669
:109F600021F8142001349B00042CDBB2EED12346EF
:109F700004AA05F110000DF083F80EAA04A905F15A
:109F80001C0014230DF05EFA00230EAA2146009354
:109F900014230548FDF7C4FB19B0F0BD21F8146087
:109FA000E0E721F81400DDE7708A002030B599B0B1
:109FB00005460024042304AA02A91030CDE9024476
:109FC0000DF05EF80EAA04A905F11C0014230DF093
:109FD00039FA14230EAA042102480094FDF7A0FBCD
:109FE00019B030BD708A002001EB4101890001F5F4
:109FF0001671B1F5966F8ABF4FF49663A0F8741589
:10A00000A0F8743570474FF496635943C0F878153B
:10A010007047000073B5B0F87035044623B3474865
:10A02000FCF788FF464E0546142D1BD9B4F872354F
:10A030002046143D5A1C2344ADB2A4F8722593F86F
:10A04000C010FFF775FF33781BB1D4F87835C4F82A
:10A050007C35B4F87225B4F870359A42E4D3002305
:10A06000C4F8703502B070BD428903899BB2934237
:10A0700018D1037B002B49D00388002B46D0314BED
:10A080001B78EBB9B4F87455772198B2B4F8702501
:10A09000854234D9501C22440133A4F8700582F85B
:10A0A000C010F2E7438902899A4204D903894289A0
:10A0B0009B1A9BB2E1E74289018803890B44F7E7C9
:10A0C00000250DF1060120462E46FAF730FA9DF8DC
:10A0D0000620EBB29A4212D90DF1070120468DF805
:10A0E0000760FAF724FAB4F8703501355A1C234496
:10A0F000A4F870259DF8072083F8C020E7E7002327
:10A10000A4F87235B4F87035002B88D1D4F87C35BA
:10A11000002BA7D00948FCF70DFF0546142DA1D947
:10A120002046143DFFF742FFD4F87C35ADB2013B29
:10A13000C4F87C35002BF1D194E700BF708A002071
:10A1400031070020AA9A002008B5F8F7B6F8D823FE
:10A15000B0FBF3F0C0B208BD122AF8B504460D46B4
:10A16000164643D9F8F7A9F8864241D8237B721ED8
:10A1700003F0FF016BB10123637300210120CBB217
:10A180009A4237D9267B06F0FF07BEB160730131D2
:10A19000F5E7606823899BB2C254238901339BB2DF
:10A1A000238123892088984200D8218121896389CD
:10A1B0009BB28B42E1D101232373DEE72B44666817
:10A1C00093F801C023899BB206F803C023890133A9
:10A1D0009BB22381238926889E4200D82781268925
:10A1E00063899BB2B342D2D12073D0E70420F8BD7B
:10A1F0000520FCE70020FAE770B5044600254FF47F
:10A200007A6004F11C0625812080658165732573C1
:10A210000DF00EFE04F5B873324660602582C4E985
:10A22000055522F8025B9342FBD104F50E71002222
:10A2300003F8012B9942FBD14823C4F838220021AE
:10A240004FF4AA72A4F83C3230460DF029FF0623E1
:10A25000666120462382014BA36170BDA8080020DF
:10A260002DE9F047ADF5227D07460E46082402ADE4
:10A27000DFF85490DFF854A0A846330604F1FF3409
:10A2800028464FF028024CBF514649460DF06EFE5D
:10A2900014F0FF044FEA460605F12805F6B2ECD1AA
:10A2A00052AA414607F11000A0230DF0CBF8A023DD
:10A2B00052AA062103480094FDF732FA0DF5227DDB
:10A2C000BDE8F087708A00209ECF0108C6CF010844
:10A2D00001EB41014908483196298ABF9623A0F82D
:10A2E0003C12A0F83C32704708B5B0F838322BB9B0
:10A2F000F9F758F8003018BF012008BD0120FCE72D
:10A3000038B50446F9F74EF8B4F83812E8B981B315
:10A310002F48FCF70FFE0546A02D2AD9B4F83A3293
:10A320002046A03D5A1C2344ADB2A4F83A2293F82B
:10A330007011FFF795FFB4F83A22B4F838329A4218
:10A34000EAD30023C4F8383213E00029E0D1214BCE
:10A350001B78BBB9B4F83C52AA2198B2B4F83822A1
:10A36000854207D80023A4F83A32B4F83832002BDB
:10A37000CED138BD501C22440133A4F8380282F8F3
:10A380007011EAE744220B462089618989B2814233
:10A3900003D1217B01F0FF0069B16068618989B256
:10A3A000405C23736189013189B2618161892588AB
:10A3B0008D4200D86381B4F83812013A4D1C12F076
:10A3C000FF022144A4F8385281F87001DCD1C9E7BA
:10A3D000708A0020AA9A002008B5F7F76EFF442380
:10A3E000B0FBF3F0C0B208BD442AF8B504460D46F0
:10A3F00024D1F7F762FF432822D900220121237BD1
:10A4000003F0FF002BB161730132442AF7D1002021
:10A41000F8BD66682389AF5C9BB2F754238901338A
:10A420009BB22381238926889E4200D820812089DF
:10A4300063899BB28342E7D12173E5E70420E7E714
:10A440000520E5E700B58FB0C27A037A01780D9256
:10A45000827A01EB81010C92427A0B92427B0A9242
:10A46000027B0992C3F380120892DA090792C3F3C0
:10A47000401203F00F0306920593C3790493837986
:10A4800003934379029303790193C378009383780C
:10A4900042780348FAF704FB0FB05DF804FB00BFF5
:10A4A000E87C002070B50346044600F500720025E4
:10A4B00003F8015B9A42FBD14FF4B976A4F810522D
:10A4C000C4F80052A4F81252304684F80452A4F89A
:10A4D000086284F8145284F815520DF0A9FCA4F80F
:10A4E0002852C4F80C023046A4F82A52C4F8185274
:10A4F000A4F81C52A4F8206284F82C5284F82D523F
:10A500000DF096FCC4F82402204670BD1FB54FF430
:10A510009C638DF80F1003AA0121ADF80C30702355
:10A520008DF80E3000230093042301F0FFFF05B0E7
:10A530005DF804FB1FB54FF4BC638DF80B108DF86C
:10A540000C200121ADF808307F2302AA8DF80A30D3
:10A5500000230093052301F0E9FF05B05DF804FB3B
:10A5600010B504468CB06F48FCF714FE4FF4A753A7
:10A570000DF10F020DF10E01ADF810300123694805
:10A580008DF81230684B1B788DF81330674B1B78B1
:10A590008DF81430FCF7E0FD9DF80E302BB19DF8DE
:10A5A000143043F002038DF814305E48FCF7EDFDE3
:10A5B00028B19DF8143043F004038DF81430594845
:10A5C000FCF7DCFD28B19DF8143043F008038DF84A
:10A5D00014305448FCF7E5FD28B19DF8143043F0E1
:10A5E00010038DF814309DF80F302BB19DF8143006
:10A5F00043F020038DF814304D4A9DF81430127842
:10A60000002A14BF4022002213438DF81430002387
:10A610008DF81530474B1B78002B5ED04648FAF773
:10A6200079F88DF81600454B1B78002B5FD0444B12
:10A630001B78002B54D04348F8F71FFE8DF8170005
:10A640004048F8F722FE8DF818003F4B1B78002B8E
:10A6500052D03E4802F085FD8DF819003C4B1B7826
:10A66000002B4CD03B48FFF76FFD8DF81A003A4B9A
:10A670001B78002B46D03948FEF7D5FE8DF81B001D
:10A68000374B1B78002B40D03648FEF75CF88DF82E
:10A690001C00354B1B78002B3AD03448FAF7B6FF34
:10A6A0008DF81D00324B1B78ABB33248FFF794FE98
:10A6B0008DF81E00304B1B7883B33048F6F7C2FA92
:10A6C0008DF81F00002304AA01212046089300935F
:10A6D000142301F02BFF0CB010BD8DF81630A2E74B
:10A6E0000A2327488DF81730F7F704FEABE78DF8FB
:10A6F00017308DF81830A8E78DF81930AEE78DF8CF
:10A700001A30B4E78DF81B30BAE78DF81C30C0E77B
:10A710008DF81D30C6E78DF81E30CBE78DF81F3061
:10A72000D0E700BF708A0020A99A0020AA9A0020D2
:10A73000A89A002030070020407A00202F07002030
:10A7400031070020845800203707002030EF002018
:10A750003507002000D200203407002028AA00205E
:10A7600033070020AC95002032070020E87C002051
:10A770003607002080D700202E070020F413002089
:10A780009831002010B5184BB4B004461748029316
:10A7900040F27F33ADF80C30FDF7D6FA10228DF879
:10A7A0000E0000210DF10F000DF07AFC0F480DF1A5
:10A7B0000F01FDF7CBFA17230D48A3F11702D2B210
:10A7C000825C32B134A91944013301F8C82CDBB2E0
:10A7D000F3E70092012102AA20468DF8093001F02A
:10A7E000A5FE34B010BD00BFE0000002708A00205A
:10A7F000EECF0108072A2DE9F04F97B036D94B78F4
:10A8000000208C7903EB83030E7804F00109C4F374
:10A81000400A5B008F7891F803C0C4F3800491F87C
:10A8200004E091F8058016AD05EB000BC51DEDB2F7
:10A830004D5D0BF8345C00F108050130EDB2C0B29B
:10A840009542F0DB16AA09A91044002200F8342C26
:10A85000324600970648CDE905A4CDE90389CDE944
:10A8600001CEFAF7B9F817B0BDE8F08F0420FAE787
:10A87000E87C0020052AF0B5164693B028D94B781D
:10A88000C87803EB83030A7800EB80008F785B00C5
:10A8900091F804C04400002012AD05EB000E451DE8
:10A8A000EDB24D5D0EF8345C851D0130EDB2C0B2E5
:10A8B000B542F1DB12A90844002100F8341C05A9B7
:10A8C00000970448CDE9014CFAF7C6F813B0F0BD83
:10A8D0000420FBE7E87C00200D2A02D90846FFF798
:10A8E000B1BD042070470000032AF0B591B021D912
:10A8F00088780E7800EB80004B78CF7844000420F5
:10A90000051F0DF1400C90425CFA85F506DA11F84E
:10A9100000C0013005F834CCC0B2F1E7002203A931
:10A92000054805F8342C3246CDE90047FAF720F9FE
:10A9300011B0F0BD0420FBE7E87C002010B5044610
:10A940004FF4E132012101F0B3FD20464FF41652DD
:10A950000321BDE8104001F0ABBD0000134B1B7894
:10A96000012B30B591B01FD8114B1B78E3B1E02318
:10A970000024ADF80C3010238DF80E30E5B2EB1C3E
:10A98000AA42DBB206D910AD2B440D5D013403F8A9
:10A99000345CF3E703320121D3B20022009203AA10
:10A9A0008DF80D3001F0C2FD11B030BDA99A002024
:10A9B00030070020134B1B78012B30B589B01FD80E
:10A9C000114B1B78E3B1E0230024ADF80C301123C8
:10A9D0008DF80E30E5B2EB1CAA42DBB206D908AD09
:10A9E0002B440D5D013403F8145CF3E703320121BD
:10A9F000D3B20022009203AA8DF80D3001F096FD2B
:10AA000009B030BDA99A0020300700201FB50C4BBB
:10AA10001B78012B10D80B4B1B786BB14FF478735C
:10AA200003AA0121ADF80C3012238DF80E3000235B
:10AA30000093032301F07AFD05B05DF804FB00BF2D
:10AA4000A99A0020300700201FB50C4B1B78012B62
:10AA500010D80B4B1B786BB14FF4787303AA01210C
:10AA6000ADF80C3013238DF80E3000230093032330
:10AA700001F05CFD05B05DF804FB00BFA99A002061
:10AA80003007002030B5164C8DB0247814F0FD044A
:10AA900023D1144D2D7805B300294FF0E00514BFE4
:10AAA0001A211821ADF808508DF80A102146CDB2B0
:10AAB000EC1CAB42E4B206D90CAD2C44555C013120
:10AAC00004F8285CF3E7033300220121DBB2009293
:10AAD00002AA8DF8093001F029FD0DB030BD00BF8C
:10AAE000A99A00202F0700201FB50E4B1B7813F0EA
:10AAF000FD0313D10C4A127882B14FF47872002909
:10AB000000934FF00101ADF80C2014BF1B22192255
:10AB100003238DF80E2003AA01F008FD05B05DF8AF
:10AB200004FB00BFA99A00202F070020144B1B78BC
:10AB3000032B30B5A5B000D0FBB9124B1B78E3B1A5
:10AB4000E0230024ADF80C3020238DF80E30E5B260
:10AB5000EB1CAA42DBB206D924AD2B440D5D0134B7
:10AB600003F8845CF3E703320121D3B200220092A0
:10AB700003AA8DF80D3001F0D9FC25B030BD00BF1F
:10AB8000A99A0020370700201FB50C4B1B78032B18
:10AB900000D083B90A4B1B786BB14FF4787303AACA
:10ABA0000121ADF80C3021238DF80E3000230093E5
:10ABB000032301F0BBFC05B05DF804FBA99A00205B
:10ABC00037070020134B30B51C78A1B014F0FB04FC
:10ABD0001ED1114B1B78DBB1E023ADF808303023D8
:10ABE0008DF80A30E5B2EB1CAA42DBB206D920ADE3
:10ABF0002B440D5D013403F8785CF3E70332012147
:10AC0000D3B20022009202AA8DF8093001F08EFC26
:10AC100021B030BDA99A002035070020134B30B574
:10AC20001C78C3B014F0FB041ED1114B1B78DBB1B0
:10AC3000E023ADF80C3031238DF80E30E5B2EB1C7B
:10AC4000AA42DBB206D942AD2B440D5D013403F8B4
:10AC5000FC5CF3E703320121D3B20022009203AA85
:10AC60008DF80D3001F062FC43B030BDA99A002090
:10AC7000350700201FB50C4B1B7813F0FB030FD1D9
:10AC80000A4A127862B14FF47872009301210323CB
:10AC9000ADF80C2032228DF80E2003AA01F046FCFC
:10ACA00005B05DF804FB00BFA99A0020350700201D
:10ACB000144B1B78052B30B5A5B000D0FBB9124B57
:10ACC0001B78E3B1E0230024ADF80C3040238DF86D
:10ACD0000E30E5B2EB1CAA42DBB206D924AD2B4400
:10ACE0000D5D013403F8845CF3E703320121D3B234
:10ACF0000022009203AA8DF80D3001F017FC25B058
:10AD000030BD00BFA99A0020340700201FB50C4BAE
:10AD10001B78052B00D083B90A4B1B786BB14FF41D
:10AD2000787303AA0121ADF80C3041238DF80E3061
:10AD300000230093032301F0F9FB05B05DF804FB49
:10AD4000A99A002034070020144B1B78072B30B53C
:10AD5000A5B000D0FBB9124B1B78E3B1E02300246F
:10AD6000ADF80C3045238DF80E30E5B2EB1CAA424D
:10AD7000DBB206D924AD2B440D5D013403F8845CAD
:10AD8000F3E703320121D3B20022009203AA8DF827
:10AD90000D3001F0CBFB25B030BD00BFA99A0020DB
:10ADA00033070020144B1B78072B30B5A5B000D01B
:10ADB000FBB9124B1B78E3B1E0230024ADF80C3053
:10ADC00046238DF80E30E5B2EB1CAA42DBB206D961
:10ADD00024AD2B440D5D013403F8845CF3E70332AA
:10ADE0000121D3B20022009203AA8DF80D3001F0A8
:10ADF0009DFB25B030BD00BFA99A0020330700207D
:10AE00001FB50C4B1B78072B00D083B90A4B1B785E
:10AE10006BB14FF4787303AA0121ADF80C304923CC
:10AE20008DF80E3000230093032301F07FFB05B063
:10AE30005DF804FBA99A0020330700201FB50C4BD6
:10AE40001B78072B00D083B90A4B1B786BB14FF4EA
:10AE5000787303AA0121ADF80C3048238DF80E3029
:10AE600000230093032301F061FB05B05DF804FBB0
:10AE7000A99A002033070020214B1B780A2B30B5FC
:10AE8000ADF5037D00D01BBB1E4B1B7803B3E02345
:10AE9000FC2AD4B28DF808301FD9053400230139BB
:10AEA00003AD8DF80A4065248DF809308DF80B400C
:10AEB00011F8014F05F8014B5C1CA4B2A2420AD163
:10AEC000053300229BB20121009202AA01F02EFB61
:10AED0000DF5037D30BD2346EAE7033465238D1865
:10AEE0008DF809400DF10B048DF80A30A94204D009
:10AEF00011F8013B04F8013BF8E7D31CE1E700BF80
:10AF0000A99A0020320700207FB50D4B1B780A2B31
:10AF100000D093B90B4B1B787BB14FF49C638DF839
:10AF20000F1003AA0121ADF80C3066238DF80E3006
:10AF300000230093042301F0F9FA07B05DF804FB45
:10AF4000A99A0020320700207FB50C4B1B780A2BF2
:10AF500000D083B90A4B1B786BB14FF4787303AA06
:10AF60000121ADF80C3067238DF80E3000230093DB
:10AF7000032301F0DBFA07B05DF804FBA99A002077
:10AF800032070020214B1B780A2B30B5ADF5037D2D
:10AF900000D01BBB1E4B1B7803B3E023FC2AD4B2AA
:10AFA0008DF808301FD905340023013903AD8DF821
:10AFB0000A4055248DF809308DF80B4011F8014FE7
:10AFC00005F8014B5C1CA4B2A2420AD10533002251
:10AFD0009BB20121009202AA01F0A8FA0DF5037DAF
:10AFE00030BD2346EAE7033455238D188DF8094018
:10AFF0000DF10B048DF80A30A94204D011F8013B81
:10B0000004F8013BF8E7D31CE1E700BFA99A002050
:10B010002E07002070B5C2B01346E02402AA1480A7
:10B02000802494700024E6B2F51CB342EDB203D93B
:10B030000E5D01345655F6E703330021DBB2537041
:10B040000091012101F072FA42B070BD124B1B78E1
:10B05000632B30B5A5B01CD1E0230024ADF80C3033
:10B0600008238DF80E30E5B2EB1CAA42DBB206D9FC
:10B0700024AD2B440D5D013403F8845CF3E7033207
:10B080000121D3B20022009203AA8DF80D3001F005
:10B090004DFA25B030BD00BFA99A0020124B1B7895
:10B0A000602B30B58BB01CD1E0230024ADF8083004
:10B0B00009238DF80A30E5B2EB1CAA42DBB206D9AF
:10B0C0000AAD2B440D5D013403F8205CF3E7033235
:10B0D0000121D3B20022009202AA8DF8093001F0BA
:10B0E00025FA0BB030BD00BFA99A002090F80432B9
:10B0F00010B5A4B0C3B1E023ADF80C30F1238DF846
:10B100000E300323DA1ED2B28A5C32B124AC1C4466
:10B11000013304F8842CDBB2F4E7012103AA8DF893
:10B120000D30009101F002FA24B010BD5F2910B576
:10B130000C4600F0888020D806297ED00ED803293E
:10B1400075D005D8012939D0022961D0454960E080
:10B1500004296ED00529F9D143495AE05B297CD0F6
:10B1600005D8072967D00A29F0D1404951E05C2968
:10B1700071D05D29EAD13E494BE0672965D00ED8F0
:10B1800063295CD005D860295BD06229DED13949BA
:10B190003FE0652963D06629D8D1374939E06A296B
:10B1A000FBD005D8682952D06929CFD1334930E086
:10B1B0006B294ED06C29C9D131492AE03149324836
:10B1C000FFF794FF3148F7F7E8F83148F6F70DFC40
:10B1D0003048F7F7CBFA032C23D12F48FEF7B6F906
:10B1E000052C04D02D48FDF7B5FC072C04D02C48C5
:10B1F000FCF7EEFD0A2C02D02A48F9F79CFB2A48FE
:10B20000F6F7B8FB21462948BDE81040FBF7C0BE61
:10B2100027491D48FFF76AFF2648F8F79DFA022CD8
:10B22000D0D1254801F01EFB042CDBD0D5E7234903
:10B23000EFE72349EDE72349EBE72349E9E7234912
:10B24000E7E72349E5E72349E3E72349E1E7234922
:10B25000DFE72349DDE72349DBE72349D9E7234932
:10B26000D7E700BFEDD40108FED2010832D30108B0
:10B270004CD401085ED30108AFD301080ED40108F5
:10B28000D3D40108B1D20108C0D900208C360020E7
:10B29000DC1A0020DC3B0020BCAF0020AC9A002070
:10B2A000C08D0020E87C0020EC160020708A002071
:10B2B000C4D2010870590020F0DB0020D4D201086C
:10B2C000EED201080FD301081FD3010841D30108B2
:10B2D00078D3010893D30108CED30108EFD3010836
:10B2E0002DD401086ED4010893D40108B6D4010806
:10B2F000242A2DE9F04FA9B003D8042029B0BDE8D5
:10B30000F08F0E78C6F3001380F804324C78CD78B5
:10B3100004F0100304F0020A322D04F00409129321
:10B3200004F0200304F00808119304F04003109384
:10B33000E3D891F804C091F802B0BCF1050F17D919
:10B34000BCF1070F00F02781BCF1060F00F025814A
:10B35000BCF10A0F00F02481ACF15B03DBB2112BCE
:10B36000CBD8904A22FA03F313F0010F0DD1C4E7B2
:10B37000BCF1010F02D114F0010FF7E7BCF1020F8D
:10B3800040F0F080BAF1000FB7D08F7E0F2FB4D805
:10B390000B7F0F937C3B0E2BAFD84B7904F001044D
:10B3A0000A7D13938B7927921493CB7915930B7A9B
:10B3B00016934B7A17938B7A1893CB7A19930B7B4E
:10B3C0001A934B7B1B938B7B1C93CB7B1D930B7C2A
:10B3D0001E934B7C1F934B7D20938B7D2193CB7DC4
:10B3E0002293CB7E26934B7F23938B7F2493CB7F1B
:10B3F00061462593FFF79AFEF1436B48C1F3C011F4
:10B4000001706A496A480C702946F9F781F81AF107
:10B41000000A684918BF4FF0010A674881F800A088
:10B420002946F6F73BFF39466448F7F701FF3946EE
:10B430006348F7F783F9269B61481946F7F78AF9BD
:10B4400039466048F6F76EFC39465F48F7F72EF943
:10B4500019F100095D4B294618BF4FF001095C48FE
:10B4600083F8009001F066FE279AC6F3C0015848A1
:10B4700001F06FFE18F10008564B294618BF4FF037
:10B480000108554883F80080FEF7AEFD2099524828
:10B49000FEF7B9FD129B514A29460033504818BFA8
:10B4A00001231370FDF7AAFF21994D48FDF7B5FF61
:10B4B000109B4C4A294600334B4818BF0123137098
:10B4C000FDF72CF922994848FDF737F90BF00102F6
:10B4D000464B294646481A70FEF7FAFECBF3400366
:10B4E000444A239944481370F5F7A6FB0F9B434841
:10B4F000A3F18001DDE9242349B2F5F7DAF9119BC4
:10B500003F4A06F0010100333E4818BF0123137083
:10B51000C6F34013C6F340020D93149B803B0C937B
:10B52000139B803B0B931F9B0A931E9B09931D9BB0
:10B5300008931C9B07931B9B06931A9B0593199BCF
:10B540000493189B0393179B0293169B0193159BDF
:10B550000093C6F38003FBF790FD2A48FBF77EFDBE
:10B560000020CBE6BCF1030F04D1B9F1000F7FF44A
:10B570000CAFC2E6BCF1040F04D1B8F1000F7FF4A8
:10B5800004AFBAE6BCF1050F7FF4FFAE129B002BAF
:10B590007FF4FBAEB1E6109BF9E71BF0010FE5E687
:10B5A000119BF4E7BFFD03003107002030070020A6
:10B5B000407A00202F070020983100208458002076
:10B5C000DC3B0020DC1A00208C36002037070020EE
:10B5D00030EF00203507002000D200203407002083
:10B5E00028AA002033070020AC9500203607002051
:10B5F00080D700202E070020F4130020680A0020C6
:10B6000032070020708A002008B502B31E4B09786B
:10B610001B788B4213D0052913D907292DD0062971
:10B620002DD00A292DD0A1F15B03DBB2112B0ED84E
:10B63000164A22FA03F3DB0709D5FFF777FD00214D
:10B6400015E0012905D1124B1B78002BF5D10421FF
:10B650000DE0022901D10F4BF6E7032901D10E4B72
:10B66000F2E7042905D10D4B1B78002BE5D10846E4
:10B6700008BD0529E1D10A4BE6E70A4BE4E70A4B8E
:10B68000E2E70A4BE0E700BFA99A0020BFFD0300F4
:10B69000300700202F070020370700203507002043
:10B6A000340700203307002036070020320700202F
:10B6B00090F8043270B5A4B013B3E023ADF80C30A9
:10B6C000F2238DF80E300323DC1E24ADE4B21D44BA
:10B6D0000E5D5C1CE4B21EB105F8846C2346F3E7F2
:10B6E0001112023305F8841C24A9DBB20C44012199
:10B6F00004F8842C03AA00918DF80D3000F016FF99
:10B7000024B070BD20292DE9F04104460D461646AF
:10B710001F4600F0A9826BD8102900F0E1811FD8E4
:10B72000032900F0F0800FD8012900F0E68040F2F4
:10B73000E7801A463146FFF7DBFD0221024620462C
:10B740005AB1FEF7F7FED3E0082900F021810A295B
:10B7500000F0B081042940F0A480FEF7D7FEC7E0D6
:10B760001A2900F01C8225D8132900F0DE8118293F
:10B7700000F0F281112940F09480B34B1B78002B2C
:10B7800000F0D181DFF8E88298F80030012B00F258
:10B79000CA813A463146AD48F9F70AF8054600280D
:10B7A00000F0AE812AB2AA49AA48FFF781FF2A46D3
:10B7B0001121BFE01D2900F014821E2900F03E82F5
:10B7C0001C296ED1A44B1B78002B00F035823A4621
:10B7D0003146A248F7F752FC0546002800F0888061
:10B7E0002AB29F499B48FFF763FF2A461C21A1E02C
:10B7F000552900F038834CD8452900F0CE8223D853
:10B80000312900F05A82402900F07382302948D152
:10B81000944B1B78002B00F04782DFF8548298F895
:10B82000003013F0FB0F40F03F823A4631468E481D
:10B83000FEF792FC0546002840F0378298F8003069
:10B84000002B55D1042161E1492900F0C88250291B
:10B8500000F0E082462924D1844B1B78002B00F0B5
:10B86000BC82834B1A78984612B1072A40F0B58201
:10B87000FAB231467F48FCF76EFF0546002800F01B
:10B880009C822AB27C497348FFF712FF2A46462160
:10B8900050E0632972D006D861294DD05CD8602968
:10B8A00038D0012256E0802900F0F8821BD86529A3
:10B8B000F7D1724B1B78002B00F0CC826C4B1A78BE
:10B8C000984612B10A2A40F0C582FAB231466C4855
:10B8D000F9F7A6FE0546002840F0BD8298F8003032
:10B8E00033B90A2112E101F17003DBB2012BD8D880
:10B8F0000023C4F80032BDE8F081FEF731FEF7E71F
:10B90000FEF740FFF4E71A463146FFF77DFE294671
:10B91000024614E71A463146FEF76CFF054610B999
:10B920006021204619E702B256494A48FFF7C0FE97
:10B930002A466021204604E731461A46FEF79AFF60
:10B94000064608B92946ECE702B24F494148FFF7DD
:10B95000AFFE32462946EDE70D2B06D91046FEF71D
:10B9600071FD054610B96221DBE704252AB247497B
:10B970003848FFF79DFE2A466221DBE731461A462A
:10B98000FEF7B2FF06460028DCD002B24049DDE7F0
:10B99000374B1A789846632A4CD13A4631463D488F
:10B9A000F5F74CFD054698F800305C3BDBB2062B02
:10B9B0000AD84D2222FA03F3DB0705D53A46314671
:10B9C0003548F5F759FB054698F80030663B052BDE
:10B9D00005D83A4631463148F5F7ECFD054698F86A
:10B9E00000305D2B05D13A4631462D48F5F77EFEF5
:10B9F000054698F800305B2B05D13A463146294878
:10BA0000F5F736FE054698F800306C2B05D13A461E
:10BA100031462548F5F7F4FD054698F80030652BCA
:10BA200005D13A4631462148F5F78AFE05461DB94B
:10BA3000082176E70225B6E72AB21D490548FFF737
:10BA400037FE2A46082175E730070020407A00209B
:10BA5000E5D00108C0D900202F070020845800201D
:10BA600053D101083507002000D200203307002001
:10BA7000A99A0020AC95002025D2010832070020A9
:10BA8000E87C00201DD001083AD0010857D00108F9
:10BA900074D00108C416002058160020C8160020D3
:10BAA000DC160020D9160020D8160020DE16002053
:10BAB00091D001089B4B1B7883B93A4631469A488E
:10BAC000F5F7E8FE054600283FF412AF2AB2974981
:10BAD0009748FFF7EDFD2A460A212BE70525F5E7F4
:10BAE000944B1B78B3B1DFF83C8298F80030012BFF
:10BAF00010D83A4631469048F8F734FE054650B91A
:10BB000098F80030002B7FF4F3AE01212046FFF7B8
:10BB10000DFBEDE602252AB288498548FFF7C8FDEE
:10BB20002A46102106E702253CE6824B1B7853B1DA
:10BB30007C4E3278012A06D87F48F8F75FFE05462A
:10BB400010B93378DEE702252AB27D497848FFF73D
:10BB5000AFFD2A461321EDE67A4B1B78B3B1714B4A
:10BB60001A78984612F0FD0F10D1774B1B786BB105
:10BB70003A4631467548F7F791FB054638B998F8CB
:10BB80000030002B7FF4B4AE0221BFE702252AB2B9
:10BB90006F496748FFF78CFD2A461821CAE6694BB2
:10BBA0001B78E3B15F4B1A78984612F0FD0F16D15F
:10BBB000654B3A4631461B786BB16448F7F7B0FBEA
:10BBC00005460028DBD02AB261495948FFF770FDCD
:10BBD0002A461A21AEE65F48F6F794FBF0E7022505
:10BBE000F1E7584B1B78E3B1012F23D111780129DC
:10BBF0000CD14C4B1B78022B1CD1574B1B78002BC4
:10BC00007FF476AE5148F7F783FA71E691B9454B68
:10BC10001B78022B0ED1504B1B78002B3FF468AEE3
:10BC2000F0E702252A464D494148FFF741FD2A46E3
:10BC30001D217FE60425F5E70225D1E5414B1B7860
:10BC400083B13A4631464148F7F74CFA0546002899
:10BC50003FF44EAE2AB242493548FFF729FD2A4645
:10BC60001E2167E60225F5E73E4B1B789BB12D4B65
:10BC70001A7898460AB1032A0DD13A4631463A4815
:10BC800001F077FA054638B998F80030002B7FF4B8
:10BC90002FAE03213AE702252AB234492448FFF7A0
:10BCA00007FD2A46202145E602252AB230492048D0
:10BCB000FFF7FEFC2A4630213CE62E4B1B78B3B141
:10BCC000184B1A78984612F0FB0F10D13A463146BD
:10BCD0002948FEF741FA054600283FF4AFAD2AB2E5
:10BCE00026491348FFF7E4FC2A46312122E60225C3
:10BCF000F5E7234B1B78002B46D00A4B1A78984661
:10BD00000AB1052A40D13A4631461E48FDF793FB59
:10BD10000546D0BB98F80030002B7FF4E9AD052133
:10BD2000F4E600BFA99A0020EC160020B3D0010869
:10BD3000C0D9002030070020407A0020C6D001087A
:10BD400002D101082F07002031070020845800206D
:10BD50001ED1010898310020AA9A002038D101088C
:10BD600071D101083707002030EF00208CD1010885
:10BD7000B0D101083507002000D20020CCD1010845
:10BD80003407002028AA002002252AB25B495C481B
:10BD9000FFF78EFC2A464021CCE55A4B1B789BB11D
:10BDA000594B1A7898460AB1072A0DD1FAB2314692
:10BDB0005648FCF7D0FC054638B998F80030002BFF
:10BDC0007FF496AD0721A1E602252AB250494C48DE
:10BDD000FFF76EFC2A464521ACE5022551E5494BAB
:10BDE0001B78ABB1484B1A7898460AB1072A0FD195
:10BDF000FAB231464548FCF7AEFC05460028DCD0D7
:10BE00002AB244493E48FFF753FC2A46492191E5AE
:10BE10000225F5E7404B1B789BB13B4B1A789846BF
:10BE20000AB1062A0DD13A4631463C48FEF7DCFA03
:10BE3000054638B998F80030002B7FF459AD06213B
:10BE400064E602252AB236492D48FFF731FC2A461E
:10BE500050216FE502252AB232492948FFF728FC14
:10BE60002A46652166E5304B1B78ABB1264B1B7823
:10BE70000BB10A2B10D13A4631462C48F4F7F4FEA8
:10BE8000054600283FF434AD2AB229491C48FFF783
:10BE90000FFC2A4655214DE50225F5E70022012138
:10BEA00093B29F427FF624AD94F8143203F0FF0062
:10BEB0001BB184F815120132F2E7D4F80C52B4F831
:10BEC000103216F802C09BB205F803C0B4F8103265
:10BED00001339BB2A4F81032B4F81032B4F808520F
:10BEE0009D4201D8A4F81002B4F81002B4F812323E
:10BEF0009BB28342DFD184F81412DCE7E5D101085C
:10BF0000C0D9002033070020A99A0020AC9500205A
:10BF100000D2010846D201083607002080D7002051
:10BF20005FD201087CD201082E070020F413002004
:10BF300095D201082DE9F0410446C2B00126C51C86
:10BF4000071D0121204600F0BDFA8046002840D0A0
:10BF50000121204600F0DAFAB4F8003201463BB97C
:10BF6000E02806BF2070C4F80062A4F80232E8E7B7
:10BF7000012B06D102236070A4F80202A4F800325B
:10BF8000DFE7022BB4F8022210D10323A070A4F83B
:10BF900000321AB9FF31A4F80212D2E7032AD0D135
:10BFA00000232A462046FFF7ADFBCAE7E0540133E1
:10BFB0009BB29342A4F80032C3D1FF2B89BF043B4C
:10BFC000033B3A46E1788FBF9BB22A469BB2A178E9
:10BFD000E8E74F48FBF7E2F84BF67F33B4F812225C
:10BFE0009842B4F810329BB288BFC4F800829342E2
:10BFF00040D194F81432002B51D0B4F80852002DDF
:10C000004DD00321204600F06FFA002685423746C6
:10C01000C8BF85B2B3B29D4241D9B4F81022B4F87A
:10C0200012328DF80C709BB2934202D194F8143204
:10C03000BBB1D4F80C22B4F812329BB2D35C84F8B2
:10C0400014728DF80C30B4F8123201339BB2A4F89C
:10C050001232B4F81232B4F808229A4201D8A4F885
:10C0600012720097012303AA03212046013600F033
:10C070005DFACFE7B4F81232B4F810229A4206D92A
:10C08000B4F81052B4F81232ED1AADB2B7E7B4F802
:10C090001232B4F80822B4F810521544F4E7032120
:10C0A000204600F00FFA051E2EDDD4F81822AA4211
:10C0B00028D1B4F81C32632B03D8F92A01DC0133F0
:10C0C0001BE003AE37460321204600F01FFA08F1BB
:10C0D0000108D4F81822454506F8010B02F1FF3299
:10C0E000C4F8182202D0B8F1FA0FECD1AA1A3946D6
:10C0F0002046D2B2FEF78EFF0023A4F81C3242B0D5
:10C10000BDE8F081F92DDCDCC4F81852F4E700BF7B
:10C11000708A0020F0B51E4690F80432A5B073B3C3
:10C12000E0230324ADF80C30F3238DF80E30E51E28
:10C1300024ABEDB223444F5D651CEDB21FB103F893
:10C14000847C2C46F3E7111203F8841C24AB0121F4
:10C150001D4405F8842CA21C53FA82F2331202F813
:10C16000843C221D0334D3B224AA52FA84F403AAD5
:10C1700004F8846C00918DF80D3000F0D7F925B0EB
:10C18000F0BDF0B590F80442A5B0BDF9A860002C50
:10C190003CD0E024ADF80C40F4248DF80E4003248C
:10C1A000E51E24AFEDB2274411F805C0651CEDB2C1
:10C1B000BCF1000F03D007F884CC2C46F0E7111235
:10C1C00007F8841C24A90D4405F8842CA21C51FAFC
:10C1D00082F2191202F8841C24A9E21C51FA82F29C
:10C1E00002F8843C231D321251FA83F303F8842CA5
:10C1F000A31D053403AADBB251FA84F4012104F82B
:10C20000846C00918DF80D3000F090F925B0F0BDF0
:10C21000F0B590F80442A5B0BDF9A870BDF9AC60C6
:10C22000002C49D0E024ADF80C40F5248DF80E40E8
:10C230000324E51E0DF1900CEDB2A44411F805E0C5
:10C24000651CEDB2BEF1000F03D00CF884EC2C4657
:10C25000EFE711120CF8841C24A90D4405F8842C76
:10C26000A21C51FA82F2191202F8841C24A9E21CC1
:10C2700051FA82F202F8843C231D3A1251FA83F3F8
:10C2800003F8842C631D321251FA83F303F8847C83
:10C29000A31D51FA83F303F8842C04F10803073437
:10C2A00003AADBB251FA84F4012104F8846C0091F2
:10C2B0008DF80D3000F03AF925B0F0BD30B5E0232F
:10C2C000ADF5037DFC2AD4B28DF808301FD90534B2
:10C2D0000023013903AD8DF80A40FA248DF80930A6
:10C2E0008DF80B4011F8014F05F8014B5C1CA4B20E
:10C2F000A2420AD1053300229BB20121009202AA78
:10C3000000F014F90DF5037D30BD2346EAE7FA236A
:10C3100003348D188DF80A300DF10B038DF80940A8
:10C32000A94204D011F8014B03F8014BF8E7D31CE4
:10C33000E1E70000014800F077B900BF38040120B0
:10C3400030B501218BB0224C0546082004F062FF75
:10C3500001214FF4802004F0C5FF20460722082168
:10C3600003F0E2F807220921204603F0DDF8194B1B
:10C3700001A8019300F0DEFF02A802F0CFFD4FF408
:10C380004072154B02A92046A4F5E234CDE9022300
:10C3900002F024FD04A809F0F5F9002304A92046C1
:10C3A000079309930495CDE905330C23089309F00D
:10C3B0002DF92046012109F043FA012220460749C0
:10C3C0000AF02CFA2146064800F0EBF80BB030BD1D
:10C3D000000C0240270101010202000105010500D5
:10C3E00038040120014800F01FB900BF2CF40020E0
:10C3F00070B501218AB00646042004F00BFF264DDB
:10C400000121082004F006FF244C01214FF4801084
:10C4100004F068FF284608220C2103F085F8082262
:10C420000221204603F080F81D4B01A8019300F083
:10C4300081FF02A802F072FD4FF48052194B02A94D
:10C440002846CDE9022302F0C9FC042302A92046B4
:10C45000029302F0C3FC04A8A4F5DE3409F092F9BB
:10C46000002304A92046079309930496CDE90533D8
:10C470000C23089309F0CAF82046012109F0E0F9DD
:10C480000122204608490AF0C9F92146074800F070
:10C4900088F80AB070BD00BF00080240000C0240DE
:10C4A0003501010102020001050105002CF4002004
:10C4B0000129104602D0032902D07047FFF740BF80
:10C4C000FFF796BF012908B503D0032905D0002046
:10C4D00008BD034800F00FF9FAE70248FAE700BF89
:10C4E000380401202CF40020012908B503D00329C9
:10C4F00005D0002008BD034800F006F9FAE702481D
:10C50000FAE700BF380401202CF40020012903D0F1
:10C51000032904D000207047024800F079B802488F
:10C52000FBE700BF380401202CF400200846114628
:10C530001A46012810B59DF8084002D003280AD0F9
:10C5400010BD084800F030F8002CF9D00548BDE8CF
:10C55000104000F0C5B8044800F026F8002CEFD0D9
:10C560000148F4E7380401202CF4002008B5044801
:10C5700000F00AF80348BDE8084000F005B800BF25
:10C58000380401202CF40020002241F20801A0F818
:10C5900004280260A0F80628425241F20A014252E1
:10C5A0007047016070470000F8B504460D46164616
:10C5B0005AB3006848B341F208070978E35B9BB2BD
:10C5C0005A1CC3F30A0392B22344E253012283F8B4
:10C5D000081827440D490AF021F90022013293B2CC
:10C5E0009E420BD93B88A85C9BB2591CC3F30A033B
:10C5F00089B22344398083F80808EFE720680122D4
:10C600000249BDE8F8400AF009B9F8BD0701070082
:10C61000B0F806389BB25A1CC3F30A0392B2034423
:10C62000A0F806281879704710B50446006800285D
:10C630004ED028490AF0B8FAD8B1B4F80438B4F8A2
:10C64000062801335340C3F30A0373B1206809F08D
:10C6500057FCB4F80438C0B29BB25A1CC3F30A03A7
:10C6600092B22344A4F8042818711A491A480AF00F
:10C6700023FB1A4920680AF097FA48B341F20A02EC
:10C6800041F20803A15AE35A9BB28B420CD0A35A41
:10C690009BB2591CC3F30A0389B22344A15293F8F5
:10C6A0000818206809F0F4FB0C4920680AF004FB24
:10C6B00041F20A03E25A41F20803E35A9BB2934261
:10C6C00006D1206800220549BDE810400AF0A6B84E
:10C6D00010BD00BF05010500001001400701070063
:10C6E00010B5036804462BB1802120680AF05CFA7B
:10C6F0000028F9D110BDB0F80628B0F804389BB274
:10C70000981A18BF0120704741F2080341F20A024B
:10C71000C35A825A581C5040C0F30A00003018BF58
:10C7200001207047014B185C704700BFFED4010820
:10C73000034AC3B2000AD35C105C1844C0B270470D
:10C74000FED40108084AC3B2C0F30721D35C515C90
:10C750000B44C0F30741000E515C105C51FA83F3A7
:10C7600050FA83F0C0B27047FED40108124AC3B237
:10C7700010B5C0F30724D35C145D2344C0F3074411
:10C78000000E145D105C54FA83F350FA83F0CBB2C0
:10C79000D35C53FA80F0C1F30723D35C53FA80F0E3
:10C7A000C1F30743090ED35C53FA80F0535C53FA8C
:10C7B00080F0C0B210BD00BFFED4010800F5965253
:10C7C000002300F11801183203704361C0E90133FE
:10C7D000C0E9033321F8023B9142FBD141F2D82258
:10C7E00041F2DC2183501E4A425000F597510A6005
:10C7F00041F2E42242F20F71815241F2E82200211B
:10C80000835041F2EC2283524FF0000241F2EE23BA
:10C81000C25400F5975300F598521033103223F8A4
:10C82000021B9342FBD141F210330022C15200F5AA
:10C83000985300F599511233123123F8022B994283
:10C84000FBD141F232336321C25241F23433C1543D
:10C8500041F23833C25041F23C33C252704700BFFC
:10C860000F270F27002341F2E82263210370835032
:10C8700041F23432815441F2D82241F2DC2183501A
:10C880000E4A425000F597510A6041F2E42242F20A
:10C890000F71815241F21032835241F2323283528F
:10C8A00041F2EC22835241F2EE22835441F23832BB
:10C8B000835041F23C328352704700BF0F270F274D
:10C8C000F7B54FF47A533C4E04464FF0000C1F4628
:10C8D00030461FFA8CF5AA421ED901F10C0534F935
:10C8E0001550002D11DDA842B8BF2846AF42A8BFA1
:10C8F0002F464D1D0CF1010CADB2B5F5166F24BFDE
:10C90000A1F65B118DB22946E3E7AB42A8BF2B46E7
:10C91000AE42B8BF2E46ECE7C21933442749521045
:10C9200027485B10D5181BB26D102EB2551B12B2E2
:10C930002DB2CDE90065FFF76BFC41F2343104F50F
:10C94000975204F59850635C10321030632B24D159
:10C95000134623F8026B98421D84FAD141F2343316
:10C960000021E154002341F21031635241F232318F
:10C970006352194632F9025B2944158C90422B44CC
:10C9800009B21BB2F6D1091141F210321B11A152AA
:10C9900041F23232A35203B0F0BD04EB430701333E
:10C9A00041F2F02CDBB227F80C6041F212360F2B6B
:10C9B000BD536354D2D8D5E780C1FFFF67D60108C5
:10C9C000C0D900202DE9F04F85B04FF00009DFF805
:10C9D000B4B0BDF93C40BDF940A00294BDF8385058
:10C9E000CAF10004019203941FFA89F4019A944257
:10C9F00044D201F10C0405F1010C039A4FEAE50859
:10CA000030F814601FFA8CFC029C05F00707023511
:10CA100013F808E0361B4FEAEC040CF0070C1BF887
:10CA2000077036B21BF80CC0ADB2964207DA2EEA98
:10CA3000070703F808701E5D4CEA060C08E0002E9C
:10CA400014DA2EEA070703F808701E5D26EA0C0CBC
:10CA500003F804C04C1D09F10109A4B2B4F5166F26
:10CA600024BFA1F65B118CB22146BDE74EEA070751
:10CA7000564503F808701E5DDEDAE7E705B0BDE84D
:10CA8000F08F00BFFED5010841F2D823C35A00EB56
:10CA900083035B682DE9F04FC3F313030446594841
:10CAA00087B05840FFF74EFE032800F2A78041F2FE
:10CAB000DA23DFF858E114250026E35A4FF6FD7813
:10CAC00051494FF0030903F60117BFB2B7F5166FCE
:10CAD00028BFA3F15F074FF47A5328BFBFB23A468D
:10CAE00002F10C001EF901CB34F910008142B8BFED
:10CAF00001468342A8BF0346BCF1010F79D0BCF1C7
:10CB0000030F04D0BCF1FF3F75D1064401E010FBD8
:10CB10000866501D013D80B2B0F5166F2ABFA2F61F
:10CB20005B12024692B215F0FF05D9D141F2E8221C
:10CB3000A258B24264DA41F23432A25C632A0CD1C8
:10CB40000B4441F210325B10A352CB1A44F63E1153
:10CB500041F232324B43DB13A35241F232331422FF
:10CB600039462046E35E0DF11009DFF8A4A04FF02E
:10CB70000508029341F21033E35E01930023009312
:10CB800004ABFFF71FFF2378002B0CBF4FF0020B05
:10CB90004FF0040B19F8010B1AF8013B5840FFF74E
:10CBA000C1FD054408F1FF30EDB210F0FF08F1D1EE
:10CBB0005D4523D841F2E823052241F2DE21012020
:10CBC000E65041F2EC23E25241F2DA2304F59752A7
:10CBD000E35A138041F2DC22A75203F6FB0292B221
:10CBE000B2F5166F2ABF653B6252635207B0BDE8CB
:10CBF000F08F361A8DE710FB09668AE70020F5E70B
:10CC00002846F3E7ADB5070080C1FFFF0BD601084A
:10CC100006D6010838B50446FFF736FFB8B141F231
:10CC2000EE25635D9BB941F2383201211D48A350C6
:10CC300041F23C32A352FAF79BF901211948FAF765
:10CC4000A3F941F234336322E2540523635541F2E0
:10CC5000EE22A35C2BB3013BDBB2012BA35420D10A
:10CC600004F5975341F2E2211B8803F65F1292B25A
:10CC7000B2F5166F28BF03F1FF3262525A1C41F21F
:10CC8000E42192B2B2F5166F2CBFA3F65F13625285
:10CC90004FF0000228BF63520123237041F2EE23BC
:10CCA000E25438BD708A002041F23C3310B504468E
:10CCB000C05AB0B141F238337B22E358B3FBF0F3F2
:10CCC000C3F3072081F87A3081F879000648FDF730
:10CCD0002DFF002341F23832A35041F23C32A352DF
:10CCE00010BD7922F2E700BFC0D9002041F2E22353
:10CCF000C15A41F2E423C25A41F2DA239142C35AA3
:10CD00002DE9F0410446A4B079D2994204D89A4260
:10CD100002D32046FFF7B8FE41F2DA23E25A41F28D
:10CD2000DE23E35A9A4267D141F2EC2304F597558A
:10CD3000E35A052B16D12B8841F2E22103F65F124C
:10CD400092B2B2F5166F28BF03F1FF3262525A1C3D
:10CD500041F2E42192B2B2F5166F2ABFA3F65F1337
:10CD60006252635241F2DC2641F232384FF4F072E3
:10CD70002046A15B41F21037FFF7A2FD34F90830DD
:10CD8000274900932748B5F90020E35FFFF7F9F939
:10CD900034F908304FF4F072A15B02932046E35F50
:10CDA00001930823009305ABFFF70CFE41F2EC233F
:10CDB000E55A013DADB2E55225BB1B491948FEF7C6
:10CDC00095F929461948FAF7D3F829461748FAF78A
:10CDD000DBF81448FDF7D8FE41F2DE2342F20F7271
:10CDE0002570E25241F234336322E25441F2EE23E1
:10CDF000E55441F2E823E55024B0BDE8F0819942C2
:10CE000085D886E72B1F05A95D425D418DF814503A
:10CE1000FFF74AFF41F2E8230022E250ECE700BFAF
:10CE20001FD60108C0D9002046D60108708A00200C
:10CE30002DE9F84300F5965504460E46971E01EB82
:10CE40004308183546453BD041F2383237F8020FD7
:10CE500036F9021B41F2DA29A3580029034420467F
:10CE6000A35041F23C32A35A03F10103A3522A8892
:10CE700004EB820253684FEA4303B8BF43F0010357
:10CE8000536034F809300C3324F813102378012B45
:10CE900013D1FFF72BFF34F8093001339BB2B3F500
:10CEA000166F28BF002324F809302B8801339BB26A
:10CEB000042B88BF00232B80C4E7FFF7ABFEEAE713
:10CEC000BDE8F88370B5044600254FF47A6004F19C
:10CED0001C06258120806581657325730AF0A8FFF3
:10CEE00004F13C0332466060A561C4E9045522F8B0
:10CEF000025B9342FBD104F2EC41002203F8012BC8
:10CF00009942FBD1F023C4F8EC2484F8F2240021E8
:10CF1000A4F8F0344FF49653C4F8F8243046C4F81B
:10CF2000F43420220BF0BCF8052320462374092397
:10CF30006382024BC4E9053670BD00BFB40800200F
:10CF4000F0B590F9F2348FB01C4D0A46002B1C4B03
:10CF500040F2657740F2772C08BF1D46A3F2EE43FE
:10CF6000184E16BF4FF46D771E464FF49E7C00237B
:10CF700002A902F0C004802C1DD0C02C18D0002CB7
:10CF80000CBF2C46344621F8134001339200042B89
:10CF9000D2B2EED104AA10300AF072F8002304AA2B
:10CFA0000321009314230848FAF7BAFB0FB0F0BD31
:10CFB00021F81370E9E721F813C0E6E7C4FEFFFF8C
:10CFC00089FDFFFF4CFCFFFF708A002010B58EB07A
:10CFD00000240423103004AA02A9CDE902440AF077
:10CFE0004FF8142304AA032102480094FAF798FB8F
:10CFF0000EB010BD708A002070B5B0F8EC34044655
:10D000001BB34948F9F796FF484E0546142D1BD926
:10D01000B4F8EE342046143D5A1C2344ADB2A4F8B3
:10D02000EE2493F83C10FFF78BFF33781BB1D4F854
:10D03000F434C4F8F834B4F8EE24B4F8EC349A427A
:10D04000E4D30023C4F8EC3470BD428903899BB259
:10D0500093422DD1037BA3B1038893B1344B1B784A
:10D06000002B3BD1B4F8F054772198B2B4F8EC24FB
:10D07000A8422BD30023A4F8EE34B4F8EC34002BF0
:10D08000BFD1D4F8F834002BDED02748F9F752FF8F
:10D090000546142DD8D92046143DFFF797FFD4F844
:10D0A000F834ADB2013BC4F8F834002BF1D1CBE732
:10D0B000438902899A4204D9038942899B1A9BB207
:10D0C000CBE74289018803890B44F7E7501C2244CF
:10D0D0000133A4F8EC0482F83C10C6E77823002062
:10D0E0002189628992B28A4203D1227B02F0FF0138
:10D0F0006AB16168628992B2895C20736289013287
:10D1000092B2628162892588954200D86081B4F824
:10D11000EC24013B551C13F0FF032244A4F8EC540B
:10D1200082F83C10DCD1A5E7708A0020310700208E
:10D13000AA9A002001EB4101890001F51671B1F5B1
:10D14000966F8ABF4FF49663A0F8F014A0F8F034FD
:10D1500070474FF4966380F8F2145A43C0F8F424F1
:10D16000704708B5F5F7A9F87823B0FBF3F0C0B223
:10D1700008BD792AF8B504460D4624D1F5F79DF887
:10D18000772822D901231946227B02F0FF002AB119
:10D1900061730133792BF7D10020F8BD66682289CD
:10D1A000EF5C92B2B7542289013292B22281228975
:10D1B0002688964200D820812089628992B28242D4
:10D1C000E7D12173E5E70420E7E70520E5E7000064
:10D1D00038B543780446072B03D92521364809F092
:10D1E000D3FE2378012B03D92621334809F0CCFE46
:10D1F0006278324B9A601D462278002A58D0237BF1
:10D20000012B03D92E212C4809F0BEFEE37A032B13
:10D2100006D9053B012B03D92F21274809F0B4FE7D
:10D22000A37A022B03D93021234809F0ADFE637B9A
:10D23000012B03D93121204809F0A6FEA37B012B45
:10D2400003D932211C4809F09FFEE37B012B03D94F
:10D250003321194809F098FE637AFF2B03D134215A
:10D26000154809F091FE237A043B1B2B03D9352185
:10D27000114809F089FE6368EB60E37A227B1B06A4
:10D2800043EA027322781343A27A43EAC243627BE1
:10D2900043EA8243A27B43EA4243E27B43EA0243FE
:10D2A000627A43EA0223227A43EA42032B6138BDC1
:10D2B000DA601A61FBE700BF87D6010890ED00E055
:10D2C000054A536A23F480335362D2F8943023F032
:10D2D0000103C2F89430704700ED00E0044B40F0C9
:10D2E0000100044A5860536A43F480335362704724
:10D2F00090ED00E000ED00E0B0F5C06F10B5044621
:10D300000DD020F48073B3F5806F08D020F48063D3
:10D31000B3F5407F03D08021044809F035FE44F086
:10D32000BF64034B44F40034DC6010BD87D60108B1
:10D3300000ED00E0C378012B70B5044603D99421B9
:10D340001B4809F021FE63780F2B03D9952118485B
:10D3500009F01AFEA3780F2B03D99621144809F07F
:10D3600013FE2178012601F01F034D099E40E3784A
:10D37000CBB1104BDA686378D243C2F30222C2F118
:10D380000400C0B28340D8B20F2343FA02F2A3785C
:10D390001340094A034311441B01DBB281F80033F7
:10D3A00042F8256070BD2035034B43F82560F9E74E
:10D3B00087D6010800ED00E000E100E038B50D4B34
:10D3C00005460C46984206D0B0F1006F03D0BE214E
:10D3D000094809F0D9FD094B9C4203D9BF210648F1
:10D3E00009F0D2FD24F06041054B21F07F01294373
:10D3F000996038BD0000022087D60108FEFF0F00AB
:10D4000000ED00E0102870B505460E4603D80C4B21
:10D41000C340DB0703D4D1210A4809F0B5FD012E32
:10D42000094C07D9D221074809F0AEFD23691D43F5
:10D43000256170BD002EF9D1236923EA0505F7E7C0
:10D440001400010087D6010800ED00E0042810B5A3
:10D45000084C0AD0053003D0E921074809F094FDB3
:10D46000236823F00403236010BD236843F0040302
:10D47000F9E700BF10E000E087D6010808B50121F8
:10D480004FF4807003F0FEFF00214FF48070BDE880
:10D49000084003F0F7BF000038B53C4B05460C468A
:10D4A00098420BD003F58073984207D003F5807340
:10D4B000984203D08921364809F066FD236833F08D
:10D4C000407303D08A21324809F05EFD2379012B95
:10D4D00003D98B212E4809F057FD6379012B03D91D
:10D4E0008C212B4809F050FDA36833F0405303D042
:10D4F0008D21274809F048FDE36833F0407212D0CF
:10D50000B2F1806F0FD023F0A062B2F1006F0AD0A9
:10D51000B3F1306F07D003F17143012B03D98E2192
:10D520001B4809F031FD236933F4006303D08F21D8
:10D53000174809F029FD237D013B0F2B03D99021CA
:10D54000134809F021FD6A682179236822F04072AE
:10D5500043EA012322F4807213430E4A6B60AB68E6
:10D560001A40D4E903130B43A1680B43617943EAE2
:10D5700041031343AB60227DEB6A013A23F470034D
:10D58000D2B243EA0253EB6238BD00BF0020014033
:10D59000BBD60108FDF7FFC0002303608380036151
:10D5A000C0E9023301230375704700000268192A9D
:10D5B00010B5044603D81B4BD340DB0703D4F2213C
:10D5C000194809F0E1FC636833F4403303D0F321D8
:10D5D000154809F0D9FCA36833F4404303D0F42183
:10D5E000114809F0D1FCE36833F440730CD0B3F573
:10D5F000806F09D0B3F5006F06D0B3F5406F03D04C
:10D60000F521094809F0C0FC0849D4E9003248680E
:10D610001343074A02401343A2681343E2681343CB
:10D620004B6010BDE702E602BBD6010800230140B3
:10D63000E030FCFF0023C0E90033C0E9023370474B
:10D6400038B5124B04460D4698420CD003F5807352
:10D65000984208D003F58073984204D040F22B1111
:10D660000B4809F091FC012D09D94FF49671084837
:10D6700009F08AFCA36843F00103A36038BD002DC4
:10D68000F8D1A36823F00103F7E700BF00200140B1
:10D69000BBD6010838B5174B05460C4698420CD04E
:10D6A00003F58073984208D003F58073984204D044
:10D6B0004FF4B271104809F067FC24F400020F4BDC
:10D6C0009A420FD024F40073B3F5000F0AD0B4F5DA
:10D6D000400F07D034F4800304D040F265110648AF
:10D6E00009F052FC6B6823F4400323F400731C43DD
:10D6F0006C6038BD00200140BBD60108000240002C
:10D70000134B984270B504460E4615460CD003F5EF
:10D710008073984208D003F58073984204D040F299
:10D7200081110C4809F030FCB6F5805F04D34FF44A
:10D73000C171084809F028FCB5F5805F04D340F2B8
:10D740008311044809F020FC6662A56270BD00BF29
:10D7500000200140BBD6010838B50F4B04460D46EA
:10D7600098420CD003F58073984208D003F580737B
:10D77000984204D04FF4D571084809F005FC122DE9
:10D7800004D940F2AB11054809F0FEFB636823F0B1
:10D790001F031D43656038BD00200140BBD6010852
:10D7A000012810B5084C09D940F2E911074809F0E1
:10D7B000EBFB636843F40003636010BD0028F8D1FD
:10D7C000636823F40003F7E700230140BBD6010898
:10D7D000012810B5084C09D940F20321074809F087
:10D7E000D3FB636843F48003636010BD0028F8D165
:10D7F000636823F48003F7E700230140BBD60108E8
:10D800002DE9F0419846384B05460F46984214469C
:10D810000CD003F58073984208D003F580739842CA
:10D8200004D04FF41A71314809F0AEFB122F04D91D
:10D8300040F269212D4809F0A7FB661EF3B20F2BB9
:10D8400004D940F26A21294809F09EFBB8F1070F7C
:10D8500004D940F26B21254809F096FB092F1BD90A
:10D86000A7F10A030721EA6803EB4303994008FA8A
:10D8700003F322EA01021343EB60062C18D806EBEF
:10D8800086061F236C6BB34007FA06F624EA0304EE
:10D8900026436E63BDE8F08107EB470107232A6941
:10D8A0008B4022EA030208FA01F313432B61E4E7F9
:10D8B0000C2C0CD8E31F1F242E6B03EB83039C401E
:10D8C00026EA040407FA03F634432C63E2E70D3C2E
:10D8D000EA6A04EB84031F249C4022EA040207FA4C
:10D8E00003F41443EC62D5E700200140BBD60108E5
:10D8F0000B4B984210B504460CD003F58073984248
:10D9000008D003F58073984204D040F2DF21054827
:10D9100009F03AFBA36843F08043A36010BD00BF49
:10D9200000200140BBD601080A4B984210B50446BE
:10D930000CD003F58073984208D003F580739842A9
:10D9400004D040F2EE21044809F01EFBA068C0F3A9
:10D95000807010BD00200140BBD6010838B5124BC5
:10D9600004460D4698420CD003F58073984208D0C7
:10D9700003F58073984204D040F20B310B4809F054
:10D9800003FB012D09D94FF44371084809F0FCFA53
:10D99000A36843F48063A36038BD002DF8D1A36869
:10D9A00023F48063F7E700BF00200140BBD60108E5
:10D9B00038B5124B04460D4698420CD003F58073DF
:10D9C000984208D003F58073984204D04FF449710F
:10D9D0000B4809F0D9FA012D09D940F22531084840
:10D9E00009F0D2FAA36843F00203A36038BD002D0A
:10D9F000F8D1A36823F00203F7E700BF002001403D
:10DA0000BBD6010838B5114B04460D4698420CD0E0
:10DA100003F58073984208D003F58073984204D0D0
:10DA200040F241310A4809F0AFFA013DEBB2072B51
:10DA300004D940F24231064809F0A6FA616821F49F
:10DA4000604141EA4531616038BD00BF00200140BE
:10DA5000BBD6010838B5124B04460D4698420CD08F
:10DA600003F58073984208D003F58073984204D080
:10DA700040F25E310B4809F087FA012D09D940F2D6
:10DA80005F31084809F080FA636843F4006363601B
:10DA900038BD002DF8D1636823F40063F7E700BFB9
:10DAA00000200140BBD601080A4B984210B504463D
:10DAB0000CD003F58073984208D003F58073984228
:10DAC00004D040F27531044809F05EFAE06C80B28F
:10DAD00010BD00BF00200140BBD60108014B1868F3
:10DAE000704700BF0823014038B5124B04460D466D
:10DAF00098420CD003F58073984208D003F58073E8
:10DB0000984204D04FF46E710B4809F03DFA012D94
:10DB100009D940F2B931084809F036FAA36843F44C
:10DB20008073A36038BD002DF8D1A36823F48073FF
:10DB3000F7E700BF00200140BBD6010838B5124B03
:10DB400004460D4698420CD003F58073984208D0E5
:10DB500003F58073984204D04FF474710B4809F0B8
:10DB600013FA012D09D940F2D131084809F00CFA15
:10DB7000A36843F40073A36038BD002DF8D1A368F7
:10DB800023F40073F7E700BF00200140BBD6010873
:10DB9000012810B5084C09D940F2EB31074809F0CB
:10DBA000F3F9636843F40053636010BD0028F8D1B3
:10DBB000636823F40053F7E700230140BBD6010854
:10DBC000F8B51F462A4B06460D46984214460CD01F
:10DBD00003F58073984208D003F58073984204D00F
:10DBE00040F24341234809F0CFF9122D04D940F205
:10DBF0004441204809F0C8F9631E032B04D940F2C0
:10DC000045411C4809F0C0F9072F04D940F24641AC
:10DC1000184809F0B9F9092D1DD9A5F10A03072102
:10DC2000F26803EB4303994007FA03F322EA010287
:10DC30001343F360B36B0234C3F30152A41A1F22DF
:10DC4000E4B204EB8404A24005FA04F423EA0203DC
:10DC50001C43B463F8BD05EB4501072332698B40D3
:10DC600022EA030207FA01F313433361E2E700BF3C
:10DC700000200140BBD6010838B5114B04460D46C3
:10DC800098420CD003F58073984208D003F5807356
:10DC9000984204D040F283410A4809F075F9013DE9
:10DCA000EBB2032B04D940F28441064809F06CF929
:10DCB000A16B21F4401141EA0551A16338BD00BFB9
:10DCC00000200140BBD60108002373B5019303F186
:10DCD000804305460C4603F59033164698420CD017
:10DCE00003F58073984208D003F58073984204D0FE
:10DCF00040F2A541114809F047F9A4F11403DBB241
:10DD00000C2B05D841F2111222FA03F3DB0704D4DD
:10DD100040F2A641094809F037F9B6F5805F04D30F
:10DD200040F2A741054809F02FF90195019B1C44D9
:10DD30000194019B1E6002B070BD00BFBBD60108FC
:10DD400038B5154B05460C4698420CD003F5807348
:10DD5000984208D003F58073984204D040F2CB413A
:10DD60000E4809F011F934F440330FD024F4102296
:10DD7000B2F5802F0AD0B4F5E02F07D0B3F5002F0D
:10DD800004D040F2CC41054809F0FEF8AB6823F41A
:10DD900070231C43AC6038BD00200140BBD6010895
:10DDA00038B5104B04460D4698420CD003F58073ED
:10DDB000984208D003F58073984204D040F2ED41B8
:10DDC000094809F0E1F835F4401304D040F2EE417F
:10DDD000054809F0D9F8A36823F440131D43A56052
:10DDE00038BD00BF00200140BBD601080B4B984254
:10DDF00010B504460CD003F58073984208D003F5A3
:10DE00008073984204D040F20151054809F0BCF8F3
:10DE1000A36843F48003A36010BD00BF002001404D
:10DE2000BBD601080A4B984210B504460CD003F546
:10DE30008073984208D003F58073984204D040F272
:10DE40000F51044809F0A0F8A068C0F3805010BD3D
:10DE500000200140BBD6010838B5124B04460D46E0
:10DE600098420CD003F58073984208D003F5807374
:10DE7000984204D040F22B510B4809F085F8012D4F
:10DE800009D940F22C51084809F07EF8636843F440
:10DE90008063636038BD002DF8D1636823F480632C
:10DEA000F7E700BF00200140BBD6010838B5124B90
:10DEB00004460D4698420CD003F58073984208D072
:10DEC00003F58073984204D040F245510B4809F0A5
:10DED0005BF8012D09D940F24651084809F054F881
:10DEE000636843F48053636038BD002DF8D16368E4
:10DEF00023F48053F7E700BF00200140BBD60108A0
:10DF0000002337B5019303F1804304460D4603F522
:10DF1000903398420CD003F58073984208D003F5F3
:10DF20008073984204D040F263510E4809F02CF8F7
:10DF3000A5F11403DBB20C2B05D841F2111222FA21
:10DF400003F3DB0704D440F26451064809F01CF8DF
:10DF500001940199283129440191019B186880B2EC
:10DF600003B030BDBBD601081D4B984270B50446C6
:10DF70000D4616460CD003F58073984208D003F581
:10DF80008073984204D040F2CD51164808F0FCFF4F
:10DF9000012E04D940F2CE51124808F0F5FF40F2AC
:10DFA00005239D420FD0B5F5837F0CD040F2074387
:10DFB0009D4208D042F21A039D4204D040F2CF5154
:10DFC000084808F0E1FF0123EDB203FA05F56368A4
:10DFD00016B11D43656070BD23EA0505FAE700BF71
:10DFE00000200140BBD6010838B5134B04460D464E
:10DFF00098420CD003F58073984208D003F58073E3
:10E00000984204D040F2F2510C4808F0BDFF6B1E5C
:10E01000DBB21F2B04D80A4A22FA03F3DB0704D42D
:10E0200040F2F351054808F0AFFF23681D4214BFCA
:10E030000120002038BD00BF00200140BBD60108F0
:10E040008B80008038B50F4B05460C4698420CD0AB
:10E0500003F58073984208D003F58073984204D08A
:10E0600040F21461084808F08FFF14F0C00F00D18F
:10E0700024B940F21561044808F086FFE4432C609F
:10E0800038BD00BF00200140BBD6010838B51A4B8F
:10E0900005460C4698420CD003F58073984208D090
:10E0A00003F58073984204D040F22C61134808F0C5
:10E0B0006BFF40F205239C420FD0B4F5837F0CD058
:10E0C00040F207439C4208D042F21A039C4204D01B
:10E0D00040F22D61094808F057FF6A68286810EA85
:10E0E000142007D00123E4B203FA04F4144214BF4D
:10E0F0001846002038BD00BF00200140BBD60108F3
:10E1000038B5154B05460C4698420CD003F5807384
:10E11000984208D003F58073984204D040F25361CE
:10E120000E4808F031FF40F205239C420FD0B4F5B1
:10E13000837F0CD040F207439C4208D042F21A037E
:10E140009C4204D040F25461044808F01DFF6FEA7D
:10E1500014242C6038BD00BF00200140BBD601084C
:10E1600008B501214FF0005003F06AF900214FF08B
:10E170000050BDE8084003F063B9000038B50B68F3
:10E1800005460C4633F0040211D023F010020C2A8D
:10E190000DD023F02002142A09D023F00802242AEB
:10E1A00005D03C2B03D053211A4808F0EDFE6368DC
:10E1B00033F0400205D0802B03D05421154808F0DD
:10E1C000E3FEA36833F4407309D0B3F5806F06D043
:10E1D000B3F5006F03D055210E4808F0D5FEE36873
:10E1E00033F0020303D056210A4808F0CDFE0A4955
:10E1F00040F6FE720B68AA4023EA0202D4E900301E
:10E200000343A0680343E0680343AB4013430B6040
:10E2100038BD00BFF8D60108007400400023C0E9F3
:10E220000033C0E90233704730F0100370B5044684
:10E230000E4603D08D210B4808F0A6FE0125012EC5
:10E2400005FA04F5084C07D98E21064808F09CFE13
:10E2500023681D43256070BD002EF9D1236823EA91
:10E260000505F7E7F8D601080074004030F0100308
:10E2700070B505460E4603D0A9210C4808F084FE6F
:10E280002B09012E4FF00105094C05FA03F507D9BA
:10E29000AA21064808F078FE63681D43656070BDDA
:10E2A000002EF9D1636823EA0505F7E7F8D60108DF
:10E2B00000740040012810B5084C08D9C121084855
:10E2C00008F062FE636843F00303636010BD00283A
:10E2D000F8D1636823F00303F7E700BF0074004040
:10E2E000F8D6010830F0100370B505460C46164606
:10E2F00003D0E0210E4808F047FE402C05D0802CCA
:10E3000003D0E1210A4808F03FFE012E04FA05F48B
:10E31000084D07D9E221064808F036FE2B681C4359
:10E320002C6070BD002EF9D12B6823EA0404F7E7B6
:10E33000F8D6010800740040002337B5019330F08F
:10E34000040304460D4605D0082803D0FF210B48DE
:10E3500008F01AFE4FF6F0739D4204D94FF4807115
:10E36000064808F011FE064B01930198083020443E
:10E370000190019B1D6003B030BD00BFF8D60108BD
:10E3800000740040002337B5019330F004030446C5
:10E390000D4606D0082804D04FF48C710A4808F0C6
:10E3A000F3FD4FF6F0739D4204D940F2191106486F
:10E3B00008F0EAFD054B01930198143020440190C8
:10E3C000019B1D6003B030BDF8D601080074004009
:10E3D000F8B530F0040305460F46144606D0082869
:10E3E00004D04FF49A710E4808F0CEFD4FF6F0734A
:10E3F0009C421E4604D940F23511094808F0C4FD7C
:10E40000B74204D94FF49B71054808F0BDFD082DB3
:10E41000044B0CBF44EA072444EA0744EC50F8BD1F
:10E42000F8D6010820740040002313B5019330F0A2
:10E430001003044604D04FF4AB71074808F0A4FD64
:10E44000064B019301982C3000EB94000190019B46
:10E45000186880B202B010BDF8D601080074004000
:10E4600030F0100370B504460E4604D040F281111E
:10E470000C4808F089FD4FF48055012E05FA04F58B
:10E48000094C08D94FF4C171064808F07DFD236896
:10E490001D43256070BD002EF9D1236823EA0505D0
:10E4A000F7E700BFF8D601080074004030F0100311
:10E4B00070B504460D46164604D040F2B11114481A
:10E4C00008F062FD012E05FA04F415D94FF4D97154
:10E4D0000F4808F059FDB5F5005F04D10D4B1A68DF
:10E4E00014431C6070BDB5F1005F08D040F2B31159
:10E4F000074808F049FD02E0B5F5005FF3D1002EB2
:10E50000ECD1044A136823EA04041460EAE700BF6C
:10E51000F8D601080074004038B530F01003054605
:10E520000C4604D04FF4E9710A4808F02DFDB4F50B
:10E53000005F07D0B4F1005F04D040F2D31105486A
:10E5400008F022FD044BAC405B6B1C4214BF012061
:10E55000002038BDF8D601080074004038B530F00E
:10E56000100305460C4604D04FF4FA71084808F031
:10E570000BFDB4F5005F07D0B4F1005F04D040F2AA
:10E58000F511034808F000FDAC40024B5C6338BD58
:10E59000F8D601080074004038B530F01003054685
:10E5A0000C4604D040F20E210C4808F0EDFCB4F506
:10E5B000005F07D0B4F1005F04D040F20F2107489C
:10E5C00008F0E2FC064BAC401A68586B204003D0C0
:10E5D000224214BF0120002038BD00BFF8D6010838
:10E5E0000074004038B530F0100305460C4604D0E6
:10E5F00040F23321084808F0C7FCB4F5005F07D0AB
:10E60000B4F1005F04D04FF40D71034808F0BCFC76
:10E61000AC40024B5C6338BDF8D601080074004082
:10E620000F2810B5044603D98D21054808F0ACFC2D
:10E63000044B186820F00F002043186010BD00BF85
:10E6400035D70108003C0240012810B5084C08D914
:10E650009D21084808F098FC236843F480732360E8
:10E6600010BD0028F8D1236823F48073F7E700BFBA
:10E67000003C024035D70108012810B5084C08D9E4
:10E68000B221084808F080FC236843F4007323603B
:10E6900010BD0028F8D1236823F40073F7E700BF0A
:10E6A000003C024035D70108024A136843F4006376
:10E6B00013607047003C0240044B1A69002A04DAD8
:10E6C000034A5A6002F188325A607047003C0240A7
:10E6D00023016745024A136943F000431361704701
:10E6E000003C0240044B5A69D20704D5034A9A60A1
:10E6F00002F144329A607047003C02403B2A1908FC
:10E70000024A536943F0010353617047003C0240E1
:10E7100010F0F30F10B5044604D040F21F31054845
:10E7200008F032FC044B586920F00C00204358617B
:10E7300010BD00BF35D70108003C0240054B5869A9
:10E7400020F07F5020F47F1020F47C5020F00F0048
:10E75000704700BF003C0240024B586900F47F0044
:10E76000704700BF003C0240064B5869C0F30720C9
:10E77000AA2806D05B69C3F30723CC2B0CBFCC209F
:10E7800055207047003C0240024B586900F00C00D5
:10E79000704700BF003C024030F0407370B5054642
:10E7A0000E4600D120B940F2BA310A4808F0ECFB1D
:10E7B000012E094C08D940F2BB31064808F0E4FBB1
:10E7C00023691D43256170BD002EF9D1236923EA19
:10E7D0000505F7E735D70108003C0240421E1F2A15
:10E7E00010B5044608D9402810D10B4BDB682342F2
:10E7F00014BF0120002010BD084BD340DB07F4D428
:10E8000040F2DA31064808F0BFFBEEE78028ECD092
:10E81000B0F5803FE9D0F3E7003C02400380008080
:10E8200035D7010820F4F97323F0010310B504462D
:10E8300003B920B940F2F731024808F0A5FB024BBA
:10E84000DC6010BD35D70108003C02400E4BDA6891
:10E85000D20310D4DA68D1060FD4DA6812060ED4C7
:10E86000DA6812F0E00F0CD1DB6813F0020F14BF6E
:10E8700007200820704701207047052070470220BC
:10E8800070470620704700BF003C0240082307B5D0
:10E890008DF80730FFF7DAFF8DF807009DF8073095
:10E8A000012BF7D09DF8070003B05DF804FB0000D2
:10E8B000072870B506460D4604D94FF48F712348DA
:10E8C00008F062FB032D32D94FF4407540F21F115E
:10E8D0001E4808F059FBFFF7D9FF082826D11C4C29
:10E8E000236923F44073236123691D432561236950
:10E8F00023F0F8032361F82393FAA3F3B3FA83F325
:10E9000022699E40164346F002062661236943F4BD
:10E9100080332361FFF7BAFF236923F002032361E9
:10E92000236923F0F8032361BFF34F8F70BD002DDF
:10E93000D1D0012D06D0022D0CBF4FF400754FF43D
:10E940004075C8E74FF48075C5E700BF35D70108AB
:10E95000003C024038B50446FFF798FF0546032CFB
:10E9600021D940F26711174808F00EFB4FF44073AD
:10E97000082D16D1144C226922F4407222612269BA
:10E9800013432361236943F004032361236943F4A0
:10E9900080332361FFF77AFF2369054623F00403E0
:10E9A0002361284638BD44B1012C08D0022C0CBF8D
:10E9B0004FF400734FF44073DAE72346D8E74FF47F
:10E9C0008073D5E735D70108003C0240F8B51F46F3
:10E9D00000F1784305461646B3F5001F04D34FF403
:10E9E000CE710E4808F0D0FAFFF750FF082814D176
:10E9F0000B4C236923F440732361236943F4407370
:10EA00002361236943F001032361C5E90067FFF730
:10EA10003DFF236923F001032361F8BD35D70108C9
:10EA2000003C024000F17843B3F5001F70B5054685
:10EA30000E4604D340F2C7110D4808F0A5FAFFF7BF
:10EA400025FF082813D10B4C236923F4407323615D
:10EA5000236943F400732361236943F001032361B5
:10EA60002E60FFF713FF236923F00103236170BDBC
:10EA700035D70108003C024000F17843B3F5001F90
:10EA800070B505460E4604D340F2F1110D4808F06A
:10EA90007BFAFFF7FBFE082813D10B4C236923F404
:10EAA00040732361236943F480732361236943F036
:10EAB000010323612E80FFF7E9FE236923F00103A0
:10EAC000236170BD35D70108003C024000F1784356
:10EAD000B3F5001F70B505460E4604D340F21B2166
:10EAE0000C4808F051FAFFF7D1FE082811D10A4C62
:10EAF000236923F44073236123692361236943F06D
:10EB0000010323612E70FFF7C1FE236923F0010387
:10EB1000236170BD35D70108003C024038B530F4A0
:10EB20007F0304460D4600D120B940F2A5210B48D1
:10EB300008F02AFA012D04D940F2A621074808F06E
:10EB400023FAFFF7A3FE082805D1054B5A691DB12A
:10EB500022EA04045C6138BD1443FBE735D70108A1
:10EB6000003C0240AA2810B5044606D0552804D01F
:10EB700040F2CB21074808F007FAFFF787FE082884
:10EB800006D1054B586920F47F4040EA04205861C3
:10EB900010BD00BF35D70108003C02402DE9F84305
:10EBA0001F4630F0100304460D461646DDE908897D
:10EBB00004D04FF43F71204808F0E6F935F0200307
:10EBC00004D040F2FD211C4808F0DEF936F0400385
:10EBD00004D040F2FE21184808F0D6F937F080033F
:10EBE00004D040F2FF21144808F0CEF938F08043F9
:10EBF00004D04FF44071104808F0C6F939F0804352
:10EC000004D040F201310C4808F0BEF9FFF73EFE97
:10EC100008280ED1094A536923F0404323F0F0033A
:10EC200043EA090040EA08003843304328432043C0
:10EC30005061BDE8F88300BF35D70108003C0240B1
:10EC400038B531F0400305460C4612D0802910D06B
:10EC5000B1F5005F0DD021F00403B3F5004F08D0EB
:10EC600048F21303994204D040F23D310E4808F0B7
:10EC70008BF9102D06D0202D04D040F23E310A48E9
:10EC800008F082F9FFF702FE08280BD1074A102D81
:10EC900093690BBF1B0C9BB21B0443EA044408BFDF
:10ECA0001C43946138BD00BF35D70108003C0240C9
:10ECB000034A536943F002035361FFF7E7BD00BF06
:10ECC000003C024008B5434B98422DD003F58063C9
:10ECD00098423CD003F5806398423FD003F58063AF
:10ECE000984242D003F58063984245D003F5806393
:10ECF000984248D003F5806398424BD003F5806377
:10ED000098424ED003F58063984251D003F580635A
:10ED1000984256D003F5806398420FD031212E4897
:10ED2000BDE8084008F030B90121084602F020FB98
:10ED300000210120BDE8084002F01ABB01214FF478
:10ED4000806002F015FB00214FF48060F2E70121A2
:10ED5000022002F00DFB00210220EBE7012104203C
:10ED600002F006FB00210420E4E70121082002F064
:10ED7000FFFA00210820DDE70121102002F0F8FA57
:10ED800000211020D6E70121202002F0F1FA002115
:10ED90002020CFE70121402002F0EAFA00214020A4
:10EDA000C8E70121802002F0E3FA00218020C1E7BA
:10EDB00001214FF4807002F0DBFA00214FF48070E3
:10EDC000B8E701214FF4007002F0D2FA00214FF4AD
:10EDD0000070AFE70000024074D701082DE9F84F3A
:10EDE0004C4B04460D4698422BD003F58063984265
:10EDF00027D003F58063984223D003F580639842BF
:10EE00001FD003F5806398421BD003F580639842BE
:10EE100017D003F58063984213D003F580639842BE
:10EE20000FD003F5806398420BD003F580639842BE
:10EE300007D003F58063984203D07F21364808F05D
:10EE4000A3F82B881BB98021334808F09DF82B7953
:10EE5000032B03D98121304808F096F8EB79022B77
:10EE600003D982212C4808F08FF8002601274FF0A3
:10EE70000308DFF8A49007FA06F32A68934343D106
:10EE80004FEA460A236808FA0AFB6FEA0B0B03EA0B
:10EE90000B0323602B79216803FA0AF2013B0A4332
:10EEA000012B226023D86B79032B03D99421484688
:10EEB00008F06AF8A3680BEA0303A3606B79A26801
:10EEC00003FA0AF31343A360AB79012B03D99B2107
:10EED000484608F059F8636807FA06F223EA020385
:10EEE0006360AB796268B3409BB213436360E368CD
:10EEF00008FA0AF223EA0203E360EB79E26803FA14
:10EF00000AFA4AEA0202E2600136102EB3D1BDE8E5
:10EF1000F88F00BF0000024074D701084FF6FF725F
:10EF20000023C0E9002370474FF4803337B50193C5
:10EF30000446214B0D4698422BD003F5806398423E
:10EF400027D003F58063984223D003F5806398426D
:10EF50001FD003F5806398421BD003F5806398426D
:10EF600017D003F58063984213D003F5806398426D
:10EF70000FD003F5806398420BD003F5806398426D
:10EF800007D003F58063984203D0CA210B4807F0ED
:10EF9000FBFF1DB9CB21094807F0F6FF019B2B436E
:10EFA0000193019BE361E561019BE361E3690193E7
:10EFB000E369019303B030BD0000024074D701083B
:10EFC00038B5314B05460C4698422BD003F580638B
:10EFD000984227D003F58063984223D003F58063DD
:10EFE00098421FD003F5806398421BD003F58063DD
:10EFF000984217D003F58063984213D003F58063DD
:10F0000098420FD003F5806398420BD003F58063DC
:10F01000984207D003F58063984203D0F9211B483A
:10F0200007F0B2FF631E9BB21F2B07D9402C0FD1F4
:10F030002B691C4214BF0120002038BD144A22FA5B
:10F0400003F3DB07F4D4FA21104807F09DFFEFE744
:10F05000802CEDD0B4F5807FEAD0B4F5007FE7D006
:10F06000B4F5806FE4D0B4F5006FE1D0B4F5805F03
:10F07000DED0B4F5005FDBD0B4F5804FD8D0B4F566
:10F08000004FD5D0DFE700BF0000024074D7010871
:10F090008B8000801A4B984210B504462CD003F5A3
:10F0A0008063984228D003F58063984224D003F50A
:10F0B0008063984220D003F5806398421CD003F50A
:10F0C0008063984218D003F58063984214D003F50A
:10F0D0008063984210D003F5806398420CD003F50A
:10F0E0008063984208D003F58063984204D040F2D0
:10F0F0001111044807F048FF206980B210BD00BF1D
:10F100000000024074D7010838B5324B05460C4662
:10F1100098422CD003F58063984228D003F5806391
:10F12000984224D003F58063984220D003F5806391
:10F1300098421CD003F58063984218D003F5806391
:10F14000984214D003F58063984210D003F5806391
:10F1500098420CD003F58063984208D003F5806391
:10F16000984204D04FF492711B4807F00DFF631EC4
:10F170009BB21F2B07D9402C10D16B691C4214BFC6
:10F180000120002038BD154A22FA03F3DB07F4D42E
:10F1900040F22511104807F0F7FEEEE7802CECD086
:10F1A000B4F5807FE9D0B4F5007FE6D0B4F5806F88
:10F1B000E3D0B4F5006FE0D0B4F5805FDDD0B4F5F6
:10F1C000005FDAD0B4F5804FD7D0B4F5004FD4D07B
:10F1D000DEE700BF0000024074D701088B8000808A
:10F1E0001A4B984210B504462CD003F58063984220
:10F1F00028D003F58063984224D003F580639842B9
:10F2000020D003F5806398421CD003F580639842B8
:10F2100018D003F58063984214D003F580639842B8
:10F2200010D003F5806398420CD003F580639842B8
:10F2300008D003F58063984204D04FF49E710448CF
:10F2400007F0A2FE606980B210BD00BF000002405E
:10F2500074D7010838B51D4B04460D4698422CD092
:10F2600003F58063984228D003F58063984224D048
:10F2700003F58063984220D003F5806398421CD048
:10F2800003F58063984218D003F58063984214D048
:10F2900003F58063984210D003F5806398420CD048
:10F2A00003F58063984208D003F58063984204D048
:10F2B00040F25111064807F067FE25B94FF4A971D5
:10F2C000034807F061FEA56138BD00BF00000240A1
:10F2D00074D7010838B51D4B04460D4698422CD012
:10F2E00003F58063984228D003F58063984224D0C8
:10F2F00003F58063984220D003F5806398421CD0C8
:10F3000003F58063984218D003F58063984214D0C7
:10F3100003F58063984210D003F5806398420CD0C7
:10F3200003F58063984208D003F58063984204D0C7
:10F330004FF4B371064807F027FE25B940F2671174
:10F34000034807F021FE2D04A56138BD00000240EE
:10F3500074D70108364B984270B505460C461646E0
:10F360002CD003F58063984228D003F5806398423F
:10F3700024D003F58063984220D003F5806398423F
:10F380001CD003F58063984218D003F5806398423F
:10F3900014D003F58063984210D003F5806398423F
:10F3A0000CD003F58063984208D003F5806398423F
:10F3B00004D04FF4BE711F4807F0E6FD631E9BB2F8
:10F3C0001F2B0AD9402C13D1012E2CD94FF4BF7119
:10F3D000184807F0D9FDAC6170BD174A22FA03F353
:10F3E000DB07F1D440F27D11124807F0CDFDEBE7C9
:10F3F000802CE9D0B4F5807FE6D0B4F5007FE3D06F
:10F40000B4F5806FE0D0B4F5006FDDD0B4F5805F67
:10F41000DAD0B4F5005FD7D0B4F5804FD4D0B4F5CE
:10F42000004FD1D0DEE7002ED5D12404D3E700BFB2
:10F430000000024074D701088B80008038B51A4B59
:10F4400004460D4698422CD003F58063984228D09C
:10F4500003F58063984224D003F58063984220D05E
:10F4600003F5806398421CD003F58063984218D05E
:10F4700003F58063984214D003F58063984210D05E
:10F4800003F5806398420CD003F58063984208D05E
:10F4900003F58063984204D040F29511034807F0C9
:10F4A00073FD656138BD00BF0000024074D70108DC
:10F4B00038B51B4B04460D4698422CD003F58063AB
:10F4C000984228D003F58063984224D003F58063E6
:10F4D000984220D003F5806398421CD003F58063E6
:10F4E000984218D003F58063984214D003F58063E6
:10F4F000984210D003F5806398420CD003F58063E6
:10F50000984208D003F58063984204D040F2A511D8
:10F51000044807F039FD63695D40656138BD00BF8F
:10F520000000024074D70108294B984270B5044688
:10F530000E4615462CD003F58063984228D003F57B
:10F540008063984224D003F58063984220D003F56D
:10F55000806398421CD003F58063984218D003F56D
:10F560008063984214D003F58063984210D003F56D
:10F57000806398420CD003F58063984208D003F56D
:10F580008063984204D040F20521124807F0FCFC49
:10F590000F2E04D940F206210E4807F0F5FC0F2D7E
:10F5A00004D940F207210B4807F0EEFC06F00703F0
:10F5B000F6080F2104EB86049B00226A99409D40C7
:10F5C00022EA01022262226A1543256270BD00BF51
:10F5D0000000024074D7010808B5114B984211D0C1
:10F5E00003F58063984219D003F58063984215D0E3
:10F5F00003F58063984211D048210A48BDE80840CD
:10F6000007F0C2BC01214FF4001001F019FF0021E6
:10F610004FF40010BDE8084001F012BF08BD00BF64
:10F6200000540040B2D7010838B53A4B04460D46A5
:10F6300098420FD003F5806398420BD003F58063A6
:10F64000984207D003F58063984203D06121324885
:10F6500007F09AFC6B6833F4805303D062212E4884
:10F6600007F092FCAB680F2B03D963212A4807F0FF
:10F670008BFCEB6833F4801206D0B3F5001F03D087
:10F680006421254807F080FC2B69B3F5806F03D314
:10F690006521214807F078FC6B6933F4004303D0FF
:10F6A00066211D4807F070FCAB6933F4806303D01A
:10F6B0006721194807F068FC2368184A23F0010302
:10F6C000236023681A40D5E9013143EA012313433B
:10F6D0002A6923602B6823F070632361236843F059
:10F6E000010323600023A360E360AB691343EA686E
:10F6F000A360A36843F40043A360236813436A69CB
:10F700002360636823F0784323F40043134363606A
:10F7100038BD00BF00540040B2D70108FFE0CF0061
:10F7200000234FF40042C0E90033C0E90233036113
:10F73000C0E905237047000038B5134B04460D4659
:10F7400098420FD003F5806398420BD003F5806395
:10F75000984207D003F58063984203D0C8210B4834
:10F7600007F012FC012D08D9C921084807F00CFC4C
:10F77000236843F00103236038BD002DF8D12368CE
:10F7800023F00103F7E700BF00540040B2D701089F
:10F790000F4B984210B504460FD003F58063984292
:10F7A0000BD003F58063984207D003F5806398423D
:10F7B00003D0DF21074807F0E7FB236823F00103AC
:10F7C00023602368236843F00103236010BD00BF5A
:10F7D00000540040B2D70108174B984270B5044658
:10F7E0000D4616460FD003F5806398420BD003F503
:10F7F0008063984207D003F58063984203D0FF21CD
:10F800000E4807F0C1FB012E04D94FF480710B485C
:10F8100007F0BAFB35F0FE0300D125B940F2011123
:10F82000064807F0B1FB236816B11D43256070BD83
:10F8300023EA0505FAE700BF00540040B2D70108EB
:10F8400038B5144B04460D46984210D003F580633A
:10F8500098420CD003F58063984208D003F580638A
:10F86000984204D040F219110B4807F08DFB012D8E
:10F8700009D94FF48D71084807F086FB236823F4FB
:10F880000033236038BD002DF8D1236843F40033E2
:10F89000F7E700BF00540040B2D7010838B5144B59
:10F8A00004460D46984210D003F5806398420CD070
:10F8B00003F58063984208D003F58063984204D032
:10F8C0004FF499710B4807F05FFB012D09D940F205
:10F8D0003311084807F058FBE36843F40043E36042
:10F8E00038BD002DF8D1E36823F40043F7E700BFEB
:10F8F00000540040B2D70108194B984270B5054634
:10F900000E46144610D003F5806398420CD003F5E0
:10F910008063984208D003F58063984204D04FF486
:10F92000AB71104807F030FBFF2E04D940F257119D
:10F930000C4807F029FB072C04D94FF4AC71094897
:10F9400007F022FBEB68240206F0FE0623F4FF63B7
:10F9500004F4E06423F0060334431C43EC6070BD00
:10F9600000540040B2D7010838B5144B04460D4688
:10F97000984210D003F5806398420CD003F5806361
:10F98000984208D003F58063984204D04FF4B971CF
:10F990000B4807F0F9FA012D09D940F27311084814
:10F9A00007F0F2FA236843F40023236038BD002DEA
:10F9B000F8D1236823F40023F7E700BF0054004088
:10F9C000B2D7010838B5144B04460D46984210D002
:10F9D00003F5806398420CD003F58063984208D009
:10F9E00003F58063984204D040F28B110B4807F076
:10F9F000CBFA012D09D94FF4C671084807F0C4FAB3
:10FA0000236843F48033236038BD002DF8D1236888
:10FA100023F48033F7E700BF00540040B2D7010859
:10FA200038B5144B04460D46984210D003F5806358
:10FA300098420CD003F58063984208D003F58063A8
:10FA4000984204D04FF4D3710B4807F09DFAB5F5F6
:10FA5000806F04D340F2A711074807F095FA636856
:10FA6000C5F3090523F47F7323F003031D43656089
:10FA700038BD00BF00540040B2D7010838B5144B60
:10FA800004460D46984210D003F5806398420CD08E
:10FA900003F58063984208D003F58063984204D050
:10FAA00040F2C1110B4807F06FFA012D09D94FF44C
:10FAB000E171084807F068FA636843F40063636023
:10FAC00038BD002DF8D1636823F40063F7E700BF69
:10FAD00000540040B2D7010838B5144B04460D4617
:10FAE000984210D003F5806398420CD003F58063F0
:10FAF000984208D003F58063984204D040F2022176
:10FB00000B4807F041FA012D09D940F203210848BA
:10FB100007F03AFA636843F00073636038BD002D64
:10FB2000F8D1636823F00073F7E700BF005400408A
:10FB3000B2D7010838B5144B04460D46984210D090
:10FB400003F5806398420CD003F58063984208D097
:10FB500003F58063984204D040F21B210B4807F064
:10FB600013FA012D09D94FF40771084807F00CFA70
:10FB7000636843F08073636038BD002DF8D163681B
:10FB800023F08073F7E700BF00540040B2D70108AC
:10FB900038B50E4B04460D46984210D003F58063ED
:10FBA00098420CD003F58063984208D003F5806337
:10FBB000984204D040F23521054807F0E5F9616824
:10FBC00021F47F0141EA0541616038BD00540040E5
:10FBD000B2D7010838B5144B04460D46984210D0F0
:10FBE00003F5806398420CD003F58063984208D0F7
:10FBF00003F58063984204D04FF414710B4807F06A
:10FC0000C3F95DB1B5F5806F04D040F251210748CA
:10FC100007F0BAF9636843F4806302E0636823F491
:10FC20008063636038BD00BF00540040B2D7010854
:10FC300038B5144B04460D46984210D003F5806346
:10FC400098420CD003F58063984208D003F5806396
:10FC5000984204D040F26A210B4807F095F9012D33
:10FC600009D940F26B21084807F08EF9636843F424
:10FC70000053636038BD002DF8D1636823F400534E
:10FC8000F7E700BF00540040B2D7010838B5144B65
:10FC900004460D46984210D003F5806398420CD07C
:10FCA00003F58063984208D003F58063984204D03E
:10FCB00040F283210B4807F067F9012D09D94FF471
:10FCC0002171084807F060F9636843F4804363607A
:10FCD00038BD002DF8D1636823F48043F7E700BFF7
:10FCE00000540040B2D7010838B5144B04460D4605
:10FCF000984210D003F5806398420CD003F58063DE
:10FD0000984208D003F58063984204D040F29E21C7
:10FD10000B4807F039F9012D09D940F29F21084815
:10FD200007F032F9636843F48053636038BD002DF7
:10FD3000F8D1636823F48053F7E700BF0054004014
:10FD4000B2D7010838B5144B04460D46984210D07E
:10FD500003F5806398420CD003F58063984208D085
:10FD600003F58063984204D040F2B7210B4807F0B6
:10FD70000BF9012D09D94FF42E71084807F004F949
:10FD8000636823F40043636038BD002DF8D16368D5
:10FD900043F40043F7E700BF00540040B2D7010826
:10FDA0000D4B984210B5044610D003F5806398427D
:10FDB0000CD003F58063984208D003F58063984225
:10FDC00004D040F2CE21054807F0DEF8A069000C0F
:10FDD00000F0FE0010BD00BF00540040B2D7010883
:10FDE0000E4B984210B5044610D003F5806398423C
:10FDF0000CD003F58063984208D003F580639842E5
:10FE000004D040F2DF21064807F0BEF8A36913F4DE
:10FE1000803F14BF4FF48060002010BD00540040AC
:10FE2000B2D701082DE9F0411C46264B05460E4687
:10FE300098429046069F10D003F5806398420CD0FC
:10FE400003F58063984208D003F58063984204D09C
:10FE500040F20A311C4807F097F8B6F5806F04D3DA
:10FE600040F20B31184807F08FF8B4F1007F07D04B
:10FE700034F0807304D04FF44371134807F084F8D2
:10FE8000B7F5804F0AD0B7F5105F07D037F40053AD
:10FE900004D040F20D310C4807F076F86B6844EA64
:10FEA0000844C6F3090623F07F733C4323F4593317
:10FEB000344323F47F7323F003031C436C60BDE8D9
:10FEC000F08100BF00540040B2D7010838B5144B90
:10FED00004460D46984210D003F5806398420CD03A
:10FEE00003F58063984208D003F58063984204D0FC
:10FEF00040F24F310B4807F047F8012D09D94FF474
:10FF00005471084807F040F8236843F480032360E5
:10FF100038BD002DF8D1236823F48003F7E700BF34
:10FF200000540040B2D7010838B5144B04460D46C2
:10FF3000984210D003F5806398420CD003F580639B
:10FF4000984208D003F58063984204D04FF45A7168
:10FF50000B4807F019F8012D09D940F2693108481A
:10FF600007F012F8636943F40043636138BD002D64
:10FF7000F8D1636923F40043F7E700BF0054004061
:10FF8000B2D7010838B5144B04460D46984210D03C
:10FF900003F5806398420CD003F58063984208D043
:10FFA00003F58063984204D040F281310B4806F09B
:10FFB000EBFF012D09D940F28231084806F0E4FF39
:10FFC000636943F00043636138BD002DF8D1636974
:10FFD00023F00043F7E700BF00540040B2D7010808
:10FFE00038B5144B04460D46984210D003F5806393
:10FFF00098420CD003F58063984208D003F58063E3
:020000040801F1
:10000000984204D040F29B310B4806F0BDFF012D11
:1000100009D94FF46771084806F0B6FF636943F4E5
:100020008053636138BD002DF8D1636923F4805398
:10003000F7E700BF00540040B2D7010838B5144BB1
:1000400004460D46984210D003F5806398420CD0C8
:1000500003F58063984208D003F58063984204D08A
:1000600040F2B6310B4806F08FFFB5F5805F04D340
:1000700040F2B731074806F087FF6369C5F30B0507
:1000800023F47F6323F00F031D43656138BD00BF78
:1000900000540040B2D7010838B5144B04460D4651
:1000A000984210D003F5806398420CD003F580632A
:1000B000984208D003F58063984204D040F2D131D1
:1000C0000B4806F061FFB5F5805F04D340F2D231F2
:1000D000074806F059FF6369064923F07F6301EA88
:1000E000054123F470231943616138BD0054004079
:1000F000B2D701080000FF0F38B5144B04460D4677
:10010000984210D003F5806398420CD003F58063C9
:10011000984208D003F58063984204D040F2EB3156
:100120000B4806F031FF012D09D94FF47B710848C7
:1001300006F02AFF236843F40003236038BD002D36
:10014000F8D1236823F40003F7E700BF0054004010
:10015000B2D7010838B5144B04460D46984210D06A
:1001600003F5806398420CD003F58063984208D071
:1001700003F58063984204D040F204410B4806F036
:1001800003FF012D09D940F20541084806F0FCFEA5
:10019000236843F08063236038BD002DF8D12368C5
:1001A00023F08063F7E700BF00540040B2D7010896
:1001B0000C4B984210B5044610D003F5806398426A
:1001C0000CD003F58063984208D003F58063984211
:1001D00004D040F21B41044806F0D6FE206AC0B2AB
:1001E00010BD00BF00540040B2D70108002337B54E
:1001F00001930546184B0C46984210D003F58063D6
:1002000098420CD003F58063984208D003F58063D0
:10021000984204D040F24B41104806F0B5FE1C2C29
:100220000BD904F0FB03202B12D10195019B1C4438
:100230000194019B186803B030BD4FF01133E340C7
:10024000DB07F2D440F24C41044806F09DFEECE797
:10025000282CEAD0F6E700BF00540040B2D70108CE
:1002600038B50C4B04460D46984210D003F5806318
:1002700098420CD003F58063984208D003F5806360
:10028000984204D040F27441034806F07DFEA56216
:1002900038BD00BF00540040B2D701080C4B984253
:1002A00010B5044610D003F5806398420CD003F5D6
:1002B0008063984208D003F58063984204D040F2EE
:1002C0008241044806F060FE606AC0B210BD00BF03
:1002D00000540040B2D70108174B984270B504464D
:1002E0000D46164610D003F5806398420CD003F5F6
:1002F0008063984208D003F58063984204D040F2AE
:10030000AD410E4806F040FE012E04D940F2AE4148
:100310000A4806F039FE35F4404300D125B940F2D1
:10032000AF41064806F030FE236816B11D43256034
:1003300070BD23EA0505FAE700540040B2D7010872
:1003400038B5214B05460C46984210D003F5806322
:1003500098420CD003F58063984208D003F580637F
:10036000984204D04FF4A561184806F00DFE621EB5
:100370001F2A07D9402C0FD1AB691C4214BF0120A2
:10038000002038BD124BD340DB07F5D440F2295191
:100390000E4806F0F9FDEFE7802CEDD0B4F5807F34
:1003A000EAD0B4F5007FE7D0B4F5806FE4D0B4F5BF
:1003B000006FE1D0B4F5805FDED0B4F5005FDBD034
:1003C000B4F5004FD8D0E1E700540040B2D701089F
:1003D0008B80008038B5114B04460D46984210D0F2
:1003E00003F5806398420CD003F58063984208D0EF
:1003F00003F58063984204D040F25151084806F05A
:10040000C3FD25F43F4323F0FF0303B925B940F2B0
:100410005251034806F0B8FDE56138BD0054004074
:10042000B2D7010838B5284B05460C46984210D083
:1004300003F5806398420CD003F58063984208D09E
:1004400003F58063984204D040F273511F4806F0D0
:100450009BFDA21E1E2A05D9402C15D12B6803F046
:10046000400319E01A4BD340DB070AD440F2745121
:10047000164806F089FD14F47C5F0AD114F0C00F11
:10048000ECD12B68234007E0802CE7D0B4F5807FC7
:1004900009D12B6803F08003A869204002D0181C02
:1004A00018BF012038BDB4F5007FF2D0B4F5806FDD
:1004B000EFD0B4F5006FECD0B4F5805FE9D0B4F5BF
:1004C000005FE6D0D2E700BF00540040B2D7010879
:1004D0004540004038B5114B04460D46984210D0B7
:1004E00003F5806398420CD003F58063984208D0EE
:1004F00003F58063984204D040F2AF51084806F0FB
:1005000043FD25F47F5323F03E0303B925B94FF48F
:10051000B661034806F038FDE56138BD005400407F
:10052000B2D7010808B501214FF0805000F088FFD4
:1005300000214FF08050BDE8084000F081BF00006E
:10054000012810B5084C08D94F21084806F01CFDB9
:10055000236843F48073236010BD0028F8D123681A
:1005600023F48073F7E700BF00700040EFD7010865
:1005700030F0600310B5044605D0802B03D08821ED
:10058000044806F001FD044A136803F0E0031C432D
:10059000146010BDEFD7010800700040012810B5AD
:1005A000084C08D99F21084806F0EEFC236843F068
:1005B0001003236010BD0028F8D1236823F0100336
:1005C000F7E700BF00700040EFD70108012970B5C0
:1005D00004460E4600F47C5511D9DF211E4806F072
:1005E000D3FCB4F5807F0DD11C4AD3682B43D36074
:1005F000936823EA050343EA9414946070BDB0F550
:10060000807F04D024F40043B3F5007F07D1002E8F
:10061000EAD1124BDC6824EA0504DC60EEE724F43E
:100620008033B3F5806FF2D024F40033B3F5006F5C
:10063000EDD024F48023B3F5805FE8D024F40023C8
:10064000B3F5005FE3D0B4F5824FE0D0E02102487B
:1006500006F09AFCDBE700BFEFD70108007000400E
:10066000012810B5084C09D940F24D11074806F091
:100670008BFC636843F40073636010BD0028F8D1FD
:10068000636823F40073F7E700700040EFD70108B8
:10069000B0F5004F10B5044609D020F40043B3F57F
:1006A000804F04D040F27111044806F06DFC044AFA
:1006B000136803F440431C43146010BDEFD70108D6
:1006C00000700040012810B5084C09D940F2911182
:1006D000074806F059FC236843F48033236010BDBB
:1006E0000028F8D1236823F48033F7E70070004036
:1006F000EFD70108012810B5084C09D94FF4D6717D
:10070000074806F041FC236843F40033236010BD22
:100710000028F8D1236823F40033F7E70070004085
:10072000EFD70108012810B5084C09D94FF4E8713A
:10073000074806F029FC236843F44023236010BDDA
:100740000028F8D1236823F44023F7E70070004025
:10075000EFD70108012810B5084C09D94FF4F571FD
:10076000074806F011FC236843F40063236010BDC2
:100770000028F8D1236823F40063F7E700700040F5
:10078000EFD70108012810B5084C09D940F2022121
:10079000074806F0F9FB236843F48063236010BD2B
:1007A0000028F8D1236823F48063F7E70070004045
:1007B000EFD70108012810B5084C09D94FF40B7187
:1007C000074806F0E1FB236843F40073236010BD83
:1007D0000028F8D1236823F40073F7E70070004085
:1007E000EFD70108012838B504460D4604D940F278
:1007F000C721114806F0C8FB6B1E012B04D94FF42A
:1008000032710D4806F0C0FB0C4B012D186820F426
:10081000406020F0030040EA04001860084B1A69A9
:1008200042F004021A6105D130BF1A6922F00402B5
:100830001A6138BD20BFF8E7EFD70108007000400B
:1008400000ED00E0B0F5006F38B504460D4608D065
:1008500040F20143984204D040F20731114806F0BB
:1008600093FB6B1E012B04D94FF442710D4806F027
:100870008BFB0D4A012D136823F4406323F003031F
:1008800044EA0304094B14601A6942F004021A6135
:1008900005D130BF1A6922F004021A6138BD20BFA9
:1008A000F8E700BFEFD701080070004000ED00E05E
:1008B000054A136843F002031360044A136943F0C6
:1008C0000403136130BF70470070004000ED00E08A
:1008D00000F10043013B012B10B5044627D900F17C
:1008E0000043043B1C2B0BD9082816D9B4F5804FC4
:1008F00020D1154B5B68234214BF012000200BE080
:10090000124A22FA03F3DA07F0D50F4BD8682040D9
:1009100010F03F0018BF012010BD4FF48A73C34090
:10092000DB07E6D440F27531094806F02DFB002CB8
:10093000DFDAEAE7B4F5803FDBD0B4F5003FD8D08A
:10094000B4F5402FD5D0EDE7007000401110001035
:10095000EFD7010800F10043013B012B10B504461D
:100960000ED900F10043043B1C2B14D902281ED0E1
:10097000B0F5402F09D040F2A331104806F004FB37
:10098000002C0DDBB4F5402F11D10D4A536843F410
:10099000402353600AE00B4A22FA03F3DB07EAD54F
:1009A000074B04F03F049A6814439C6010BD044A4E
:1009B000136843EA84041460F8E700BFEFD7010826
:1009C0000070004011100010174B1A6842F08102AD
:1009D0001A6000229A60196821F0A16121F4803127
:1009E00019605A601149586801435960C3F884205E
:1009F000D3F8841041F0005141F44051C3F8841001
:100A0000C3F88820D3F8881041F0105141F44051C8
:100A1000C3F88810196821F480211960DA60C3F8DE
:100A20008C20C3F89020704700380240103000043A
:100A3000012810B5044605D9052803D0D221044861
:100A400006F0A2FA034B00221A701C7010BD00BF02
:100A50003CD80108023802401F2810B5044604D9CA
:100A60004FF48571074806F08FFA0749F8230A68A2
:100A700022F0F80293FAA3F3B3FA83F39C401443F1
:100A80000C6010BD3CD8010800380240012810B5A8
:100A9000084C09D940F22D11074806F075FA236871
:100AA00043F00103236010BD0028F8D1236823F030
:100AB0000103F7E7003802403CD80108012810B5CF
:100AC000044606D9042804D040F24D110A4806F025
:100AD0005BFA0A4B012C1A6F22F005021A6702D04A
:100AE000042C05D010BD1A6F42F001021A67F9E715
:100AF0001A6F42F00502F9E73CD8010800380240BD
:100B0000012810B5084C09D940F27111074806F0C8
:100B10003BFA636F43F00103636710BD0028F8D10F
:100B2000636F23F00103F7E7003802403CD8010867
:100B30002DE9F0411D4630F48003074688461646ED
:100B4000069C04D040F2A711264806F01DFAA8F131
:100B500002033D2B04D94FF4D471224806F014FA55
:100B6000A6F1C003F02B04D940F2A9111D4806F0EC
:100B70000BFA082D04D84FF4AA73EB40DB0704D41A
:100B80004FF4D571174806F0FFF9A31E0D2B04D9B9
:100B900040F2AB11134806F0F7F947F6C07292FA2B
:100BA000A2F24FF44031B2FA82F291FAA1F14FF081
:100BB0007063B1FA81F193FAA3F3B3FA83F36D088A
:100BC00006FA02F204FA03F3013D43EA08038D40FA
:100BD0003B431343044A2B4343F000535360BDE8A7
:100BE000F08100BF3CD8010800380240012810B550
:100BF000084C09D940F2C111074806F0C5F923682D
:100C000043F08073236010BD0028F8D1236823F0DF
:100C10008073F7E7003802403CD80108F8B51C465D
:100C2000A0F1310306460D46B3F5C07F174604D345
:100C30004FF4F671134806F0A7F9AB1E062B04D942
:100C400040F2ED110F4806F09FF9BB1E0D2B04D9A1
:100C50004FF4F7710B4806F097F9A31E052B04D942
:100C600040F2EF11074806F08FF92407064B6D0894
:100C700044EA0764013D44EA861444EA0544C3F8A3
:100C80008440F8BD3CD8010800380240012810B566
:100C9000084C09D940F2FD11074806F075F92368A0
:100CA00043F08063236010BD0028F8D1236823F04F
:100CB0008063F7E7003802403CD80108F8B51C46CD
:100CC000A0F1310306460D46B3F5C07F174604D3A5
:100CD00040F22621134806F057F9AB1E062B04D923
:100CE00040F227210F4806F04FF9BB1E0D2B04D907
:100CF0004FF40A710B4806F047F9A31E052B04D9DF
:100D000040F22921074806F03FF92407064B6D08F9
:100D100044EA0764013D44EA861444EA0544C3F802
:100D20008840F8BD3CD8010800380240012810B5C1
:100D3000084C09D940F23A21074806F025F9236802
:100D400043F08053236010BD0028F8D1236823F0BE
:100D50008053F7E7003802403CD80108012810B55D
:100D6000084C09D94FF41571074806F00DF92368AE
:100D700043F40023236010BD0028F8D1236823F436
:100D80000023F7E7003802403CD8010838B530F4BA
:100D9000C00304460D4604D040F277210D4806F00A
:100DA000F3F835F080630CD025F00073B3F1A06F39
:100DB00007D0B5F1C06F04D04FF41E71054806F09E
:100DC000E3F8054B996821F0EC61294321439960D0
:100DD00038BD00BF3CD801080038024038B530F0BB
:100DE000404304460D4604D040F29D210D4806F0D4
:100DF000CBF835F000530CD025F08053B3F1205FD1
:100E000007D0B5F1405F04D040F29E21054806F0BE
:100E1000BBF8054B996821F078412943214399603B
:100E200038BD00BF3CD8010800380240022810B588
:100E3000044604D940F2F921044806F0A5F8044A12
:100E4000936823F003031C43946010BD3CD8010851
:100E500000380240024B986800F00C00704700BF59
:100E60000038024030F0800310B5044612D020F064
:100E70002003902B0ED020F04003A02B0AD020F0AE
:100E80001003C02B06D0F02804D040F22E310548C4
:100E900006F07AF8044A936823F0F0031C43946048
:100EA00010BD00BF3CD801080038024030F4805328
:100EB00010B504460CD020F40063B3F5A05F07D052
:100EC000B0F5C05F04D040F24D31054806F05CF843
:100ED000044A936823F4E0531C43946010BD00BFA0
:100EE0003CD801080038024030F4805310B5044665
:100EF0000CD020F40063B3F5A05F07D0B0F5C05F5D
:100F000004D04FF45B71054806F03EF8044B986836
:100F100020F4604040EAC400986010BD3CD801084D
:100F2000003802401D4A936803F00C03042B10B5EF
:100F30001AD0082B1AD01A4B184A03609368194923
:100F4000C3F30313CC5C0368E34043609468C4F3C9
:100F500082240C5D23FA04F484609268C2F3423266
:100F60008A5CD340C36010BD0F4BE5E754685168FD
:100F70006302526801F03F0148BF0B4BC2F3881275
:100F800058BF074BB3FBF1F35343044A5268C2F313
:100F9000014201325200B3FBF2F3CDE700380240C8
:100FA0000024F4002CD8010800127A00B0F5807FEC
:100FB00010B5044613D0B0F5007F10D020F4A02166
:100FC0001F4B20F48032994210D11E4924F0704307
:100FD0008A6823F4407322F4F81213438B60194B90
:100FE000C4F30B041A6F14431C6710BD20F41021C6
:100FF000154B9942E9D020F4403314498B42E4D098
:1010000020F4881001F5C0218842DED001F50031BE
:101010008B42DAD001F580218B42D6D001F58021B8
:101020008B42D2D00A4B9A42CFD040F21E4109489F
:1010300005F0AAFF04F44073B3F5407FCFD1C4E7B5
:10104000000302000038024000030400000308000F
:1010500000031C003CD80108012810B5084C09D930
:1010600040F23C41074805F08FFF236F43F40043F3
:10107000236710BD0028F8D1236F23F40043F7E75E
:10108000003802403CD80108012810B5084C09D9A5
:1010900040F25441074805F077FF236F43F4803353
:1010A000236710BD0028F8D1236F23F48033F7E7BE
:1010B000003802403CD8010830F4000310B5044663
:1010C00004D040F26E41064805F05EFF054B9A6879
:1010D00022F400029A6098682043986010BD00BF17
:1010E0003CD801080038024031F4800370B5064650
:1010F0000D4607D0B1F5000F04D04FF491611248AE
:1011000005F042FF012E114C0FD940F289410E48E3
:1011100005F03AFFD4F88C3023F44003C4F88C3047
:10112000D4F88C3043EA85050AE0002EF2D1D4F8D9
:101130008C3023F44013C4F88C30D4F88C301D4329
:10114000C4F88C5070BD00BF3CD801080038024084
:1011500010B5441E1F2C04D940F2AB41054805F0E0
:1011600013FF054AD2F88C3023F01F031C43C2F84A
:101170008C4010BD3CD801080038024010B5441E18
:101180001F2C04D940F2C941064805F0FDFE064B6C
:10119000D3F88C0020F4F85040EA0420C3F88C0007
:1011A00010BD00BF3CD801080038024030F4403385
:1011B00010B5044604D040F2ED41064805F0E4FEC7
:1011C000054AD2F88C3023F440331C43C2F88C40DB
:1011D00010BD00BF3CD8010800380240012810B5FE
:1011E0000A4C0BD94FF4A261094805F0CDFED4F8A2
:1011F0008C3043F08073C4F88C3010BD0028F6D1D9
:10120000D4F88C3023F08073F5E700BF003802403B
:101210003CD801080E4B034070B505460E4603B995
:1012200020B940F241510B4805F0AEFE012E0A4CA8
:1012300008D940F24351074805F0A6FE236B1D4331
:10124000256370BD002EF9D1236B23EA0505F7E76E
:1012500000E80B813CD801080038024030F0F1036F
:1012600070B505460E4600D120B940F261510A48DA
:1012700005F08AFE012E094C08D940F26251064859
:1012800005F082FE636B1D43656370BD002EF9D1CE
:10129000636B23EA0505F7E73CD8010800380240F4
:1012A00030F0030370B505460E4600D120B940F278
:1012B0007E510A4805F068FE012E094C08D940F21B
:1012C0007F51064805F060FEA36B1D43A56370BD0A
:1012D000002EF9D1A36B23EA0505F7E73CD80108F6
:1012E0000038024010F4585F70B505460E4600D134
:1012F00020B940F2B5510A4805F046FE012E094CCE
:1013000008D940F2B651064805F03EFE236C1D4355
:10131000256470BD002EF9D1236C23EA0505F7E79B
:101320003CD80108003802400E4B034070B505461A
:101330000E4603B920B940F2E3510B4805F024FEF4
:10134000012E0A4C08D940F2E451074805F01CFE72
:10135000636C1D43656470BD002EF9D1636C23EA94
:101360000505F7E7CC8008F33CD8010800380240B7
:101370000E4B034070B505460E4603B920B940F246
:101380000D610B4805F000FE012E0A4C08D940F211
:101390000E61074805F0F8FD23691D43256170BD06
:1013A000002EF9D1236923EA0505F7E700E81FDDE0
:1013B0003CD801080038024030F0F10370B5054612
:1013C0000E4600D120B940F22A610A4805F0DCFD42
:1013D000012E094C08D940F22B61064805F0D4FDD6
:1013E00063691D43656170BD002EF9D1636923EA0D
:1013F0000505F7E73CD801080038024030F0030348
:1014000070B505460E4600D120B940F244610A4845
:1014100005F0BAFD012E094C08D940F24561064895
:1014200005F0B2FDA3691D43A56170BD002EF9D181
:10143000A36923EA0505F7E73CD801080038024014
:1014400010F4585F70B505460E4600D120B94FF430
:10145000CF610A4805F098FD012E094C08D940F2E9
:101460007961064805F090FD236A1D43256270BD31
:10147000002EF9D1236A23EA0505F7E73CD80108D5
:10148000003802400E4B034070B505460E4603B9C6
:1014900020B940F2A2610B4805F076FD012E0A4CFE
:1014A00008D940F2A361074805F06EFD636A1D4349
:1014B000656270BD002EF9D1636A23EA0505F7E77E
:1014C000CC8608F33CD80108003802400E4B03409C
:1014D00070B505460E4603B920B940F2D3610B48FA
:1014E00005F052FD012E0A4C08D940F2D46107489C
:1014F00005F04AFD236D1D43256570BD002EF9D111
:10150000236D23EA0505F7E7006810813CD8010840
:101510000038024030F0F10370B505460E4600D1A8
:1015200020B940F2F3610A4805F02EFD012E094C66
:1015300008D940F2F461064805F026FD636D1D43AD
:10154000656570BD002EF9D1636D23EA0505F7E7E7
:101550003CD801080038024030F0030370B505465E
:101560000E4600D120B94FF4E2610A4805F00CFDA7
:10157000012E094C08D940F21171064805F004FD0E
:10158000A36D1D43A56570BD002EF9D1A36D23EA9F
:101590000505F7E73CD801080038024010F4585F11
:1015A00070B505460E4600D120B940F247710A4891
:1015B00005F0EAFC012E094C08D94FF4E961064810
:1015C00005F0E2FC236E1D43256670BD002EF9D1A7
:1015D000236E23EA0505F7E73CD8010800380240EE
:1015E0000E4B034070B505460E4603B920B940F2D4
:1015F00075710B4805F0C8FC012E0A4C08D940F261
:101600007671074805F0C0FC636E1D43656670BDCA
:10161000002EF9D1636E23EA0505F7E7CC8008F3C5
:101620003CD801080038024030F0180310B50446D9
:1016300004D040F28E71064805F0A6FC054B1A6FE7
:1016400022F018021A67186F2043186710BD00BFF8
:101650003CD8010800380240012810B5094C09D9CE
:1016600040F29F71084805F08FFCD4F8903023F0C9
:10167000006304E0F9D1D4F8903043F00063C4F87B
:10168000903010BD003802403CD80108012810B548
:10169000094C09D940F2B671084805F075FCD4F838
:1016A000903023F0805304E0F9D1D4F8903043F027
:1016B0008053C4F8903010BD003802403CD8010877
:1016C000012810B5094C09D940F2CD71084805F040
:1016D0005BFCD4F8903023F0806304E0F9D1D4F8B7
:1016E000903043F08063C4F8903010BD0038024061
:1016F0003CD8010838B531F4803305460C4607D094
:10170000B1F5003F04D040F2ED71254805F03CFCF6
:10171000244B9D4212D003F580639D4227D003F5F0
:1017200080639D422FD003F580639D4213D040F229
:10173000EE711B48BDE8384005F026BC1A4BD3F8C3
:10174000902022F44032C3F89020D3F89020144324
:10175000C3F8904038BD144BD3F8902022F44002D7
:10176000C3F89020D3F8902042EA8414F0E70E4B9F
:10177000D3F8902022F44022C3F89020D3F8902090
:1017800042EA8404E4E7084BD3F8902022F44012A4
:10179000C3F89020D3F8902042EA0414D8E700BFA1
:1017A0003CD80108005400400038024038B531F4FC
:1017B000803305460C4607D0B1F5003F04D040F613
:1017C0002701454805F0E0FB444B9D4222D0A3F59C
:1017D0004C439D424FD003F580639D4233D003F5C7
:1017E0004C439D425FD0A3F548439D4237D003F55B
:1017F00080639D424BD003F520539D425FD003F59B
:1018000080639D4213D040F628013348BDE838403C
:1018100005F0BABB324BD3F8902022F00302C3F894
:101820009020D3F890201443C3F8904038BD2C4B3F
:10183000D3F8902022F44042C3F89020D3F89020AF
:1018400042EA8434F0E7264BD3F8902022F03002AD
:10185000C3F89020D3F8902042EA0414E4E7204B28
:10186000D3F8902022F0C002C3F89020D3F8902043
:1018700042EA8414D8E71A4BD3F8902022F00C02E5
:10188000C3F89020D3F8902042EA8404CCE7144BAC
:10189000D3F8902022F44072C3F89020D3F890201F
:1018A00042EA0424C0E70E4BD3F8902022F44062B1
:1018B000C3F89020D3F8902042EA8424B4E7084B80
:1018C000D3F8902022F44052C3F89020D3F890200F
:1018D00042EA0434A8E700BF3CD8010800100140E8
:1018E0000038024038B531F0407305460C4604D04C
:1018F00040F674010C4805F047FB0C4B9D4206D0A6
:1019000040F675010848BDE8384005F03DBB084B7E
:10191000D3F8902022F04072C3F89020D3F89010B2
:101920002143C3F8901038BD3CD801080024004082
:101930000038024043B2002B70B505460E4604DC69
:1019400040F6A3010A4805F01FFB012E094C08D9F7
:1019500040F6A401064805F017FB207828432070C4
:1019600070BD002EF9D1207820EA0500F7E700BF0E
:101970003CD801080D380240A0F12103DBB21C2B3A
:1019800010B504460DD900F0DF03412B0ED0A4F1B1
:101990007903062B0AD940F6CC010D4805F0F4FA7C
:1019A00004E00C4A22FA03F3DB07F0D562090A4B84
:1019B000012A06D1186804F01F04E04000F001007D
:1019C00010BD022A01D1186FF5E7586FF3E700BF89
:1019D0003CD80108010001150038024013B500236E
:1019E00041F2883401933120FFF7C6FF019B013398
:1019F0000193019BA34201D00028F4D03120FFF7CE
:101A0000BBFF003018BF012002B010BD024A536F67
:101A100043F080735367704700380240431EDBB2C7
:101A20001F2B10B504460AD9802801D040280BD1BD
:101A3000084BDB681C4214BF0120002010BD064A81
:101A400022FA03F3DB07F3D440F60B11034805F049
:101A50009BFAEDE7003802408B8000803CD80108FB
:101A600010B5044620B940F62B11034805F08CFA56
:101A7000024B1C7010BD00BF3CD801080E3802405C
:101A800030B5046A42EA031324F001040462856954
:101A9000046A25F0F30524F00A042B430C43836108
:101AA00044F00104046230BD30B5046A120224F02F
:101AB000100442EA033304628569046A25F473451D
:101AC00024F0A0042B4344EA0114836144F0100481
:101AD000046230BD08B5584B98423CD0B0F1804FFD
:101AE00078D0A3F57C4398427BD003F5806398427D
:101AF0007ED003F58063984200F0818003F5806317
:101B0000984200F0838003F58063984200F085805E
:101B100003F57043984200F0878003F570539842B4
:101B200023D003F58063984228D003F58063984260
:101B30002DD0A3F59833984232D003F580639842B4
:101B400038D003F5806398423BD056213B48BDE82E
:101B5000084005F019BA01210846FFF793FC00215F
:101B60000120BDE80840FFF78DBC01214FF4803013
:101B7000FFF788FC00214FF48030F2E701214FF499
:101B80000030FFF77FFC00214FF40030E9E701212E
:101B90004FF48020FFF776FC00214FF48020E0E72F
:101BA00001214020FFF74CFC00214020BDE8084007
:101BB000FFF746BC01218020FFF742FC0021802076
:101BC000F4E701214FF48070FFF73AFC00214FF455
:101BD0008070EBE701210846FFF732FC002101206D
:101BE000E4E701210220FFF72BFC00210220DDE7C2
:101BF00001210420FFF724FC00210420D6E7012165
